:020000040800F2
:10000000506100203103000815340008C1280008A1
:1000100011340008F50E0008FB6200080000000023
:10002000000000000000000000000000790200084D
:10003000B515000800000000CD020008CD490008F9
:100040004B0300084B0300084B0300084B03000858
:100050004B0300084B0300084B0300084B03000848
:100060004B0300084B0300084B0300084B03000838
:100070004B0300084B0300084B0300084B03000828
:100080004B0300084B0300084B0300084B03000818
:10009000251100084B0300084B0300084B03000820
:1000A0004B0300084B0300084B0300084B030008F8
:1000B000754E00088D4E0008A54E00084B03000841
:1000C0004B0300084B0300084B0300084B030008D8
:1000D0004B030008815B0008F55C0008E55F000841
:1000E0004B0300084B0300084B030008D54E0008E3
:1000F000E95300084B030008ED4E00084B030008CD
:100100004B0300084B030008BD4E00084B030008DA
:100110004B030008515A00084B0300084B0300082A
:100120004B0300084B0300084B0300084B03000877
:100130004B0300084B0300084B0300084B03000867
:100140004B0300084B0300084B0300084B03000857
:100150004B0300084B0300084B0300084B03000847
:100160004B0300084B0300084B0300084B03000837
:100170004B0300084B0300084B0300084B03000827
:100180004B0300084B03000800F002F800F064F88D
:100190000AA090E8000C82448344AAF10107DA45E2
:1001A00001D100F059F8AFF2090EBAE80F0013F0D0
:1001B000010F18BFFB1A43F0010318472CDF0000A2
:1001C0004CDF00000A444FF0000C10F8013B13F024
:1001D000070408BF10F8014B1D1108BF10F8015BA0
:1001E000641E05D010F8016B641E01F8016BF9D193
:1001F00013F0080F1EBF10F8014BAD1C0C1B09D1EA
:100200006D1E58BF01F801CBFAD505E014F8016B5B
:1002100001F8016B6D1EF9D59142D6D370470000ED
:100220000023002400250026103A28BF78C1FBD8FF
:10023000520728BF30C148BF0B607047642900F0E7
:100240000381732900F03E82002070471FB50CF037
:100250004EFB1FBD10B510BD00F0B0FA1146FFF700
:10026000F5FF08F08DF900F0CEFA03B4FFF7F2FFC6
:1002700003BC07F0B1FD00002A4B19680868B0E81C
:10028000F04F80F30988BFF36F8F4FF0000080F3C9
:10029000118870470000000006480068006880F37D
:1002A000088862B661B6BFF34F8FBFF36F8F00DF70
:1002B00000BF00BF08ED00E0DFF80C00016841F46A
:1002C00070010160704700BF88ED00E0EFF3098026
:1002D000BFF36F8F134B1A681EF0100F08BF20ED8D
:1002E000108A20E9F04F106008B44FF0500080F3FE
:1002F0001188BFF34F8FBFF36F8F0AF085FD4FF06A
:10030000000080F3118808BC19680868B0E8F04F55
:100310001EF0100F08BFB0EC108A80F30988BFF3FD
:100320006F8F7047E8000020EFF3058070470000F2
:100330000948804709480047FEE7FEE7FEE7FEE779
:10034000FEE7FEE7FEE7FEE7FEE7FEE704480549B5
:10035000054A064B70470000DD4900088901000886
:10036000505B002050610020505D0020505D002057
:10037000704700000FB4044910B503AA029800F0BA
:10038000A5F910BC5DF814FBD00000202DE9F04168
:100390000E460446002020622046E168884730B3BC
:1003A000252805D0D4E901219047206A401CF2E7B6
:1003B000E168204600278847050018D0A5F14100D4
:1003C000192802D820354FF40067324629462046C6
:1003D0002760FFF733FF40B1012804D0F61D26F057
:1003E00007060836D8E7361DD6E72846DAE7206A3A
:1003F000BDE8F08170B50C460546012A05D0287885
:10040000800600D5EA69002302E0012305E05B1CB9
:10041000934202D2E05C0028F9D1A869E618C01A1C
:10042000A861286A184428622846AFF3008004E0D7
:10043000D5E9012114F8010B9047B442F8D32846BE
:10044000AFF3008070BD00002DE9F04106460024A6
:1004500010687529314616A510D0AFF3008000282A
:1004600002DA404213A507E031688A0701D512A5D8
:1004700002E0490704D511A5012401E0AFF3008093
:1004800000210A2206F1240709E0B0FBF2FCB0FBD0
:10049000F2F302FB1C00303078541846491C002847
:1004A000F3D123462A463046BDE8F04100F086B835
:1004B000000000002D0000002B00000020000000C4
:1004C000032A40F2308010F0030C00F0158011F880
:1004D000013BBCF1020F624498BF11F801CB00F858
:1004E000013B38BF11F8013BA2F1040298BF00F8AC
:1004F00001CB38BF00F8013B11F0030300F0F88096
:10050000083AC0F0088051F8043B083A51F804CB8F
:10051000A0E80810F5E7121D5CBF51F8043B40F855
:10052000043BAFF30080D20724BF11F8013B11F860
:1005300001CB48BF11F8012B24BF00F8013B00F8A4
:1005400001CB48BF00F8012B704702F0FF0343EADC
:10055000032242EA024200F002B84FF000020429EE
:10056000C0F0128010F0030C00F0F680CCF1040C07
:10057000BCF1020F18BF00F8012BA8BF20F8022B16
:10058000A1EB0C0100F0E8B85FEAC17C24BF00F8E1
:10059000012B00F8012B48BF00F8012B7047704772
:1005A00070477047704710B500F0FCF8006810BD48
:1005B00010B5044600F0F6F8046010BD2DE9F047D0
:1005C0000D4699469246044600F1240801688806C3
:1005D00004D5E06921F01001216000E00120A8426B
:1005E00001DD471B00E00027A1697A1902EB090031
:1005F000081AA0612078C00602D42046AFF300801C
:10060000002608E0D4E901211AF806009047206A84
:10061000401C761C20624E45F4DB2078C0060AD5CB
:100620002046AFF3008006E0D4E901213020904756
:10063000206A401C2062381EA7F10107F4DC07E0A5
:10064000D4E9012118F805009047206A401C206277
:10065000281EA5F10105F3DC2046AFF300802078C9
:10066000000602D50220BDE8F0870120FBE700006C
:1006700001694A1C02610878704700B58FB0CDE966
:1006800001310021059105497944CDE90310114656
:100690006846FFF77BFE0FB000BD0000E5FFFFFFDF
:1006A00010B5436913B1AFF3008001E0FFF7A2FE7C
:1006B000012010BD127800F124010A7000224A7056
:1006C0000122EDE711684FF0FF32E9E7074B70B503
:1006D0000D467B44FFF7D1FF0446284600F066F83C
:1006E00010B14FF0FF3070BD204670BD4F7E00004E
:1006F00010B5203AC0F00B80B1E81850203AA0E8BD
:100700001850B1E81850A0E81850BFF4F5AF5FEAF0
:10071000027C24BFB1E81850A0E8185044BF18C9A3
:1007200018C0BDE810405FEA827C24BF51F8043B4A
:1007300040F8043B08BF7047D20728BF31F8023B9E
:1007400048BF11F8012B28BF20F8023B48BF00F832
:10075000012B70474FF0000200B5134694469646B1
:10076000203922BFA0E80C50A0E80C50B1F12001C4
:10077000BFF4F7AF090728BFA0E80C5048BF0CC072
:100780005DF804EB890028BF40F8042B08BF7047D0
:1007900048BF20F8022B11F0804F18BF00F8012B42
:1007A0007047000000487047EC5A0020007B00F0C2
:1007B0008000704700487047EC5A00207546FFF7EC
:1007C000F9FFAE4605006946534620F0070085460E
:1007D00018B020B5FFF7BAFDBDE820404FF0000685
:1007E0004FF000074FF000084FF0000B21F0070119
:1007F000AC46ACE8C009ACE8C009ACE8C009ACE85C
:10080000C0098D46704710B50446AFF300802046FE
:10081000BDE81040FFF729BD21B1826842F0010216
:10082000826003E0826822F001028260704700006B
:100830000021084A1168084A1140D0E900231A43F0
:1008400083681A43C3681A431143044AC2F8041365
:100850007047000004230140E030FCFF002001400D
:100860000146C86C80B270470246002013680B40F6
:100870000BB1012000E000207047000030B50246B7
:10088000002000235068104C20400D790C6844EA89
:1008900005242043506090680C4C2040D1E903545B
:1008A0002C438D682C434D7944EA450420439060E5
:1008B000D06A20F470000C7D641EE4B2234340EA49
:1008C0000350D06230BD0000FFFEFFFCFDF7FFC00B
:1008D000F0B504460D4600200021092D11DDE06829
:1008E000A5F10A0606EB4607072606FA07F1884334
:1008F000A5F10A0606EB460603FA06F10843E06096
:100900000CE0206905EB4507072606FA07F1884346
:1009100005EB450603FA06F108432061072A0FDAC2
:10092000606B561E06EB86071F2606FA07F1884302
:10093000561E06EB860605FA06F10843606322E0C0
:100940000D2A0FDA206BD61F06EB86071F2606FA44
:1009500007F18843D61F06EB860605FA06F1084321
:10096000206310E0E06AA2F10D0606EB86071F2661
:1009700006FA07F18843A2F10D0606EB860605FA92
:1009800006F10843E062F0BD816841F0804181607A
:1009900070470000F8B53848D0ED000A9FED371ACF
:1009A0009FED370A10EE810AF3EE0B0A80EE201A53
:1009B000BDEEC10A10EE106A642E00DD64263148D7
:1009C00090ED000ADFED300A20EE200ABDEEC00AED
:1009D00010EE104A002C00DA64422C4890ED000A18
:1009E000DFED290A20EE200ABDEEC00A10EE105AF3
:1009F000002D00DA6D422648007808B9012000E099
:100A00000020234908702348007801281BD1224880
:100A100090ED000ABDEEC00A10EE103A1F4890EDAE
:100A2000000ABDEEC00A10EE102A1D4890ED000A23
:100A3000BDEEC00A10EE101A1AA0FFF79BFC0020B2
:100A40001449087017E01248007850B91948B0F9F5
:100A50000400EAB2E1B23346009017A0FFF78AFC27
:100A600009E01448B0F90430B0F90220B0F90010E0
:100A700015A0FFF77FFCF8BD1800002000007A44A5
:100A800000401C46745A00200000C842885A0020CA
:100A90002C020020A2010020800100207C01002007
:100AA0006C0100207B4325643A25643A25647D244B
:100AB00000000000300200207B4125643A25643AA2
:100AC00025643A25647D24007B4225643A25643AF6
:100AD00025647D240000000000B58DB001210220B6
:100AE00003F052FA0121080203F06EFA02200B9083
:100AF00003208DF8300000208DF833000BA9154835
:100B000001F004FB0121080203F06EFA00214FF40A
:100B1000807003F069FA002007900A9009904FF462
:100B20000030089007A8FFF783FE002001908DF8A1
:100B300008008DF809000390059001208DF8180039
:100B400001A90548FFF79AFE01210348FFF764FE5B
:100B50000DB000BD000402400020014000B58DB082
:100B60000121022003F010FA0121480203F02CFABF
:100B700001200B9003208DF8300000208DF8330009
:100B80000BA9154801F0C2FA0121480203F02CFA22
:100B900000214FF4007003F027FA002007900A901C
:100BA00009904FF40030089007A8FFF741FE00209D
:100BB00001908DF808008DF8090003900590012040
:100BC0008DF8180001A90548FFF758FE01210348D8
:100BD000FFF722FE0DB000BD0004024000210140DD
:100BE0001CB507F0ADFC019063E10A2101A809F0F2
:100BF000DDFEB048006840F6B831884204DAAD48FE
:100C00000068401CAB49086001F0EEFCAA4800688F
:100C10000028E9D1A948007810B101F015FB16E0D1
:100C2000A748007810B103F0ABFA10E0A5480078AF
:100C300010B103F073F80AE0A34890ED001AA3483E
:100C4000D0ED000AA24890ED000A00F0B5FC02F0D9
:100C50007BF9A04890ED000ABDEEC00A10EE100A24
:100C600004F0CEFE002879D19B4890ED021AF0EEF8
:100C7000410A90ED001AB0EE410A01F0EDFF00EEDE
:100C8000100AB8EEC00A944880ED010A934890ED2E
:100C9000021AF0EE410A90ED001AB0EE410A02F09D
:100CA00033F800EE100AB8EEC00A8C4880ED010A55
:100CB0008B4890ED021AF0EE410A90ED001AB0EE6A
:100CC000410A02F079F800EE100AB8EEC00A844832
:100CD00080ED010A834890ED021AF0EE410A90ED92
:100CE000001AB0EE410A02F0BFF800EE100AB8EEAA
:100CF000C00A7C4880ED010A44F23C1002F060F921
:100D000079480078062828D2DFE800F003294E64ED
:100D100085AA0020734C009094ED010ABDEEC00A34
:100D200010EE103A6E4C94ED010AB1EE400ABDEEA1
:100D3000C00A10EE102A694C94ED010AB1EE400A87
:100D4000BDEEC00A10EE101A634C94ED010ABDEE20
:100D5000C00A10EE100A03F0F9FCA2E0A2E00020A5
:100D6000604C009094ED010ABDEEC00A10EE103AFE
:100D70005B4C94ED010AB1EE400ABDEEC00A10EEE4
:100D8000102A564C94ED010ABDEEC00A10EE101A5E
:100D9000514C94ED010AB1EE400ABDEEC00A10EECE
:100DA000100A03F0D3FC7CE0504800684B4A0090E6
:100DB00092ED010ABDEEC00A10EE101A464A92EDFD
:100DC000010ABDEEC00A10EE100A494B5A4203F068
:100DD000BDFC66E00020434C009094ED010ABDEE9E
:100DE000C00A10EE103A3E4C94ED010ABDEEC00A66
:100DF00010EE102A394C94ED010ABDEEC00A10EE37
:100E0000101A354C94ED010ABDEEC00A10EE100A1E
:100E100003F09CFC45E00020324C009094ED010A68
:100E2000BDEEC00A10EE103A2D4C94ED010AB1EE61
:100E3000400ABDEEC00A10EE102A284C94ED010ABB
:100E4000B1EE400ABDEEC00A10EE101A224C94ED2D
:100E5000010ABDEEC00A10EE100A03F077FC20E094
:100E60000020204C009094ED010ABDEEC00A10EE67
:100E7000103A1B4C94ED010ABDEEC00A10EE102A88
:100E8000164C94ED010ABDEEC00A10EE101A124C79
:100E900094ED010ABDEEC00A10EE100A03F056FCF4
:100EA00000BF06E00020034602460146009003F022
:100EB0004DFC9AE6D4010020B801002099010020E1
:100EC0009A01002098010020780100207401002080
:100ED0007001002018000020745A0020885A002059
:100EE0009C5A0020B05A00206401002068010020B4
:100EF00061BEFFFF00BFFEE71CB50121084603F0FD
:100F000043F84FF48070009001208DF80400002019
:100F10008DF8060003208DF8050001208DF80700EC
:100F20006946024801F0F2F81CBD000000000240D2
:100F30002DE9FE4304460D4616461F46DDF828906F
:100F40004FF0000814B10DB106B117B90120BDE88A
:100F5000FE83601EC4B2681EC5B2701EC6B2781E83
:100F600087B20121082003F00FF80121480603F0A1
:100F70001BF80320019002208DF8080000208DF856
:100F80000A0003208DF8090001208DF80B0001A94B
:100F9000614801F0BBF8092200215F4801F0FEF82A
:100FA000092201215C4801F0F9F800205B49086042
:100FB0000846006840F00100086008E008F1010000
:100FC0001FFA80F8B8F1640F01DD0220BFE7534833
:100FD000001D006800F001000028EFD04F480068B5
:100FE0004E490860084600680860084600680860C6
:100FF0000846006840F01000086008460068086075
:10100000084600680860002044491C310860084612
:10101000006840EA897008600846006840EA046099
:1010200008600846006840EA055008600846006805
:1010300040EA0640086008460068384308603748C0
:10104000006820F001003549086009E008F101005E
:101050001FFA80F84FF6F070804501DD032076E737
:101060002E48001D006800F001000028EED12C4839
:10107000006840F001002A49086029481C300068D7
:1010800020F0010026491C31086025480C3000681A
:1010900040F0010022490C3108602148001D006821
:1010A0001F49091D08601E48143000681C4914318E
:1010B000086000201A494031086000211848443077
:1010C000016017481C30006840F0010014491C31D1
:1010D0000860134800680020114908600F48143068
:1010E000006840F002000D491431086014208DF8AA
:1010F000000001208DF8010003208DF8020001207E
:101100008DF80300684602F087F9012202210348A6
:1011100000F0F2F900201AE7000C024000640040E1
:101120000066004000B52DED028B89B003A805A92B
:1011300006AB07AACDE9001008A9002000F088F846
:1011400040F281110898884266D101203449087024
:101150000020344908703449087034490870344913
:10116000087034490870344908709DF80D009DF8E6
:101170000C1000EB012000B200EE100AB8EEC00A1D
:10118000DFED2E0A80EE201A2D4880ED001A9DF822
:101190000F009DF80E1000EB012000B200EE100AC7
:1011A000B8EEC00ADFED250A80EE201A254880ED52
:1011B000001A9DF811009DF8101000EB012000B2FC
:1011C00000EE100AB8EEC00ADFED1C0A80EE201A0D
:1011D000B0EE418A1C48007802280AD1F0EE480A95
:1011E000174890ED000A05F08BF8184880ED000ACA
:1011F00011E09DF811009DF8101000EB012000B2E5
:1012000000EE100AB8EEC00ADFED0C0A80EE201ADC
:101210000E4880ED001A00BF09B0BDEC028B00BD86
:101220009B010020980100209A01002099010020D4
:101230009C0100209D010020DE01002000007A4476
:10124000700100207401002064010020780100205A
:10125000F0B5DDE90554324E06EB0016366806F0AF
:1012600004061670167836B92D4E06EB0016366851
:10127000760D0E6005E02A4E06EB00163668F6087D
:101280000E60274E06EB0016366806F002061E704A
:10129000234E06EB0016766806F00F062E70204EE1
:1012A00006EB0016B66826701D4E06EB0016B668F3
:1012B000360A66701A4E06EB0016B668360CA67033
:1012C000174E06EB0016B668360EE670144E06EBA7
:1012D0000016F6682671124E06EB0016F668360AFE
:1012E00066710F4E06EB0016F668360CA6710C4EB2
:1012F00006EB0016F668360EE67130B9094E366810
:1013000046F02006074F3E6009E0012807D1054E50
:10131000361D366846F02006024F3F1D3E60F0BD88
:10132000B06500400C640040F8B506460D46002448
:101330000823002211463046009500F015F80746B4
:1013400001E0601C84B2384600F094F8072803D00E
:1013500040F6FF708442F4DB40F6FF70844201DB0C
:101360000120F8BD0020FCE7F0B505460E46059CBF
:101370003E48006800F0806008B100210FE03B4863
:10138000006800F0006008B1012108E037480068FB
:1013900000F0805008B1022101E0FF20F0BD0027DD
:1013A000334800EB011007601EB9C5F30A056D054F
:1013B00002E025F06045ED002D4800EB01100068CB
:1013C00028432B4F07EB01173860294800EB011029
:1013D000006840EA8607264800EB011007602448B1
:1013E00000EB0110006840EA4207214800EB0110C1
:1013F000076003F00F031E4800EB0110406820F067
:101400000F071B4800EB01104760194800EB011063
:1014100040681843164F07EB01177860E079000623
:10142000A77940EA0740677940EA07272079074310
:101430000F4800EB0110C760E0780006A77840EA8B
:101440000740677840EA072027783843084F07EBC2
:101450000117B860064800EB0110006840F0010772
:10146000034800EB01100760084697E70864004056
:10147000806500400146002021B1012913D00229D6
:1014800033D121E01B4A126802F001021043194ACD
:10149000126802F002021043164A126802F08062DB
:1014A00040EA126023E0134A126802F0010210437E
:1014B000104A126802F0020210430E4A126802F04B
:1014C000006240EA526012E00A4A126802F0010229
:1014D0001043084A126802F002021043054A1268DB
:1014E00002F0805240EA926001E0052000BF00BF98
:1014F00070470000086400401AB143690B43436120
:1015000002E043698B434361704700001CB500242F
:1015100005E01848005D0DF80400601CC4B2082CFA
:10152000F7DB694640F20110FFF7FEFE002407E0FA
:10153000104904F10800085C0DF80400601CC4B2F6
:10154000082CF5DB69464FF48170FFF7EDFE0024AF
:1015500007E0084904F11000085C0DF80400601C65
:10156000C4B2082CF5DB694640F20310FFF7DCFE3D
:101570001CBD00008C06002010B502460B46002062
:10158000012B08D1002104E0084C645C60404C1C35
:10159000E1B29142F8DB43B9002104E0044C645C01
:1015A00060404C1CE1B29142F8DB10BD8C0600207B
:1015B000BC0600207047000000B52DED108B89B0EF
:1015C000B0EE408AF0EE609AF0EE418AB0EE0C0A7E
:1015D000B0EE409AFC48007818B1FB48007801282A
:1015E00014D1B0EE681AF0EE690AB0EE480A03F0C2
:1015F000FBF8F64890ED000AB0EE408A90ED010A43
:10160000F0EE409A90ED020AF0EE408AEE48007843
:10161000002879D139EE880AED48D0ED000AED486E
:1016200090ED001A70EE810A08EEE00AEA4880EDBB
:10163000020AB1EE690A30EE080AE548D0ED000A68
:10164000E44890ED001A70EE810A08EEE00AE348E3
:1016500080ED020A39EE880ADD48D0ED000ADD4847
:1016600090ED001A70EE810A08EEA00ADC4880EDC9
:10167000020AB1EE690A30EE080AD548D0ED000A38
:10168000D44890ED001A70EE810A08EEA00AD54801
:1016900080ED020AD048D0ED020AB0EE600AB0EE4A
:1016A000491AF1EE490A08F0CAFDCB4880ED020A5A
:1016B000CA48D0ED020AB0EE600AB0EE491AF1EE67
:1016C000490A08F0BCFDC54880ED020AC448D0EDC7
:1016D000020AB0EE600AB0EE491AF1EE490A08F0CB
:1016E000AEFDBF4880ED020ABE48D0ED020AB0EE62
:1016F000600AB0EE491AF1EE490A08F0A0FDB948B7
:1017000080ED020A38E3FFE7AF48007801287AD17C
:10171000B548D0ED000AB0EE690A00EEA80AAE485E
:1017200080ED020AB04890ED000A20EE280A10EE83
:10173000101A08460BF06AF841EC1B0BB6EE000AD3
:1017400029EE800A10EE101A08460BF05FF8CDE97A
:10175000040118EE100A0BF059F841EC1C0B9FED38
:10176000A30B05F01DFEB0EE40FAF0EE60FA9FED1F
:10177000A10B53EC102B51EC1F0B0AF063FB41EC57
:101780001D0B0AF065FA41EC1E0B53EC1C2B0AF002
:1017900047FDCDE902019DED040B53EC102B9DEDAF
:1017A000020B51EC100B0AF047FF53EC1B2BCDE959
:1017B00006019DED060B51EC100B0AF087FA41EC87
:1017C0001A0B0AF051FA85498860874890ED000AA3
:1017D00020EE280A10EE101A08460BF017F841EC1C
:1017E0001B0BB6EE000A29EE800A10EE101A08460E
:1017F0000BF00CF841EC1C0B18EE100A0BF006F87D
:1018000041EC1D0B00E05BE09FED780B05F0C8FD9F
:101810008DED040B9FED770B53EC102B9DED040B1E
:1018200051EC100B0AF00EFB53EC1D2BCDE9060119
:101830009DED060B51EC100B0AF0F2FC41EC1F0B76
:1018400053EC1C2B0AF0F8FE41EC1E0B53EC1B2B47
:101850000AF03CFA41EC1A0B0AF006FA604988607B
:101860005D48D0ED020AB0EE600AB0EE491AF1EE22
:10187000490A08F0E4FC584880ED020A5748D0EDC8
:10188000020AB0EE600AB0EE491AF1EE490A08F019
:10189000D6FC524880ED020A5148D0ED020AB0EE63
:1018A000600AB0EE491AF1EE490A08F0C8FC4C484B
:1018B00080ED020A9FED510A4A4880ED020A5BE280
:1018C0004148007802287DD19FED4D0AF0EE40DAC4
:1018D000B0EE68AA3F4890ED000AF6EE000A20EE4E
:1018E000200A10EE101A08460AF090FF41EC1B0B7C
:1018F0001AEE100A0AF08AFFCDE904019DED040BEF
:1019000005F08EFDB0EE40EAF0EE60EA3048006887
:101910000AF07CFF41EC1F0B53EC1E2B0AF092FAED
:1019200041EC1C0B53EC1B2B0AF086FECDE90601A3
:101930009DED060B51EC100B0AF096F90AEE900A99
:101940009FED301ADFED300AB0EE4A0A08F077FC5E
:10195000B0EE40AAB5EEC0AAF1EE10FA20D01D48B4
:10196000D0ED000AB6EE001AB0EE6A0A01EE600A87
:1019700020EE080AC0EE2A0A1748C0ED020A1548F0
:10198000D0ED000AB6EE001AB0EE6A0A01EE200AA7
:1019900020EE080AC0EE2A0A1048C0ED020A05E04F
:1019A0000D4880ED028A0D4880ED028A9FED170AEE
:1019B0002AEE000A10EE101A08460AF027FF41EC42
:1019C0001E0B25E0C0E0000064010020685A0020E2
:1019D000900100208C010020745A0020885A0020B9
:1019E0009C5A0020B05A0020940100200000000002
:1019F000000008400000000000000040000000005F
:101A0000D7231F449A99193F9A9919BFE5D0E23F0D
:101A10001AEE100A0AF0FAFE41EC1C0B1FED0B1B2C
:101A2000B0EE4C0AF0EE6C0A04F092FEB0EE40BA52
:101A3000F0EE60BA9FEDD20B53EC102B51EC1B0B68
:101A40000AF0EEFBCDE902011AEE100A0AF0DEFE02
:101A500041EC1B0B1FED1B1BB0EE4B0AF0EE6B0AAB
:101A600004F076FEB0EE40CAF0EE60CA9FEDC60B01
:101A700053EC102B51EC1C0B0AF0D2FBCDE900010A
:101A80009DED020B53EC102B9DED000B51EC100B58
:101A90000AF01CF941EC1F0B53EC1E2B0AF0CCFD95
:101AA0009FEDBB0B53EC102BCDE904019DED040B16
:101AB00051EC100B0AF00AF9CDE906019DED060B79
:101AC00051EC100B0AF0D0F80DEE100A9FEDB20A9F
:101AD0007DEE400A9FEDB10A00EEAD0ABDEEC00AF0
:101AE000AF4880ED000AAF48D0ED020AB0EE600AC0
:101AF000B0EE491AF1EE490A08F0A1FBA94880EDC1
:101B0000020AA948D0ED020AB0EE600AB0EE491A06
:101B1000F1EE490A08F093FBA34880ED020A1FED9D
:101B2000490AA24880ED020A1FED4C0AA04880ED48
:101B3000020A40F698024FF448719948006808F08C
:101B400093FB9749086017E19A480078032842D12F
:101B5000994890ED000A68EE800AB0EE001A80EE17
:101B6000810A38EE400A8F4880ED020A924890EDD3
:101B7000000A68EE800AB0EE001A80EE810A30EEAC
:101B8000080A894880ED020A8648D0ED020AB0EEC4
:101B9000600AB0EE491AF1EE490A08F050FB81489C
:101BA00080ED020A8048D0ED020AB0EE600AB0EE85
:101BB000491AF1EE490A08F042FB7B4880ED020A1F
:101BC0001FED720A794880ED020A1FED740A784809
:101BD00080ED020AD0E07748007804287DD176486D
:101BE00090ED000A7548D0ED000A30EE200A60EE54
:101BF000280AB0EE001A80EE810A38EE400A6948E1
:101C000080ED020A6C4890ED000A6C48D0ED000AA5
:101C100030EE200A60EE280AB0EE001A80EE810A4B
:101C200038EE400A604880ED020A634890ED000AF1
:101C30006248D0ED000A30EE200A60EE280AB0EECD
:101C4000001A80EE810A30EE080A584880ED020A38
:101C5000594890ED000A5948D0ED000A30EE200AAC
:101C600060EE280AB0EE001A80EE810A30EE080A13
:101C70004F4880ED020A4B48D0ED020AB0EE600AF0
:101C8000B0EE491AF1EE490A08F0D9FA454880ED5C
:101C9000020A4548D0ED020AB0EE600AB0EE491AD9
:101CA000F1EE490A08F0CBFA3F4880ED020A3F48BE
:101CB000D0ED020AB0EE600AB0EE491AF1EE490A20
:101CC00008F0BDFA394880ED020A3948D0ED020A21
:101CD000B0EE600AB0EE491A00E007E0F1EE490A02
:101CE00008F0ADFA324880ED020A45E0314800784C
:101CF000052841D1304890ED000A68EE800AB0EE28
:101D0000001A80EE810A38EE400A264880ED020A69
:101D1000294890ED000A68EE800AB0EE001A80EEC5
:101D2000810A30EE080A204880ED020A1D48D0EDF5
:101D3000020AB0EE600AB0EE491AF1EE490A08F064
:101D40007EFA184880ED020A1748D0ED020AB0EE7C
:101D5000600AB0EE491AF1EE490A08F070FA12482A
:101D600080ED020A1FEDDB0A104880ED020A1FED2C
:101D7000DD0A0F4880ED020A09B0BDEC108B00BDF2
:101D800000000000D34DF43F000000809318E4BF32
:101D900000000000022BF93F4C37C93F0000C84447
:101DA00068010020745A0020885A00209C5A0020A4
:101DB000B05A0020640100208C0100209001002016
:101DC0001CB50121082002F0DFF808200090002057
:101DD0008DF8040003208DF8050001208DF8070020
:101DE0006946024800F092F91CBD0000000C024058
:101DF00000B589B00121084602F0D6F80121032080
:101E000002F0C2F84FF40040019003208DF8090061
:101E100002208DF8080001208DF80A008DF80B00D3
:101E200001A92B4800F072F90820019003208DF8D9
:101E3000090002208DF8080001208DF80A008DF8B5
:101E40000B0001A9234800F061F901220F2120486D
:101E500000F0A4F9012203211E4800F09FF906A812
:101E600003F0C4FD0020ADF818004FF6FF70079096
:101E70000020ADF82000ADF81A0006A94FF0804010
:101E800003F072FD00231A4603214FF0804003F057
:101E90003EFB03A803F0B0FB0020ADF8140003A93B
:101EA0004FF0804003F071FB0121880703F00EFB27
:101EB00001221146900703F0A8FB00214FF080405B
:101EC00003F024FD0121880703F006FB09B000BDE3
:101ED000000002400004024000B589B00121022048
:101EE00002F062F80121022002F04EF83020019049
:101EF00003208DF8090002208DF8080001208DF8DC
:101F00000A008DF80B0001A9204800F0FFF802221A
:101F100004211E4800F042F9022205211B4800F06E
:101F20003DF906A803F062FD0020ADF818004FF659
:101F3000FF7007900020ADF82000ADF81A0006A948
:101F4000134803F011FD00231A460321104803F043
:101F5000DEFA03A803F050FB0020ADF8140003A93B
:101F60000B4803F012FB0121094803F0AFFA0122EC
:101F70001146074803F049FB0021054803F0C6FC61
:101F80000121034803F0A8FA09B000BD0004024093
:101F90000004004000B589B00121042002F004F8DB
:101FA0000121022001F0F0FFC020019003208DF8F4
:101FB000090002208DF8080001208DF80A008DF834
:101FC0000B0001A9204800F0A1F8022206211E48BA
:101FD00000F0E4F8022207211B4800F0DFF806A811
:101FE00003F004FD0020ADF818004FF6FF700790D5
:101FF0000020ADF82000ADF81A0006A9134803F040
:10200000B3FC00231A460321104803F080FA03A80A
:1020100003F0F2FA0020ADF8140003A90B4803F016
:10202000B4FA0121094803F051FA01221146074888
:1020300003F0EBFA0021054803F068FC0121034896
:1020400003F04AFA09B000BD000402400008004055
:1020500000B589B00121082001F0A6FF0121084642
:1020600001F092FF02220021264800F097F8022298
:102070000121244800F092F80320019002208DF8FD
:1020800009008DF8080001208DF80A008DF80B007A
:1020900001A91C4800F03AF806A803F0A7FC0020AC
:1020A000ADF818004FF6FF7007900020ADF8200043
:1020B000ADF81A0006A9144803F056FC00231A468E
:1020C0000321114803F023FA03A803F095FA002036
:1020D000ADF8140003A90C4803F057FA01210A488F
:1020E00003F0F4F901221146074803F08EFA0021AB
:1020F000054803F00BFC0121034803F0EDF909B09A
:1021000000BD000000000240000C0040F0B50A468F
:1021100000210023002400BF3DE0012505FA01F362
:10212000156805EA03049C4234D105684F00032674
:10213000BE40B543056015794E00B540066835438D
:1021400005601579012D02D01579022D16D185680B
:102150004F000326BE40B543856055794E00B5401B
:10216000866835438560456801268E40B5434560E5
:10217000456896798E40B6B235434560C5684F00D4
:102180000326BE40B543C560D5794E00B540C6684C
:102190003543C560491C1029BFD3F0BDF0B50023FD
:1021A00000244D07ED0E02FA05F3CE1000F12005D4
:1021B00055F826504E07F70E0F26BE40B543CF10F8
:1021C00000F1200646F82750CE1000F1200555F802
:1021D000265045EA0304CE1000F1200545F82640BC
:1021E000F0BD01837047000010B5044607230122AB
:1021F00021460848FEF76CFB0648FEF7C5FB00BF0A
:1022000002210448FEF730FB0028F9D00148FEF710
:1022100027FB10BD0020014010B504460723012212
:1022200021460848FEF754FB0648FEF7ADFB00BF09
:1022300002210448FEF718FB0028F9D00148FEF7F8
:102240000FFB10BD0021014010B50124D9480078D2
:1022500018B1D8480078012874D1D74800780928E7
:1022600071D2DFE800F07F05122231435262710023
:10227000D24890ED000AD24880ED000A9FEDD10AC5
:10228000D14880ED000A012478E0CC4890ED000AA6
:10229000CB4880ED000AC94890ED000AB1EE400A33
:1022A000C94880ED000A012468E09FEDC60AC448D1
:1022B00080ED000AC14890ED000AB1EE400AC24824
:1022C00080ED000A012459E0BC4890ED000AB1EE0F
:1022D000400ABB4880ED000AB84890ED000AB1EE14
:1022E000400AB94880ED000A012447E0B34890ED68
:1022F000000AB1EE400AB24880ED000A9FEDB10A33
:10230000B14880ED000A012438E0AC4890ED000AA5
:10231000B1EE400AAA4880ED000AA84890ED000AF4
:10232000A94880ED000A012428E09FEDA60AA448F0
:1023300080ED000AA14890ED000AA34880ED000A54
:1023400001241BE049E00DE09C4890ED000A9C4808
:1023500080ED000A994890ED000A9B4880ED000A44
:1023600001240BE09FED970A954880ED000A9FED50
:10237000950A954880ED000A002400BF00BF002C9C
:1023800011D19248007801280ED18C4890ED000AB6
:10239000DFED8F0A80EE201A9FED8E0A21EE000AF3
:1023A0008D4880ED000AA6E08C48007801280ED107
:1023B000824890ED000ADFED860A80EE201A9FED3C
:1023C000880A21EE000A844880ED000A93E09FED20
:1023D0007D0A814880ED000A8DE077480078092861
:1023E0006AD2DFE800F06905111D283644525D000D
:1023F000724890ED000A724880ED000A9FED710A64
:10240000754880ED000A62E06C4890ED000A6C4867
:1024100080ED000A9FED720A6F4880ED000A56E0D9
:102420009FED680A664880ED000A9FED6D0A6A48D4
:1024300080ED000A4BE0614890ED000AB1EE400AE1
:102440005F4880ED000A9FED660A634880ED000A50
:102450003DE05A4890ED000AB1EE400A584880ED40
:10246000000A9FED580A5C4880ED000A2FE05348AF
:1024700090ED000AB1EE400A514880ED000A9FED50
:10248000550A554880ED000A21E09FED4E0A4C4860
:1024900080ED000A9FED4F0A4F4880ED000A16E0DC
:1024A000464890ED000A464880ED000A9FED490A33
:1024B000494880ED000A0AE09FED420A404880ED5D
:1024C000000A9FED400A444880ED000A00BF00BFAB
:1024D0003E480078012805D19FED3E0A3E4880ED38
:1024E000000A08E03D480078012804D19FED3C0A2D
:1024F000394880ED000A2F48007802280DD136486F
:1025000090ED000AF0EE000A20EE200AF2EE020A38
:1025100080EE201A80ED001A29E026480078032872
:1025200007D024480078052803D0224800780428E2
:102530001DD1234890ED000AB5EEC00AF1EE10FA65
:1025400006D2254890ED000AB1EE400A80ED000A5F
:10255000214890ED000A1948D0ED000A20EE200A2B
:10256000DFED1B0A80EE201A1B4880ED001A14488C
:1025700090ED000ADFED1B0A80EE201A80ED001AB4
:10258000114890ED000ADFED170A80EE201A80ED69
:10259000001A114890ED000A80ED000A90ED001A33
:1025A0000948D0ED000A064890ED000AFFF704F84C
:1025B00010BD000064010020A00100206C0100207B
:1025C0007001002000000000740100209E01002026
:1025D0000000FA43DB0FC93F780100209F01002073
:1025E000DB0FC9BF00007A4410B52DED048B02202B
:1025F00001F094FD75490860032001F08FFD7349D7
:102600004860042001F08AFD70498860052001F0CF
:1026100085FD6E49C8606E48007806281AD2DFE84A
:1026200000F0031A374C6178684890ED000AB8EE64
:10263000C08A90ED010AF8EEC08A8068404200EE40
:10264000100AB8EEC09A6148C068404200EE100A15
:10265000F8EEC09A72E05D480068404200EE100A51
:10266000B8EEC08A59484068404200EE100AF8EEC1
:10267000C08A56488068404200EE100AB8EEC09A00
:102680005248C068404200EE100AF8EEC09A55E089
:102690004E4890ED000AB8EEC08A4068404200EE15
:1026A000100AF8EEC08A494890ED020AB8EEC09AC6
:1026B00090ED030AF8EEC09A40E0444890ED000A1D
:1026C000B8EEC08A4068404200EE100AF8EEC08AB8
:1026D0003E4890ED020AB8EEC09A90ED030AF8EE7B
:1026E000C09A2BE0394890ED000AB8EEC08A90ED10
:1026F000010AF8EEC08A8068404200EE100AB8EE87
:10270000C09A3248C068404200EE100AF8EEC09A03
:1027100014E02E4890ED000AB8EEC08A40684042AE
:1027200000EE100AF8EEC08A284890ED020AB8EED2
:10273000C09A90ED030AF8EEC09A00BF00BF9FED6B
:10274000250A28EE000A2448D0ED000A20EE200ACF
:102750002248D0ED000A80EE201A214880ED001AB0
:102760009FED1C0A28EE800A1B48D0ED000A20EEDF
:10277000200A1A48D0ED000A80EE201A194880ED90
:10278000001A9FED140A29EE000A1348D0ED000A42
:1027900020EE200A1148D0ED000A80EE201A1248DF
:1027A00080ED001A9FED0B0A29EE800A0A48D0ED51
:1027B000000A20EE200A0948D0ED000A80EE201A17
:1027C0000A4880ED001ABDEC048B10BDC45A0020ED
:1027D000640100200000C84288010020840100201C
:1027E000745A0020885A00209C5A0020B05A0020B9
:1027F0002DE9F04107460C460025002608E0384642
:10280000FFF7F2FC0544052005F02EFE701CC6B251
:10281000A642F4DBB5FBF4F080B2BDE8F081000025
:1028200010B52DED0E8B0820FFF7F6FC044609F0DD
:10283000A7FC41EC1E0B9FED180B53EC102B09F07D
:10284000EFFC41EC1D0B9FED160B53EC102B09F028
:10285000E7FC41EC1C0B9FED140B53EC102B09F023
:10286000DFFC41EC1B0B9FED120B53EC102B09F01E
:10287000E9FA41EC1A0B9FED100B53EC102B09F009
:10288000E1FA41EC190B09F0EFF908EE100AB0EE8D
:10289000480ABDEC0E8B10BD6666666666660A4029
:1028A00000000000000026400000008014AEEF3F52
:1028B000000000000000F03F000000000000B040F9
:1028C00000BFFEE710B500200E4908600E48006802
:1028D00020F440000C4908600846006840F480007D
:1028E000086000200949C1F8AC02012005F0DCFDB8
:1028F00001200449086005F0D7FD00200349C1F814
:10290000A80210BDA882404200040240008040425C
:102910001CB50121022001F037FB4FF4406000900C
:1029200001208DF8040000208DF8060003208DF8AA
:10293000050001208DF8070069460548FFF7E6FB12
:102940000120044908600449C1F8AC021CBD000024
:1029500000040240A88240420080404210B500209E
:102960000E4908600E48006820F440000C490860D9
:102970000846006840F48000086001200949C1F859
:10298000AC0205F091FD01200449086005F08CFDC2
:1029900000200449C1F8A80210BD0000A8824042EE
:1029A000000402400080404270B5054600241748EC
:1029B000006820F440001549086008460068086077
:1029C000002619E0002012490860012005F06CFD86
:1029D00001201049C1F8A8026006040E0C487C389A
:1029E000006810B144F0010401E024F0010401206A
:1029F00005F05AFD701CC6B2082EE3DB15B9FFF7CF
:102A000061FF01E0FFF7AAFF204670BD000402400D
:102A1000A88240420080404270B504460D46002620
:102A200000F01AF8204600F0CBF800F06BF82846CA
:102A300000F0C6F800F066F800F00EF844F001006F
:102A400000F0BEF800F05EF80120FFF7ADFF06468B
:102A500000F034F8304670BD10B51548006820F419
:102A60004000134908600846006840F48000086090
:102A70000120104908601048D0F82C0200B910BDA0
:102A800001200C49091F086005F00EFD00200A49CD
:102A9000C1F8AC0207488038006800B1EFE70120B8
:102AA00005F002FD00200349091F086000BFE6E7AA
:102AB00000040240AC8240420080404210B50E4803
:102AC000006820F440000C4908600846006840F4A3
:102AD000800008600020094908600949C1F8AC027B
:102AE000012005F0E1FC0120044908600449C1F817
:102AF000AC0205F0D9FC10BD00040240A88240429F
:102B00000080404210B500241448006820F44000C2
:102B100012490860084600680860012010490860F2
:102B200005F0C2FC01200F49C1F8A80205F0BCFC69
:102B30000AE0601CC4B2322C03DDFFF7BFFF0020A7
:102B400010BD012005F0B0FC054880380068002861
:102B5000EFD10349091F08600120F1E7000402409A
:102B6000AC824042008040422DE9F04780468946D1
:102B700014461D46089E49464046FFF74DFF07464E
:102B8000601CFF2101FA00F0C4F108012944491E2C
:102B9000FF220A41104300F0FF0AC5F1080006FABF
:102BA00000F0C6B2C4F10700064107EA0A0737433E
:102BB0003A464946404600F035F80120BDE8F08726
:102BC00070B504461448006820F4400012490860BB
:102BD0000846006840F48000086000200F49086043
:102BE000002516E0E0090D49091D08606006040E85
:102BF000012005F059FC01200949C1F8A80205F09F
:102C000053FC002005490860012005F04DFC681CBC
:102C1000C5B2082DE6DB70BD00040240A882404228
:102C20000080404270B504460D461646FFF714FF7B
:102C30002046FFF7C5FFFFF765FF2846FFF7C0FFF7
:102C4000FFF760FF3046FFF7BBFFFFF75BFFFFF7C3
:102C500035FF012070BD000030EEC01A234880ED22
:102C6000001A90ED001A2248D0ED001A31EE611AD8
:102C70002048D0ED001A21EE211A1F48D0ED001A8D
:102C80001A4890ED002A01EE821A1C48D0ED001A75
:102C900031EE211A80ED001A90ED001ADFED181ABE
:102CA000B4EEE11AF1EE10FA03DD9FED151A80ED96
:102CB000001A124890ED001ADFED121AB4EEE11A74
:102CC000F1EE10FA03D29FED0F1A80ED001A0748BB
:102CD00090ED001A064880ED001A084890ED001AA1
:102CE000BDEEC11A11EE100A70470000E00100208D
:102CF000E80100207C01002080010020E401002088
:102D000000788246007882C630EEC01A234880EDF3
:102D1000001A90ED001A2248D0ED001A31EE611A27
:102D20002048D0ED001A21EE211A1F48D0ED001ADC
:102D30001A4890ED002A01EE821A1C48D0ED001AC4
:102D400031EE211A80ED001A90ED001ADFED181A0D
:102D5000B4EEE11AF1EE10FA03DD9FED151A80EDE5
:102D6000001A124890ED001ADFED121AB4EEE11AC3
:102D7000F1EE10FA03D29FED0F1A80ED001A07480A
:102D800090ED001A064880ED001A084890ED001AF0
:102D9000BDEEC11A11EE100A70470000EC010020D0
:102DA000F40100207C01002080010020F0010020BF
:102DB00000788246007882C630EEC01A234880ED43
:102DC000001A90ED001A2248D0ED001A31EE611A77
:102DD0002048D0ED001A21EE211A1F48D0ED001A2C
:102DE0001A4890ED002A01EE821A1C48D0ED001A14
:102DF00031EE211A80ED001A90ED001ADFED181A5D
:102E0000B4EEE11AF1EE10FA03DD9FED151A80ED34
:102E1000001A124890ED001ADFED121AB4EEE11A12
:102E2000F1EE10FA03D29FED0F1A80ED001A074859
:102E300090ED001A064880ED001A084890ED001A3F
:102E4000BDEEC11A11EE100A70470000F801002013
:102E5000000200207C01002080010020FC010020F5
:102E600000788246007882C630EEC01A234880ED92
:102E7000001A90ED001A2248D0ED001A31EE611AC6
:102E80002048D0ED001A21EE211A1F48D0ED001A7B
:102E90001A4890ED002A01EE821A1C48D0ED001A63
:102EA00031EE211A80ED001A90ED001ADFED181AAC
:102EB000B4EEE11AF1EE10FA03DD9FED151A80ED84
:102EC000001A124890ED001ADFED121AB4EEE11A62
:102ED000F1EE10FA03D29FED0F1A80ED001A0748A9
:102EE00090ED001A064880ED001A084890ED001A8F
:102EF000BDEEC11A11EE100A704700000402002056
:102F00000C0200207C01002080010020080200202B
:102F100000788246007882C61CB50121102001F09D
:102F200033F80120009000208DF8040003208DF874
:102F3000050001208DF8070069460248FFF7E6F812
:102F40001CBD00000010024010B5322004F046FF06
:102F50000446022C0BD1064806490A68026089889B
:102F60008180054805490A6802608988818010BD12
:102F700050020020560200205C0200206202002065
:102F80001CB50121084600F0FFFF4FF4805000906F
:102F900001208DF8040000208DF8060003208DF834
:102FA000050001208DF8070069460448FFF7AEF8D8
:102FB0004FF480510148FFF714F91CBD0000024096
:102FC00000B52649D1ED010AB0EE600A00EE900A84
:102FD000B8EEE01A414200EE901AF8EEE00A07F06F
:102FE0002EF91E4981ED010A1D49D1ED010AB0EE0D
:102FF000600A00EE900AB8EEE01A414200EE901A24
:10300000F8EEE00A07F01BF9154981ED010A1549B0
:10301000D1ED010AB0EE600A00EE900AB8EEE01AB7
:10302000414200EE901AF8EEE00A07F008F90D4967
:1030300081ED010A0C49D1ED010AB0EE600A00EE03
:10304000900AB8EEE01A414200EE901AF8EEE00A5B
:1030500007F0F5F8044981ED010A00BD745A00201B
:10306000885A00209C5A0020B05A002070B50446AF
:103070000025BC2C01DB012510E0622C01DB0225C0
:103080000CE02A2C01DB032508E0142C01DB0425CD
:1030900004E00A2C01DB052500E006252A461A215A
:1030A000D020FFF7BFFD70BD70B50446B4F57A7F40
:1030B00001DD4FF47A74042C00DA04244FF47A70A2
:1030C00090FBF4F0401EC5B22A461921D020FFF72C
:1030D000A9FD0546264604EBD671C1F34F00FFF764
:1030E000C5FF70BD10B580226B21D020FFF79AFD7F
:1030F000C82005F0B9F900226B21D020FFF792FD1E
:10310000012000F03DF8002000F030F83220FFF7F9
:10311000CBFF00223821D020FFF784FD00226A2156
:10312000D020FFF77FFD00222321D020FFF77AFD7A
:1031300080223721D020FFF775FD7521D020FFF7C1
:103140006BFC0446682C0DD101226B21D020FFF7C7
:1031500069FD00226C21D020FFF764FD3220FFF7CB
:10316000A3FF01E0012010BD0020FCE738B50446B4
:10317000022304221C21D0200094FFF7F5FC38BD67
:1031800038B50446022304221B21D0200094FFF707
:10319000EBFC38BD08B505F0D3F9009058E00A21E2
:1031A000684607F003FC2B480068B0F57A7F4BDADD
:1031B00028480068401C274908602748008827499C
:1031C0000988084400B224490880084640882349F9
:1031D0004988084400B220494880084680881F4931
:1031E0008988084400B21C4988801D4800881D4910
:1031F0000988084400B21A490880084640881949DD
:103200004988084400B21649488008468088154914
:103210008988084400B21249888000200CE00E49D9
:1032200031F910100B4A128812B291FBF2F109B277
:103230000D4A22F81010401C0328F0DB0B48094906
:103240000A6802608988818000F070F800F010F848
:10325000A5E70000400200204402002030020020C8
:103260004A02002036020020500200205C020020AA
:1032700010B53C21D020FFF7CFFB04463B21D020E6
:10328000FFF7CAFB04EB002000B2244908803E216E
:10329000D020FFF7C1FB04463D21D020FFF7BCFB47
:1032A00004EB002000B21D4948804021D020FFF7E8
:1032B000B3FB04463F21D020FFF7AEFB04EB002018
:1032C00000B21649888016480068B0F57A7F23DB83
:1032D00008460088134908801048408848800F48F5
:1032E00080888880084600880F490988401A00B203
:1032F0000A4908800B4840880B494988401A00B2A7
:10330000064948800748808807498988401A00F59F
:10331000804000B20149888010BD000036020020C4
:1033200040020020620200205C02002010B544210F
:10333000D020FFF771FB04464321D020FFF76CFB40
:1033400004EB002000B22C4908804621D020FFF772
:1033500063FB04464521D020FFF75EFB04EB002011
:1033600000B2254948804821D020FFF755FB04468C
:103370004721D020FFF750FB04EB002000B21E498C
:1033800088801E480068B0F57A7F05DA01201C4964
:1033900008601C4908702DE018480068B0F57A7F75
:1033A00002D10020174908704FF496701449086044
:1033B00011480088144908800F48408848800E480A
:1033C000808888800846008810490988401A00B221
:1033D000094908800C4840880C494988401A00B2C5
:1033E000054948800848808808498988401A00B201
:1033F0000149888010BD00003002002040020020FA
:10340000380000205C0100205602002050020020FD
:1034100000BFFEE77047000070B5002100230F22B7
:10342000C4781CB3174C246804F4E064C4F5E06469
:10343000C4F30721C1F10404E3B20A4144789C407B
:10344000E1B28478144021430C07210E0E4C05781C
:103450006155047804F01F050124AC4005786D1116
:10346000AD0005F1E025C5F8004109E0047804F05D
:103470001F050124AC40054D0678761145F826401D
:1034800070BD00000CED00E000E400E080E100E031
:1034900002490143024A1160704700000000FA052A
:1034A0000CED00E030B500240CE0002506E0002023
:1034B000074901EBC5010855681CC5B2802DF6DB34
:1034C000601CC4B2082CF0DB00F0D2F830BD000064
:1034D00080020020F0B5144600267F2801DC3F2939
:1034E00000DDF0BD0B46CF1701EB5777FF10C7F19A
:1034F0000707FAB2CF1701EB5777FF10A1EBC70709
:10350000FDB2C5F107070123BB40DEB24CB10A4B47
:1035100003EBC0039B5C3343074F07EBC007BB546F
:1035200008E0054B03EBC0039B5CB343024F07EB82
:10353000C007BB5400BFD4E7800200201CB50121A6
:10354000082000F021FD4FF4F040009001208DF89C
:10355000040000208DF806008DF805008DF80700A6
:1035600069464048FEF7D2FD0121080700F01CFD26
:10357000012000F003FD002000F0BAFD002000F063
:10358000FDFC002038490860642004F06DFF012034
:103590003649C1F8B0020021AE2000F04FF90021F9
:1035A000D52000F04BF90021502000F047F9002110
:1035B000A82000F043F900213F2000F03FF900214E
:1035C000D32000F03BF90021084600F037F9002134
:1035D000402000F033F900218D2000F02FF9002168
:1035E000142000F02BF90021202000F027F9002101
:1035F000022000F023F90021A12000F01FF9002192
:10360000C02000F01BF90021DA2000F017F900219A
:10361000122000F013F90021812000F00FF90021A1
:10362000EF2000F00BF90021D92000F007F900216C
:10363000F12000F003F90021DB2000F0FFF8002169
:10364000302000F0FBF80021A42000F0F7F8002162
:10365000A62000F0F3F80021AF2000F0EFF8FFF70C
:1036600021FF1CBD000C0240B0824142008041425B
:1036700030B500241CE004F1B001C8B2002100F014
:10368000DDF80021084600F0D9F80021102000F0F4
:10369000D5F8002508E0084901EBC501085D0121C6
:1036A00000F0CCF8681CC5B2802DF4DB601CC4B2FD
:1036B000082CE0DB30BD0000800200202DE9F04F37
:1036C00080460C4615461E46A346A5F12000C5B20D
:1036D00000273EE00C2E07D105EB45001F4901EB0A
:1036E000800010F8079004E01D4800EB051010F86A
:1036F00007904FF0000A26E009F0800028B121462B
:103700004046099AFFF7E6FE09E0099808B901204A
:1037100000E00020024621464046FFF7DBFE4FEA6C
:1037200049604FEA1069601CC4B2A4EB0B00B042C0
:1037300005D15C4608F1010000F0FF0806E00AF13F
:10374000010000F0FF0ABAF1080FD5DB00BF781CBA
:10375000C7B2B742BEDBBDE8F08F0000F2C9000877
:1037600066CE00082DE9FF4F81B0074691461E4600
:103770000E9D4FF0000A002439E0301B401EC1B2FC
:103780000A2004F019FFB9FBF0F00A21B0FBF1F2B6
:1037900001FB1208BAF1000F16D1701EA04213DD12
:1037A000B8F1000F0ED10120AB4605EBDB714910DB
:1037B00001FB04710090C8B22B4620220299FFF74A
:1037C0007DFF12E04FF0010A0120AB4605EBDB71F3
:1037D000491001FB04710090C8B208F13001CAB26F
:1037E0002B460299FFF76AFF00BF601CC4B2B442C7
:1037F000C3DB05B0BDE8F08F78B505460E4614462C
:1038000018E07A2D03DD002506F11000C6B23A2E2D
:1038100004DD002005460646FFF744FE0120009027
:1038200022780C2331462846FFF748FF05F10800AF
:10383000C5B2641C20780028E3D178BD10B50A46D3
:103840001AB10123124C236002E00023104C2360C4
:10385000002116E000230E4C0C34236000F080039E
:103860001BB10123241F236003E00023084C08340C
:1038700023600123064C0C3423604306180E4B1CB6
:10388000D9B20829E6DB0123014C236010BD0000FA
:10389000AC82414201460148405C704780060020EE
:1038A000002004E00021034A1154411CC8B2092839
:1038B000F8DB70478006002038B5044601200090F0
:1038C00000201E494870012000902EE0BDF8000045
:1038D000204018B101201A49086002E00020184970
:1038E00008600120164910390860052004F0DCFD4D
:1038F00000201449C1F8A002052004F0D5FD0120E4
:103900001049C1F8A0020846D0F83C0230B10B487B
:103910004078BDF80010084308494870BDF8000021
:103920004FF6FF7101EA40000090BDF80000FF284B
:10393000CCDD102004F0B8FD38BD0000800600206A
:10394000B00242420000424210B5FFF7A9FF00F06A
:103950002FF90F48C0780E49097940EA01200D4936
:10396000088000240FE00C4810F81400401E0121CC
:1039700001FA00F007490988084010B9601CC0B27C
:1039800010BD601CC4B2102CEDDB0020F8E7000075
:1039900080060020400000204400002010B50020D8
:1039A00013490860102004F07FFD0120FFF784FF19
:1039B0004320FFF781FF0020FFF77EFF0120FFF784
:1039C0007BFF0020FFF778FF0020FFF775FF002046
:1039D000FFF772FF0020FFF76FFF0020FFF76CFF7B
:1039E00001200449C1F8A802102004F05DFD10BDBB
:1039F000A80242420000424210B50020134908606C
:103A0000102004F051FD0120FFF756FF4320FFF77F
:103A100053FF0020FFF750FF0020FFF74DFF5A2013
:103A2000FFF74AFF5A20FFF747FF5A20FFF744FFEE
:103A30005A20FFF741FF5A20FFF73EFF01200449BB
:103A4000C1F8A802102004F02FFD10BDA8024242C8
:103A5000000042421CB50121102000F095FA4FF4FD
:103A60000040009000208DF8040003208DF8050030
:103A700002208DF8070069460B48FEF747FB4FF41C
:103A8000A850009001208DF8040000208DF8060059
:103A900002208DF8050001208DF8070069460248D4
:103AA000FEF734FB1CBD00000010024010B5FFF70C
:103AB0004BFF00EE100AB8EE400A2F4880ED000AD6
:103AC0000720FFF7E7FE00EE100AB8EE400A2B4889
:103AD00080ED000A0820FFF7DDFE00EE100AB8EEC8
:103AE000400A274880ED000A0520FFF7D3FE00EECC
:103AF000100AB8EE400A234880ED000A0620FFF7BE
:103B0000C9FE00EE100AB8EE400A1F4880ED000A18
:103B1000194890ED000AF1EE000AB4EE600AF1EEE9
:103B200010FA05D11948007810B901201849086029
:103B300017480068F8B1124890ED000ADFED150A49
:103B4000B4EEE00AF1EE10FA15D21048007890B900
:103B500011480068B0F57A7F0DDB01200B49087031
:103B600000200E4908700E4908700E4908700E4971
:103B700008700E49087010BDB4010020A401002097
:103B8000A8010020AC010020B00100209801002015
:103B9000640000200000EC42400200209A01002056
:103BA000990100209B0100209C0100209D01002024
:103BB0001CB50020019001200090002025490860DC
:103BC00025490878FFF778FE23494878FFF774FE07
:103BD0000220019036E00120009027E001201D49DD
:103BE00008390860052004F05FFC00201B49C1F87B
:103BF000A002052004F058FC01201849C1F8A002D9
:103C00000846D0F83C0250B115489DF80410405CBD
:103C1000BDF80010084312499DF804208854BDF8EF
:103C200000004FF6FF7101EA40000090BDF800006F
:103C3000FF28D3DD102004F037FC9DF80400401C61
:103C4000C0B201909DF804000928C4DB012001499D
:103C500008601CBDA802424242000020000042420F
:103C60008006002010B500F00BF800F009F800F015
:103C700007F8FFF793FE00F025F8FFF7BDFE10BD33
:103C800010B500200D490860102004F00DFC012043
:103C9000FFF712FE4220FFF70FFE0020FFF70CFE99
:103CA0000020FFF709FE0020FFF706FE012004496F
:103CB000C1F8A802102004F0F7FB10BDA802424290
:103CC0000000424210B50020124908600120FFF7B1
:103CD000F3FD4420FFF7F0FD0020FFF7EDFD01208C
:103CE000FFF7EAFD0320FFF7E7FD0020FFF7E4FD03
:103CF0000020FFF7E1FD0020FFF7DEFD0020FFF7C9
:103D0000DBFD01200449C1F8A802102004F0CCFB1F
:103D100010BD0000A8024242000042422DE9F041DD
:103D20001424884890ED000ADFED870A30EE600A1F
:103D3000B1EE400ABDEEC00A10EE106A834890ED65
:103D4000000ADFED810A30EE600AB1EE400ABDEEF6
:103D5000C00A10EE105A7E4890ED000ADFED7A0A94
:103D600030EE600AB1EE400ABDEEC00A10EE107AE5
:103D70006042854202DDA54200DA002560428642AB
:103D800002DDA64200DA00266042874202DDA74239
:103D900000DA00276F4890ED000AF2EE060AB4EE52
:103DA000600AF1EE10FA09D16B4890ED000AF1EECD
:103DB000040A30EE200A80ED000A12E0654890ED1A
:103DC000000AF2EE020AB4EE600AF1EE10FA08D12F
:103DD000614890ED000AF1EE040A30EE600A80EDD1
:103DE000000A5D4890ED000AB5EEC00AF1EE10FA47
:103DF00003D29FED5A0A80ED000A00EE105AB8EE89
:103E0000C00A5548D0ED000A20EE200ADFED4E0A28
:103E100080EE201A524880ED001A00EE106AB8EECB
:103E2000C00A4D48D0ED000A20EE200ADFED460A18
:103E300080EE201A4B4880ED001A00EE107AB8EEA2
:103E4000C00ADFED490A20EE200ADFED3F0A80EECE
:103E5000201A464880ED001A4548007818B14448B9
:103E6000007801280FD1414890ED000A3A48D0ED82
:103E7000000A20EE200ADFED3F0A80EE201A3B48C0
:103E800080ED001A3BE03A48007802280DD137480F
:103E900090ED000AF0EE000A20EE200AF2EE020A8F
:103EA00080EE201A80ED001A29E0314800780328BE
:103EB00007D02F480078052803D02D480078042823
:103EC0001DD1274890ED000AB5EEC00AF1EE10FAB8
:103ED00006D2264890ED000AB1EE400A80ED000AB5
:103EE000224890ED000A1C48D0ED000A20EE200A7E
:103EF000DFED200A80EE201A1C4880ED001A1848D9
:103F000090ED000ADFED1C0A80EE201A80ED001A09
:103F1000144890ED000ADFED180A80EE201A80EDBB
:103F2000001A124890ED000A80ED000A90ED001A88
:103F30000C48D0ED000A0A4890ED000AFDF73CFB62
:103F4000BDE8F081A401002000000043A80100208A
:103F5000AC010020B40100206C0100200000000032
:103F60007001002074010020DB0FC93F78010020A0
:103F7000640100200000FA4300007A44014908620D
:103F80007047000000000E4229B1064A1268024341
:103F9000044B1A6004E0034A12688243014B1A6022
:103FA000704700003038024029B1064A12680243C7
:103FB000044B1A6004E0034A12688243014B1A6002
:103FC000704700004038024029B1064A1268024397
:103FD000044B1A6004E0034A12688243014B1A60E2
:103FE000704700004438024029B1064A1268024373
:103FF000044B1A6004E0034A12688243014B1A60C2
:104000007047000024380240F0B50021002200244F
:10401000022500260223324F3F6807F00C0121B130
:10402000042905D0082937D105E02E4F076036E076
:104030002D4F076033E02A4F3F1F3F68C7F380567C
:10404000274F3F1F3F6807F03F036EB1264FB7FB76
:10405000F3F7DFF88CC0ACF1040CDCF800C0CCF353
:10406000881C07FB0CF40CE01E4FB7FBF3F7DFF8DE
:1040700070C0ACF1040CDCF800C0CCF3881C07FB6A
:104080000CF4174F3F1F3F68C7F301477F1C7D00AB
:10409000B4FBF5F7076002E0124F076000BF00BFF6
:1040A0000F4F3F6807F0F0010909104F7A5C07686D
:1040B000D74047600A4F3F6807F4E051890A0B4F29
:1040C0007A5C4768D7408760054F3F6807F46041D6
:1040D000490B064F7A5C4768D740C760F0BD0000C7
:1040E000083802400024F40000127A00D6000020B4
:1040F0000021094A11701170012802D0042808D14A
:1041000003E00121044A117004E00521024A117004
:1041100000E000BF00BF704770380240014602292E
:1041200006D003290DD0042912D005291ED116E08E
:104130004FF08042526A10B200224FF080435A6220
:1041400016E00C4A126810B200220A4B1A600FE007
:10415000094A126810B20022074B1A6008E0074AA9
:10416000126810B20022054B1A6001E0002000BF67
:1041700000BF70472404004024080040240C004085
:104180002DE9F04764254FF4FA6251108748006822
:1041900006F06AF8854908604FF4FA6251108448C5
:1041A000006806F061F8824908604FF4FA62511025
:1041B0008048006806F058F87E4908604FF4FA62BB
:1041C00051107D48006806F04FF87B490860784838
:1041D0000068A0F2DC5708460068A0F2DC58754879
:1041E0000068A0F2DC5671480068A0F2DC59684211
:1041F000874202DDAF4200DA00276842804503DDD6
:10420000A84501DA4FF000086842864202DDAE425E
:1042100000DA00266842814503DDA94501DA4FF046
:1042200000096648D0ED000A00EE106AB8EEC00A38
:1042300030EE800ABDEEC00A10EE104A002C00DA03
:10424000002407FB04F04FF4FA7190FBF1F000EE4C
:10425000100AB8EEC00A5A4880ED000AC8F1000002
:10426000604390FBF1F000EE100AB8EEC00A55482A
:1042700080ED000AC9F1000000EE100AB8EEC00A95
:10428000DFED510A20EE200ADFED500A80EE201A01
:104290004F4880ED001A4F48007818B14D4800781B
:1042A00001280FD14A48D0ED000A00EE104AB8EEBE
:1042B000C00A20EE800ADFED450A80EE201A80ED6C
:1042C000001A3BE04348007802280DD1404890EDA9
:1042D000000AF0EE000A20EE200AF2EE020A80EE5A
:1042E000201A80ED001A29E03A480078032807D008
:1042F00038480078052803D03648007804281DD1B6
:104300002F4890ED000AB5EEC00AF1EE10FA06D281
:104310002F4890ED000AB1EE400A80ED000A2C48CB
:10432000D0ED000A00EE104AB8EEC00A20EE800A76
:10433000DFED260A80EE201A80ED001A204890ED6D
:10434000000ADFED250A80EE201A80ED001A1D48D4
:1043500090ED000ADFED200A80EE201A80ED001AB1
:104360001B4890ED000A80ED000A1C4800780028E8
:104370000EDD9FED1B0A124880ED000A9FED180A22
:10438000134880ED000A15480078401E1349087054
:104390000F4890ED001A0B48D0ED000A084890ED48
:1043A000000AFDF709F9BDE8F08700009000002041
:1043B00094000020980000209C0000206C01002048
:1043C0007001002074010020DB0FC93F0000FA4398
:1043D000780100206401002000007A4410020020CF
:1043E0000000000010B52DED088BB0EE40BAF0EEE5
:1043F00060BAB0EE418AF0EE618AB0EE429AF0EE19
:10440000629AB0EE43AA51EC1B0B07F02DFC1D493C
:104410000860084680ED018AC0ED058ABDEEC90A34
:1044200080ED020ABDEEE90A80ED030A80ED04AAE0
:10443000C06880008968484300EE100AB8EEC00AE0
:10444000114880ED000A0F4890ED040ADFED0F0AD5
:1044500020EE200A0E4880ED000A0A4890ED000A7E
:104460000C4880ED000A074890ED010A0A4880EDEB
:10447000000A044890ED050A084880ED000ABDECEA
:10448000088B10BDD45A002084010020DB0F494066
:10449000880100208C010020900100209401002060
:1044A00010B54FF4AD70554908600A210920FEF798
:1044B0009FF95249096890FBF1F05149087008468C
:1044C0000078052801DD052008704D480078062891
:1044D0005ED2DFE800F0031221303F4E9FED493AF3
:1044E000F2EE0A2AB3EE0E2ADFED471A9FED471AC5
:1044F0009FED470BFFF776FF4AE09FED473AF2EE5C
:104500000A2AB3EE0E2ADFED451A9FED3F1A9FED02
:10451000440BFFF767FF3BE09FED433AF2EE0A2AB8
:10452000B3EE0E2ADFED381A9FED401A9FED400BD7
:10453000FFF758FF2CE09FED3C3AF2EE0A2AB3EE6B
:104540000E2ADFED311A9FED301A9FED3B0BFFF77E
:1045500049FF1DE09FED343AF2EE0A2AB3EE0E2A2F
:10456000DFED291A9FED361A9FED360BFFF73AFF64
:104570000EE09FED363AF2EE0A2AB3EE0E2ADFED98
:10458000221A9FED211A9FED320BFFF72BFF00BF80
:1045900000BF1B48007806282ED2DFE800F0030A8F
:1045A00011181F2608202C4908600E202B4908608E
:1045B00022E00620284908600A20284908601BE0FC
:1045C00004202549086007202449086014E00420DD
:1045D000214908600720214908600DE008201E4994
:1045E00008600B201D49086006E004201A49086095
:1045F00007201A49086000BF00BF10BD60010020FD
:10460000640100209A99993D000000007B14AE3DA2
:10461000022B8716D9CEB73F8FC2753D643BDF3D75
:104620000000000000000000B81E853DBC74133E71
:10463000000000806ABCC43F000000A0EFA7C63F96
:10464000295C8F3E00000000D7A3D03FC520303D3D
:10465000000000E07A14CE3FC8010020CC01002009
:104660000CB50020019000903448006840F4803080
:104670003249086000BF3148006800F40030009003
:104680000198401C0190009818B90198B0F5A04F0E
:10469000F1D12A48006800F4003010B101200090E8
:1046A00001E0002000900098012846D123484030C6
:1046B000006840F08050214940310860204800687F
:1046C00040F440401E4908601C48083000681B49FF
:1046D000083108600846006840F400400860084659
:1046E000006840F4A05008601648091F0860081FC1
:1046F000006840F08070091F086000BF0F48006824
:1047000000F000700028F9D040F205700E490860F2
:104710000A480830006820F00300084908310860A2
:104720000846006840F00200086000BF03480830F7
:10473000006800F00C000828F8D10CBD00380240D9
:104740000070004008544007003C024070B5049CD3
:10475000002807DA44F29F151E4E356005441E4EB0
:10476000356006E044F29F151B4E35602D1A194E38
:104770003560002906DA44F29F15184E75630D4422
:10478000B56305E044F29F15144EB5636D1A756369
:10479000002A06DA44F29F15114EB563154475637D
:1047A00005E044F29F150E4E7563AD1AB563002BFC
:1047B00006DA44F29F150A4E35641D44F56305E0A0
:1047C00044F29F15064EF563ED1A3564054D2C60D5
:1047D00070BD0000344401403448014000400140B5
:1047E000000001403818004000B5F0EE403AF0EE0D
:1047F000602AB0EE413A9FED680AB0EE402AF5EE2D
:10480000C03AF1EE10FA07DD644890ED000A30EE90
:10481000020A80ED000A1AE0F5EEC03AF1EE10FA55
:1048200007D25E4890ED000A30EE420A80ED000AA1
:104830000DE0F5EEC03AF1EE10FA08D1574890EDD0
:10484000000ADFED570A20EE200A80ED000AF5EE9F
:10485000C02AF1EE10FA07DD504890ED010A30EE63
:10486000020A80ED010A1AE0F5EEC02AF1EE10FA14
:1048700007D24A4890ED010A30EE420A80ED010A63
:104880000DE0F5EEC02AF1EE10FA08D1434890EDA4
:10489000010ADFED430A20EE200A80ED010AB5EEA1
:1048A000C03AF1EE10FA07DD3C4890ED020A30EE16
:1048B000020A80ED020A1AE0B5EEC03AF1EE10FAF3
:1048C00007D2364890ED020A30EE420A80ED020A25
:1048D0000DE0B5EEC03AF1EE10FA08D12F4890ED98
:1048E000020ADFED2F0A20EE200A80ED020AB0EE68
:1048F000630A03F009FEB0EE404AB0EE630A03F02B
:1049000003FEB1EE400AF0EE404A2448D0ED000A22
:10491000B0EE600AB0EE441AF0EE640A05F08FFCC7
:104920001E4880ED000AB0EE620A03F0EDFDB0EE25
:10493000404AB0EE620A03F0E7FDB1EE400AF0EE45
:10494000404A1648D0ED010AB0EE600AB0EE441AB3
:10495000F0EE640A05F073FC104880ED010AB0EE39
:10496000430A03F0D1FDB0EE404AB0EE430A03F033
:10497000CBFDB1EE400AF0EE404A0848D0ED020A05
:10498000B0EE600AB0EE441AF0EE640A05F057FC8F
:10499000024880ED020A00BD0AD7233C685A002075
:1049A0006666663F042808D14FF0E021096941F0AE
:1049B00004014FF0E022116107E04FF0E0210969A6
:1049C00021F004014FF0E0221161704710B506F0AC
:1049D00097FE012801D006F019FB10BD10B515484F
:1049E000006840F47000134908601348006840F004
:1049F00001001149086000200F49083108600E4885
:104A000000680E4908400C4908600D48091D0860FF
:104A1000081F006820F48020091F08600020064954
:104A20000C310860FFF71CFE4FF00060014980392F
:104A3000086010BD88ED00E000380240FFFFF6FE80
:104A400010300024F0B50C46154600210022068CDB
:104A50004FF6FE773E400684018B028C4FF60C76B3
:104A600031407E1C06EA03162E4331434FF6F5769D
:104A7000324044F00106324301830284F0BDF0B5B8
:104A80000C461546002100220026078C4FF6EF7CCD
:104A900007EA0C070784018B028C4FF6FF7707EAC1
:104AA000041640F6FF4739404FF6FF7707EA033711
:104AB00039434FF6FF7707EA052739434FF65F770B
:104AC0003A4046F010073A4301830284F0BDF0B546
:104AD0000C461546002100220026078C4FF6FF6C7D
:104AE00007EA0C070784818B028C4FF6FF7707EAF1
:104AF00004264FF60C7739404FF6FF7707EA031785
:104B00002F4339434FF2FF573A4046F480773A43F8
:104B100081830284F0BDF0B50C46154600210022C9
:104B20000026078C4EF6FF7C07EA0C070784818B72
:104B3000028C4FF6FF7707EA043640F6FF4739400C
:104B40004FF6FF7707EA052739434FF6FF7707EA65
:104B50000337394345F6FF773A4046F480573A43E6
:104B600081830284F0BD000030B58BB005460C4651
:104B700001210220FFF708FA01214804FFF724FA77
:104B8000032208211E48FDF709FB02208DF81C00B6
:104B900000208DF81E004FF48070069001208DF8E3
:104BA0001F0003208DF81D0006A91548FDF7AEFA79
:104BB0000995ADF820400020ADF82800ADF822009E
:104BC00008A9104800F0D0FE6020ADF804000120D4
:104BD000ADF806000020ADF8100001A9094800F06A
:104BE0001DFD0821074800F060FD0121054800F087
:104BF00061FC0121034800F06FFC0BB030BD0000E8
:104C0000000402400044014030B58BB005460C461C
:104C100001210220FFF7B8F901218804FFF7D4F938
:104C2000032209212048FDF7B9FA02208DF81C0063
:104C300000208DF81E004FF40070069001208DF8C2
:104C40001F0003208DF81D0006A91748FDF75EFA26
:104C50000995ADF820400020ADF82800ADF82200FD
:104C600008A9124800F080FE6020ADF80400012081
:104C7000ADF806000020ADF8100001A90B4800F0C7
:104C8000CDFC0821094800F010FD0121074800F083
:104C90002FFC0121054800F00DFC0121034800F024
:104CA0001BFC0BB030BD0000000402400048014076
:104CB00030B58BB005460C4601214020FFF774F952
:104CC00001210220FFF760F902208DF828004FF43F
:104CD0004040099003208DF8290000208DF82A001B
:104CE00001208DF82B0009A92248FDF70FFA0922AF
:104CF0000E212048FDF752FA09220F211D48FDF729
:104D00004DFA0795ADF818400020ADF82000ADF839
:104D10001A0006A9184800F027FE6020ADF804002C
:104D20000120ADF8060000200390ADF81000ADF8AA
:104D3000140001A9104800F071FC01A90E4800F010
:104D4000BDFC08210C4800F0B0FC08210A4800F026
:104D500014FD0121084800F0CBFB0121064800F0BA
:104D6000BBFB40F2DC50044938310860091F086081
:104D70000BB030BD000402400018004030B58BB0CD
:104D800005460C4601210846FFF71EF901211020B7
:104D9000FFF7FAF8012209213448FDF7FFF9012253
:104DA0000B213248FDF7FAF901220D212F48FDF7BA
:104DB000F5F901220E212D48FDF7F0F94FF4D4400A
:104DC000099002208DF8280003208DF8290000208A
:104DD0008DF82A0001208DF82B0009A92348FDF742
:104DE00095F90795ADF818400120ADF82000002096
:104DF000ADF81A0006A91E4800F0B6FD6020ADF817
:104E000004000120ADF806000020ADF8100001A953
:104E1000174800F003FC01A9154800F04FFC01A958
:104E2000134800F0B7FC01A9114800F019FD012159
:104E30000F4800F05DFB08210D4800F036FC08210A
:104E40000B4800F09AFC0821094800F000FD0821F9
:104E5000074800F04EFD0121054800F02BFB012121
:104E6000034800F039FB0BB030BD000000100240D9
:104E7000000001404FF08040008A4FF08040008ADF
:104E800020F001004FF080410882704704480088FC
:104E90000348008820F001000149088070470000A5
:104EA00010040040044800880348008820F00100F6
:104EB000014908807047000010080040044800883D
:104EC0000348008820F00100014908807047000075
:104ED000100C0040044800880348008820F00100BE
:104EE00001490880704700001018004010B5CA48FA
:104EF0000068B0F5C86F15DDC848007890B9C8489B
:104F00000068B0F57A7F0DDB0120C44908700020ED
:104F1000C4490870C4490870C4490870C44908707D
:104F2000C4490870C448007800F08000002857D1B8
:104F30000221C24800F018FB002851D00221BF48CE
:104F400000F0C7FABC48007800F04000C0B3BB488E
:104F500000F0FEFABA49088008460088B949098875
:104F6000884204DA42F20F70B749086002E000207C
:104F7000B5490860B2480088B2490988401AB24968
:104F800009680844B14908600968B14A1268881A7A
:104F9000002801DB014600E04142B1F5FA7F03DD64
:104FA000AB480068A9490860A8480068A84908609B
:104FB0000020A14908700021A04800F06DFB0FE01F
:104FC000FFE79E4800F0C4FA9E4908809A4800789E
:104FD00040F04000984908700221984800F05CFBBE
:104FE0009C48007800F08000002857D104219348A5
:104FF00000F0BAFA002851D00421904800F069FA74
:105000009448007800F04000C0B38C4800F0A3FA48
:10501000914908800846008890490988884204DA46
:1050200042F20F708E49086002E000208C4908604F
:105030008948008889490988401A894909680844CB
:10504000754908600968874A1268881A002801DBD8
:10505000014600E04142B1F5FA7F03DD8148006876
:105060006D4908606C4800687E49086000207949F5
:1050700008700021714800F073FB0FE0FFE76F48F4
:1050800000F069FA754908807248007840F04000E5
:10509000704908700221694800F062FB724800788C
:1050A00000F08000002857D10821644800F05CFA25
:1050B000002851D00821614800F00BFA6A480078B6
:1050C00000F04000C0B35D4800F048FA674908802E
:1050D0000846008866490988884204DA42F20F705F
:1050E0006449086002E00020624908605F48008867
:1050F0005F490988401A5F49096808445E490860A9
:1051000009685E4A1268881A002801DB014600E03F
:105110004142B1F5FA7F03DD5848006856490860FE
:10512000554800685549086000204F490870002123
:10513000424800F07FFB0FE0FFE7404800F00EFA26
:105140004B4908804848007840F0400046490870C4
:1051500002213A4800F06EFB4948007800F08000D8
:10516000002857D11021354800F0FEF9002851D011
:105170001021324800F0ADF94148007800F04000BD
:10518000C0B32E4800F0EDF93E490880084600887B
:105190003D490988884204DA42F20F703B490860B1
:1051A00002E00020394908603648008836490988FD
:1051B000401A364909680844354908600968354A83
:1051C0001268881A002801DB014600E04142B1F56F
:1051D000FA7F03DD2F4800682D4908602C480068DD
:1051E0002C4908600020264908700021134800F06F
:1051F00073FB0FE0FFE7114800F0B3F92249088084
:105200001F48007840F040001D49087002210B48FB
:1052100000F062FB10BD0000940000209A01002005
:105220004002002099010020980100209B010020ED
:105230009C0100209D010020680000200004014026
:105240006C0000206A0000208000002090000020F8
:10525000A00000206E0000207200002070000020DE
:1052600084000020A40000207400002078000020AA
:10527000760000208800002098000020A800002070
:105280007A0000207E0000207C0000208C0000209E
:105290009C000020AC00002030B589B005460C46CB
:1052A00001210220FEF790FE01210420FEF76CFE92
:1052B0004FF47070079002208DF8200003208DF8C5
:1052C000210000208DF8220002208DF8230007A97C
:1052D0004348FCF71BFF032206214148FCF75EFF11
:1052E000032207213E48FCF759FF032208213C48CE
:1052F000FCF754FF032209213948FCF74FFF0595BD
:10530000ADF810400020ADF81800ADF8120004A967
:10531000344800F029FB0020ADF80000ADF8020091
:105320000120ADF804000020ADF806000F20ADF814
:10533000080069462B4800F028F90420ADF8000069
:105340000020ADF802000120ADF804000020ADF807
:105350000600ADF808006946224800F016F908205A
:10536000ADF800000020ADF802000120ADF8040007
:105370000020ADF80600ADF808006946194800F0B5
:1053800004F90C20ADF800000020ADF80200012067
:10539000ADF804000020ADF80600ADF8080069463D
:1053A000104800F0F2F82E208DF80C0002208DF845
:1053B0000D008DF80E0001208DF80F0003A8FEF7F8
:1053C0002BF801221E21074800F01FF90121054892
:1053D00000F08EF80121034800F07EF809B030BDDE
:1053E00000080240000401400348008820F001004A
:1053F00001490880704700001004014030B58BB0AF
:1054000005460C4601210804FEF7DEFD01211020AF
:10541000FEF7BAFD032205212448FCF7BFFE032254
:1054200006212248FCF7BAFE6020069002208DF883
:105430001C0003208DF81D0000208DF81E000120A7
:105440008DF81F0006A91948FCF760FE0995ADF814
:1054500020400020ADF82800ADF8220008A914482B
:1054600000F082FA6020ADF804000120ADF80600DB
:105470000020ADF8100001A90D4800F0CFF801A9F7
:105480000B4800F01BF90821094800F00EF908212B
:10549000074800F072F90121054800F00BF80121DE
:1054A000034800F019F80BB030BD000000100240B6
:1054B0000040014021B1028842F08002028004E0F5
:1054C00002884FF67F731A4002807047CA430282F7
:1054D0007047CA430282704721B1028842F001023C
:1054E000028004E002884FF6FE731A400280704783
:1054F00031B1B0F8442042F40042A0F8442005E065
:10550000B0F84420C2F30E02A0F844207047F0B572
:105510000C4615461E460021002200230189028BFD
:10552000038C4FF6F877394021434FF6FC473A4059
:1055300040F201173A434FF6DD773B404FF6FF77D5
:1055400007EA06172F433B43018102830384F0BD22
:105550000146486B70470146886B70470146C86B2F
:1055600070470146086C704730B5024600200023A2
:105570000024158A05EA0103958905EA010413B19F
:105580000CB1012000E0002030BD70B505460C468E
:10559000208850B92389A28861882846FFF752FAEB
:1055A000E188284600F0B4F925E0208804280AD1D3
:1055B0002389A28861882846FFF761FAE188284696
:1055C00000F0AFF917E0208808280AD12389A288C3
:1055D00061882846FFF77BFAE188284600F0AEF99B
:1055E00009E02389A28861882846FFF794FAE188B8
:1055F000284600F0ACF970BD0021018041800121F6
:1056000081800021C180018170471AB183890B43D9
:10561000838102E083898B438381704770B50024C6
:1056200000220023058C4FF6FE7635400584028C5F
:105630008388048B4FF68F752C40B51E2C400D8847
:105640002C43751E2A408D892A434D882A43104DCC
:10565000A84202D00F4DA84213D14FF6F7752A4049
:10566000CD892A434FF6FB752A408D882A434FF691
:10567000FF652B404FF6FF552B400D8A2B434D8A7B
:105680002B43838004838D684563028470BD0000D2
:1056900000000140000401400A460021018C4FF641
:1056A000FD7319401143018470470A460021018BA4
:1056B0004FF6F773194011430183704770B500240A
:1056C00000220023058C4FF6EF7635400584028CCE
:1056D0008388048B48F6FF752C404FF6FF452C401D
:1056E0000D884FF6FF7606EA05252C434FF6DF7549
:1056F0002A408D8906EA05152A434D8806EA0515D4
:105700002A43154DA84202D0144DA8421DD14FF690
:105710007F752A40CD894FF6FF7606EA05152A43A4
:105720004FF6BF752A408D8806EA05152A434FF6C5
:10573000FF352B404FF2FF752B400D8A06EA850599
:105740002B434D8A06EA85052B43838004838D68AD
:105750008563028470BD0000000001400004014028
:105760000A460021018C4FF6DF7319404FF6FF7394
:1057700003EA02131943018470470A460021018B92
:105780004FF2FF7319404FF6FF7303EA02231943E8
:105790000183704770B5002400220023058C4FF66A
:1057A000FF6635400584028C8388848B4FF68F75A5
:1057B0002C404FF6FC752C400D882C434FF6FF55BE
:1057C0002A408D894FF6FF7606EA05252A434D8843
:1057D00006EA05252A43154DA84202D0144DA842D9
:1057E0001DD14FF2FF752A40CD894FF6FF7606EAAC
:1057F00005252A434FF6FF352A408D8806EA052500
:105800002A434EF6FF752B404DF6FF752B400D8A4F
:1058100006EA05152B434D8A06EA05152B438380BE
:1058200084838D68C563028470BD00000000014060
:10583000000401400A460021018C4FF6FF53194035
:105840004FF6FF7303EA02231943018470470A46A7
:105850000021818B4FF6F773194011438183704704
:1058600070B5002200230024058C4EF6FF763540EB
:105870000584038C8488828B48F6FF752A404FF696
:10588000FF452A400D884FF6FF7606EA05252A4394
:105890004DF6FF752B408D8906EA05352B434D8863
:1058A00006EA05352B430A4DA84202D0094DA8420D
:1058B00008D14BF6FF752C400D8A4FF6FF7606EAAD
:1058C00085152C43848082838D680564038470BDB4
:1058D00000000140000401400A460021018C4DF601
:1058E000FF7319404FF6FF7303EA02331943018433
:1058F00070470A460021818B4FF2FF7319404FF623
:10590000FF7303EA022319438183704741627047A2
:10591000028B4FF6F3731A400283028B0A43028311
:105920007047028B4FF2FF331A400283028B4FF60F
:10593000FF7303EA01231A4302837047828B4FF6F9
:10594000F3731A408283828B0A4382837047828B6F
:105950004FF2FF331A408283828B4FF6FF7303EAC4
:1059600001231A438283704700220288184B984211
:105970000ED0184B98420BD0B0F1804F08D0164B88
:10598000984205D0154B984202D0154B984204D14D
:105990004FF68F731A404B881A43124B984207D028
:1059A000114B984204D04FF6FF431A400B891A431B
:1059B00002804B68C3620B880385054B984202D076
:1059C000044B984201D18B7A03860123838270476E
:1059D00000000140000401400004004000080040B5
:1059E000000C004000100040001400404FF0FF3158
:1059F0004160002101800181418081727047000077
:105A000001460A2906DB0C4A12681AB10B4A1278C1
:105A1000012A0ED101200022094B1A60094B1A609D
:105A2000094B5A639A63094B9A639A631A64DA635F
:105A300000E00020704700000C8241425C01002021
:105A4000344401403448014000400140000001401E
:105A500010B52DED028B40F225513B4800F08EFB36
:105A600000286ED0384800F043FCC4B237480068C4
:105A7000B0F57A7F03DA0020BDEC028B10BD34480C
:105A80003449097844547B2C03D0324800780028EC
:105A900005DD30480078401C2E49087002E00020E7
:105AA0002C4908702B4800780B284AD1002029493E
:105AB00008702748807A7D2843D100210920FBF710
:105AC0005BFD2349497A88423BD100202249087076
:105AD000224908702249087022490870224908703A
:105AE000224908701A4A1179D07800F075FC2048D4
:105AF00080ED000A164A9179507900F06DFC1D483E
:105B000080ED000A124A117AD07900F065FCB0EEFF
:105B1000408A1948007802280AD1F0EE480A144851
:105B200090ED000A00F0ECFB144880ED000A07E05D
:105B3000074A117AD07900F04FFC104880ED000A36
:105B400000BF002098E7000000500040D401002072
:105B5000BC060020C5000020980100209A0100200A
:105B6000990100209B0100209D010020DE01002002
:105B700070010020740100206401002078010020E1
:105B80002DE9F0412DED028B40F22551434800F004
:105B9000F5FA00287FD000260127404800F0A8FB36
:105BA000C5B23F480068B0F57A7F04DA0020BDEC4A
:105BB000028BBDE8F0813B483B49097845547B2D79
:105BC00003D039480078002805DD37480078401CAC
:105BD0003549087002E000203349087032480078E7
:105BE0000B2857D10020304908702E48807A7D2834
:105BF00050D1002403E02B48005D4640641C092C72
:105C0000F9DB2848407AB04200D10027002F41D16B
:105C10002648007858B901202449087000202449FA
:105C2000087024490870244908702449087000202D
:105C3000234908701B4A1179D07800F0CDFB214828
:105C400080ED000A174A9179507900F0C5FB1E4893
:105C500080ED000A134A117AD07900F0BDFBB0EE56
:105C6000408A1A48007802280BD1F0EE480A1548FD
:105C700090ED000A00F044FB154880ED000A08E0B2
:105C800009E0084A117AD07900F0A6FB104880EDAF
:105C9000000A00BF00BF002089E70000001001409B
:105CA000D4010020DC060020B80000209C01002068
:105CB00099010020980100209A0100209B010020FA
:105CC000DE0100207001002074010020640100202A
:105CD0007801002000B5002200BF05E00449885C7F
:105CE00004F046FC501CC2B2182AF7DB00BD0000CD
:105CF0008C06002010B52DED0C8B40F225519F48ED
:105D000000F03CFA00287DD09C48001D04889C4887
:105D10000068B0F57A7F03DA0020BDEC0C8B10BD73
:105D2000412C15D197480078412811D19648007828
:105D300070B9002095490870954908700120924972
:105D400008700020934908709349087093490870BF
:105D50008C490C704B2C03D101209149087006E04E
:105D6000492C01D04A2C02D100208D4908708C4862
:105D7000007888B9412C06DB482C04DCA4F14000F3
:105D8000884908702FE0082C02DC86490C702AE054
:105D900000208449087026E081480078012822D13B
:105DA000432C06D100208049087001207F490870EB
:105DB0000DE0472C06D101207B49087000207B496B
:105DC000087004E000207849087078490870412C78
:105DD00001D0452C04D1A4F140007249087002E0C2
:105DE000002070490870582C08D1714890ED000AC5
:105DF000DFED700A30EE200A80ED000A592C0AD13E
:105E00006B4800E0B7E090ED000ADFED6A0A30EE83
:105E1000600A80ED000A7B2C02D1012066490870DF
:105E20007D2C02D102206449087063480078012863
:105E300008D16249624A12788C5461480078401C4B
:105E40005F4908705C480078022870D15B48C078D0
:105E5000502803D101205B49087070E05748407812
:105E600023286CD056480078574908703AE05449C6
:105E70000978554A1278881A06F06BF941EC1D0B27
:105E8000B0EE4D1AF0EE6D1A9FED500B00F060FC75
:105E9000B0EE40BAF0EE60BA4B490978491E474A65
:105EA000515CA1F1300006F054F941EC1C0B53ECAD
:105EB0001B2B06F0B5F941EC190B4648006806F0BB
:105EC000A5FC41EC1A0B53EC192B05F0FFFE41EC3D
:105ED000180B05F0C9FE3F4908603B480078401E9A
:105EE00039490870384800780428C0DA33484078C7
:105EF0003038092822D2DFE800F0050C131B1C1DE6
:105F00001E1F2000334890ED000A294880ED000A4A
:105F100014E0304890ED000A2F4880ED000A0DE0B3
:105F20002C4890ED000A2D4880ED000A06E016E0AE
:105F300004E003E002E001E000E000BF00BF002059
:105F40001D4908701E4908701F4908709FED240AFA
:105F5000204880ED000A32211848FAF7FEFA14486A
:105F600090ED000AB5EEC00AF1EE10FA03D29FEDF3
:105F70001C0A80ED000A0020CFE60000004400402B
:105F800040020020BC000020990100209801002060
:105F90009A0100209B0100209C0100209D0100200F
:105FA000A1010020A00100209E0100209F010020EF
:105FB0006C0100200000C842B9000020E706002064
:105FC000BA000020A2010020BB0000200000000059
:105FD00000002440C00000207C010020800100203F
:105FE0000000000010B52DED028B40F225513D4818
:105FF00000F0C4F8002873D03A4800F079F9C4B230
:1060000039480068B0F57A7F03DA0020BDEC028BD6
:1060100010BD36483649097844547B2C03D03448A7
:106020000078002805DD32480078401C30490870AF
:1060300002E000202E4908702D4800780B284FD12F
:1060400000202B4908702948807A7D2848D10021FA
:106050000920FBF791FA2549497A884240D100206E
:10606000244908702449087024490870244908709C
:106070002449087024490870244908701B4A117982
:10608000D07800F0A9F9224880ED000A174A9179EA
:10609000507900F0A1F91F4880ED000A134A117AE7
:1060A000D07900F099F9B0EE408A1B4880ED008A63
:1060B0001A48007802280AD1F0EE480A144890EDF8
:1060C000000A00F01DF9164880ED000A07E0074AB3
:1060D000117AD07900F080F9114880ED000A00BFF4
:1060E000002093E700480040D4010020BC060020B7
:1060F000C4000020980100209A010020990100208E
:106100009B0100209C0100209D010020DE01002059
:106110007001002074010020B00000206401002004
:106120007801002000B5002200BF05E00449885C2A
:1061300004F02AFA501CC2B2182AF7DB00BD000096
:106140008C06002000B5002200BF05E00449885CF1
:1061500004F028FA501CC2B2182AF7DB00BD000078
:106160008C06002021B1828942F40052828104E031
:1061700082894DF6FF731A408281704770B50246DE
:10618000002400230025002040F66A16B14200D109
:1061900000BFC1F3421501F01F03012606FA03F305
:1061A000012D02D19689334006E0022D02D1168AD4
:1061B000334001E0968A33400C12012606FA04F4BB
:1061C0001688344013B10CB1012000E0002070BDEE
:1061D000F0B50346002400260025002040F66A178B
:1061E000B94200D100BF1846C1F3421401F01F06A6
:1061F000012707FA06F5012C01D10C3004E0022C2E
:1062000001D1103000E014301AB107682F43076045
:1062100002E00768AF430760F0BD00002DE9FF47CB
:1062200005460E460024A14600BFA046B08900B135
:1062300000BF2C8A24F44054F08804432C82AC899B
:1062400041F20C608443B088318908437189084366
:106250000443AC81AC8A24F44074B0890443AC821A
:106260006846FDF7D1FE2048854202D01F4885428E
:1062700002D1DDF80C9001E0DDF80890A88900F467
:10628000004040B109EBC90000EB0910316849003A
:10629000B0FBF1F707E009EBC90000EB091031682A
:1062A0008900B0FBF1F76420B7FBF0F0040120098E
:1062B000642101FB1078A88900F4004040B132202D
:1062C00000EBC800B0FBF1F000F00700044308E069
:1062D000322000EB08106421B0FBF1F000F00F0059
:1062E00004432C81BDE8FF870010014000140140E9
:1062F00001468888C0F30800704700BFFEE7000031
:1063000000B52DED108B83B0F0EE408AB0EE60FA50
:106310009FED2A0A8DED020AB5EEC0FAF1EE10FAF1
:1063200041D0F5EEC08AF1EE10FA3CD0C8EE8FFAFB
:106330002348006806F06AFA41EC1E0B9FED210B22
:1063400053EC102B05F06CFF41EC1C0B1FEE900A78
:1063500006F05CFA41EC1D0B53EC1C2B05F0B6FC6F
:1063600041EC1B0B1948006806F050FA53EC1B2B4C
:10637000CDE900019DED000B51EC100B05F062FD25
:1063800041EC1A0BB0EE4A0AF0EE6A0A00F074F81B
:10639000B0EE409AF0EE609A51EC190B05F064FCF7
:1063A00008EE100A01E09FED0A8A0A4880ED008A93
:1063B000B0EE480A03B0BDEC108B00BD3333B33EE2
:1063C0008C0100209A9999999999A93F90010020F0
:1063D00000000000B40000202DE9F0412DED088BF5
:1063E00004460D4605EB042006B24FF47A7096FB86
:1063F000F0F100FB1167384605F0ABFE41EC1B0BDA
:106400009FED0F0B53EC102B05F00AFF41EC190B1D
:106410004FF47A7096FBF0F7384605F09AFE41EC9F
:106420001A0B53EC192B05F051FC41EC180B05F03D
:106430001BFC00EE100ABDEC088BBDE8F0810000EB
:10644000FCA9F1D24D62503F03B40198410000987D
:1064500050EAC12018BF04204A0D18BF40F00100C7
:1064600040F2FF72B2EB515F08BF40F0020001281A
:1064700008BF052002B0704770B59B482DED020B98
:106480002DED068B079D25F00044A04218DC9748AF
:10649000844202DC0AD1069840B19DED060BBDECAA
:1064A000068B02B0BDE8704001F052BC002DCCBF9D
:1064B0009FED8F0B9FED900BBDEC068B02B070BD76
:1064C0008F48A04215DD8F48A042D8BF4FF0FF345F
:1064D00058DD9DED060B51EC100BFFF7B5FF0428BE
:1064E00008BF01F069FC9DED060BBDEC068B02B008
:1064F00070BD9DED060B51EC100B01F0F9FFCDE9DD
:10650000060181489FED828BA0423CDD8248A0427B
:106510001FDD00249FED82AB9DED060B53EC1A2B83
:1065200051EC100B05F0D2FB9DED060B41EC190B65
:1065300053EC1A2B51EC100B05F072FE53EC182B98
:1065400006F07AF853EC192B05F07CFCCDE9060136
:1065500049E09DED060B012453EC182B51EC100B78
:1065600005F0B4FB9DED060B41EC190B53EC182B19
:1065700051EC100B06F060F853EC192B05F062FC9F
:10658000CDE906012FE06848A0421FDD02249FEDFF
:10659000689B9DED060B53EC192B51EC100B05F08D
:1065A0003FFE53EC182B05F091FB9DED060B41ECE3
:1065B000180B53EC192B51EC100B06F03DF853EC73
:1065C000182B05F03FFCCDE906010CE09DED060B14
:1065D000032453EC102B9FED580B51EC100B05F0DE
:1065E00031FCCDE906019DED060B53EC102B51EC6F
:1065F000100B05F015FE41EC180B53EC182B05F0B1
:106600000FFE41EC190B4E480621B0EE490AF0EEA0
:10661000690A784401F060F953EC182B51EC100B27
:1066200005F0FEFD41EC180B4648B0EE490AF0EECD
:10663000690A0521784401F04FF953EC192B51EC0C
:10664000100B05F0EDFD41EC100B51EC180B53EC69
:10665000102B002C0EDA05F039FB9DED061B53ECD8
:10666000112B05F0DDFD9DED061B53EC112B05F004
:106670000BFF35E005F02AFB9DED061B53EC112BBB
:1066800005F0CEFD41EC100B2F48784400EBC40020
:1066900090ED001B51EC100B53EC112B05F0CCFFCF
:1066A0009DED061B53EC112B05F0C6FF41EC100BC2
:1066B0002648784400EBC40090ED001B51EC100B11
:1066C00053EC112B05F0E0FE41EC100B002DA2BFA6
:1066D000BDEC068B02B070BD51EC100B05F0B8FAA2
:1066E00041EC100B01E70000000010440000F07FB7
:1066F000182D4454FB21F93F182D4454FB21F9BFB8
:106700000000DC3F0000203E0000F33F00000000DE
:10671000000000000000F03F0000E63F0000000025
:106720000000000000000040008003400000000066
:10673000000000000000F83F000000000000F0BF73
:10674000EA780000A07800002A780000E2770000D4
:106750002DE9F04D2DED040B2DED0E8B96B0DDE9FE
:106760002550279CDDF890A025F0004624F0004835
:10677000BAF1000F14BF0121002101EB4502FC49D1
:1067800053184A1093422AD3002814BF0123002330
:1067900003EB44030B44F7498B4220D358EA000132
:1067A0009FEDF59B76D0DFF8D8B35D4503D1BAF104
:1067B000000F05D188E0BAF1000F08BF002100D01A
:1067C000012101EB450111F5001F08D8002814BF75
:1067D0000121002101EB440111F5001F0BD99DEDB2
:1067E000261B9DED240B16B0BDEC0E8B04B0BDE84E
:1067F000F04D01F0B7BA0027002DBCBFE149884534
:1068000021DAE1498845A8BF02271CDAC3451ADC12
:10681000DE4901EB2851142908DDC1F1340220FAC8
:1068200002F101FA02F282420DD108E058B9C1F139
:10683000140228FA02F101FA02F2424503D101F0F2
:106840000101C1F1020756EA0A0124D1002C22DA23
:10685000002D18BF022F01D0012F0AD00220F9F716
:10686000A7FE16B0BDEC0E8B04B0BDE8F04D01F0F4
:1068700057BA0220F9F79CFE01F052FA51EC100BC6
:1068800005F0E6F941EC100B16B0BDEC0E8B04B030
:10689000BDE8F08D18E09FEDBEAB9FEDBF8B0028EB
:1068A00071D1B848804522D105F1804010F58010A3
:1068B00008BFBAF1000F07D0B3450ADC002CA8BF0F
:1068C0009DED260BE0DA0DE0B0EE490AF0EE690A24
:1068D000DAE7002C06DA9DED260B51EC100B05F0E3
:1068E000B7F96FE0AE48784490ED000BCCE7D8459F
:1068F0004DD1002C48DA2EB186423AD1BAF1000FC0
:1069000042D126E0BAF1000F13D00220F9F750FE71
:1069100001F042FA8DED020B9DED240B8DED000B85
:1069200010EE900A039961F31E0003909DED020B97
:10693000AAE78DED02AB9DED240B1AEE901A10EE36
:10694000900A8DED000B61F31E0003909DED020B8C
:106950009AE78DED028B9DED240B18EE901A10EE48
:10696000900A8DED000B61F31E0003909DED020B6C
:106970008AE709DA9DED240B51EC190B53EC102B2F
:1069800005F060FA1EE020E09DED240B7CE78642D6
:106990001BDAB4F1804F0DD0A4F10050B0F1FF50DC
:1069A00013D1002D11DB9DED240B51EC100B03F0E6
:1069B0002FFB07E09DED240B53EC102B51EC100B3B
:1069C00000F0C2BC41EC100B5EE79DED240B51ECD6
:1069D000100B01F08DFDBAF1000FCDE90E0142D18F
:1069E0009FED710B46B3A6F1E040B0F17F600CD093
:1069F0005E4538D1002D00DAA7B3022F0CBF01206D
:106A00004FF0FF3005F0A5FBDCE7002D01DD002C89
:106A10000DDA002D01DD002C1FDB002D16DA002C15
:106A200014DB012F08BF9FED620B3FF42DAFB0EEDA
:106A30004A0AF0EE6A0A27E7022F18BF002D0CD091
:106A4000012F0AD1002DFFF61FAF06E0002DB8BFC1
:106A5000002C08DA012F3FF417AFB0EE480AF0EE31
:106A6000680A11E71BE0012000EBE57050EA07011E
:106A700015D0791EB0EE498AF0EE698A084308BF46
:106A80009FED4D8B4E480025804570DD4D494E48A9
:106A9000884514DDB0420DDB002C19DB2FE001200E
:106AA000F9F786FD16B0BDEC0E8B04B0BDE8F04DD5
:106AB00001F062B9B34502DC002C09DC1FE086421C
:106AC00002DA002C1BDA03E05E452BDD002C16DD1C
:106AD0000220F9F76DFD01F05FF98DED020B53EC2B
:106AE0001A2B51EC180B05F09BFBCDE90001039923
:106AF000019861F31E0003909DED020BC4E6022095
:106B0000F9F756FD01F058F910EE901A18EE900AB8
:106B10008DED020B8DED008B61F31E0003909DED5A
:106B2000020BB1E69DED0E0B53EC192B51EC100B43
:106B300005F082FD9FED260BCDE9080153EC102BEB
:106B40009DED080B51EC100B05F06AFB9FED221B2D
:106B500053EC112B05F098FC9DED081B53EC112B09
:106B600005F05EFB9FED1E1B53EC112B3CE08CE00F
:106B7000FFFF1F00FFFF0F00000000000000F03FBC
:106B80000000F03F0000F07F0000404301FCFFFFE9
:106B9000000000000000F07F000000000000000086
:106BA000CE76000000000000000000000000008021
:106BB000000000000000F0FF000000000000F0BF37
:106BC0000000E0410000F043FFFFEF3F0000000045
:106BD000000000000000D03F555555555555D53F94
:106BE000000000000000E03F05F04EFC9DED080BAA
:106BF00041EC1A0B53EC102B51EC100B05F010FB71
:106C000053EC1A2B05F00CFB41EC1A0B9FEDFE0B1D
:106C100053EC102B9DED080B51EC100B05F000FB15
:106C200041EC1B0B9FEDFA0B51EC1A0B53EC102BA4
:106C300005F0F6FA41EC1A0B9FEDF70B53EC102B15
:106C40009DED080B51EC100B05F0EAFA53EC1A2BF2
:106C500005F0F2FC41EC1A0B51EC1B0B53EC1A2B18
:106C600005F034F80690CDE906519DED060B53EC86
:106C70001B2B51EC100B05F0DFFC53EC1A2B05F02D
:106C800003FC41EC100B00F0A1B90020B6F5801F09
:106C90000EDA9FEDE30B53EC102B9DED0E0B51EC38
:106CA000100B05F0BDFACDE90E016FF034000E4671
:106CB00000EB2650A0F2FF37C6F31300DA4940F08C
:106CC0007F6646F040568842D8BF002408DDD74989
:106CD0008142C8BF012403DC0024A6F580167F1C76
:106CE000D348784400EBC4000F9690ED00CB9DEDA7
:106CF0000E0B53EC1C2B51EC100B05F09DFC9DED85
:106D00000E0B41EC1B0B53EC1C2B51EC100B04F045
:106D1000DDFF41EC100B51EC190B53EC102B05F07F
:106D200091F841EC1D0B51EC1B0B53EC1D2B05F0A6
:106D300077FA41EC1A0BBF488DED10AB78441095F3
:106D400090ED000B4FF0005040EA660000EB8440ED
:106D50008DED080B00F5002009909DED080B53EC1C
:106D60001C2B51EC100B05F067FC9DED0E1B53EC3A
:106D7000112B05F089FB41EC100B53EC102B9DED12
:106D8000100B51EC100B05F04BFA9DED080B41EC8C
:106D90001C0B53EC102B9DED100B51EC100B05F060
:106DA0003FFA53EC1B2B05F06FFB53EC1C2B05F04B
:106DB00043FC53EC1D2B05F033FA41EC1C0B53EC58
:106DC0001A2B51EC1A0B05F02BFA41EC1B0B9A48CD
:106DD0000621B0EE4B0AF0EE6B0A784400F07CFD21
:106DE000B0EE401AF0EE601AB0EE41DAF0EE61DA81
:106DF00053EC1B2B51EC1B0B05F012FA53EC1D2B23
:106E000005F00EFA9DED100B41EC1B0B53EC1A2B09
:106E100051EC100B04F05AFF53EC1C2B05F000FA58
:106E200053EC1B2B04F052FF9DED100B41EC1B0BA0
:106E300053EC102B51EC100B05F0F2F941EC1D0B4B
:106E40009FED7FEB53EC1E2B04F040FF53EC1B2B0C
:106E500004F03CFF0890CDE908519DED080B53EC80
:106E60001E2B51EC100B05F0E7FB53EC1D2B05F02E
:106E7000E3FB53EC1B2B05F007FB9DED080B41ECEE
:106E80001D0B53EC102B9DED100B51EC100B05F06E
:106E9000C7F941EC1B0B53EC1A2B51EC1D0B05F001
:106EA000BFF99DED080B41EC1A0B53EC102B51EC84
:106EB0001C0B05F0B5F953EC1A2B04F007FF41EC5D
:106EC0001A0B51EC1B0B53EC1A2B04F0FFFE0C9029
:106ED000CDE90C519DED0C0B53EC1B2B51EC100B21
:106EE00005F0AAFB53EC1A2B05F0CEFA41EC1B0B74
:106EF0009FED550B53EC102B9DED0C0B51EC100B33
:106F000005F08EF941EC1A0B9FED510B51EC1B0B68
:106F100053EC102B05F084F941EC1B0B9FED4E0B4D
:106F200053EC102B9DED0C0B51EC100B05F078F988
:106F300053EC1B2B04F0CAFE41EC100B484878447C
:106F400000EBC40090ED001B51EC100B53EC112B27
:106F500004F0BCFE41EC1B0B384605F0FAF8CDE915
:106F6000080153EC1B2B51EC1A0B04F0AFFE41EC63
:106F7000100B3C48784400EBC40090ED00CB51EC82
:106F8000100B53EC1C2B04F0A1FE9DED081B53ECE1
:106F9000112B04F09BFE0690CDE906519DED080BE8
:106FA00053EC102B9DED060B51EC100B05F044FB40
:106FB00053EC1C2B05F040FB53EC1A2B05F03CFB6B
:106FC00053EC1B2B05F060FA41EC100B9DED261BDA
:106FD00053EC102B8DED001B00959DED260B51EC15
:106FE000100B05F01DF99DED000B41EC1A0B53EC55
:106FF000102B9DED260B51EC100B05F01DFB9DEDAC
:10700000061B53EC112B2FE0000000604715F73FE3
:10701000FE822B654715F73F44DF5DF80BAE543E0B
:1070200000000000000040438E9803007AB60B0079
:107030004A720000787200008271000000000000B7
:107040000000000000000840000000E009C7EE3F1B
:10705000FD033ADC09C7EE3FF5015B14E02F3EBEAD
:107060000E700000C86F000005F0DAF853EC1A2B20
:1070700004F02CFE9DED060B41EC1A0B53EC102B8B
:107080009DED000B51EC100B05F0CAF8CDE90C0199
:107090009DED0C0B51EC1A0B53EC102B04F016FE6B
:1070A000CDE902010C46AA498C422FDB611A084344
:1070B00018D19DED0C0B53EC102B9DED020B51ECF8
:1070C000100B05F0B9FA41EC1B0B9FEDA30B51EC33
:1070D0001A0B53EC102B04F0F9FD53EC1B2B05F0AD
:1070E0009DF92DD20220F9F763FA00F055FE10EE5B
:1070F000901A18EE900A8DED020B8DED008B61F366
:107100001E0003909DED020BFFF7BEBB944A24F0D6
:107110000041914214D39349214408437FF4EFACDA
:107120009DED0C0B53EC102B9DED020B51EC100B55
:1071300005F082FA53EC1A2B05F070F97FF6DFACFC
:1071400024F000408849894A002601EB2051824200
:107150002BDA481C4FF4801121FA00F02044844AB5
:10716000C0F30A517A44A1F2FF3192ED000B814A3B
:107170008DED080BCA4020EA0202C0F3130040F470
:107180008010C1F1140120FA01F60992002CB8BF59
:1071900076429DED080B53EC102B9DED0C0B51EC42
:1071A000100B05F049FACDE90C019DED0C0B51ECEB
:1071B0001A0B53EC102B04F089FD9FED6F0B089018
:1071C000CDE9085153EC102B9DED080B51EC100B41
:1071D00005F026F841EC1B0B9FED690B53EC102BCF
:1071E0009DED080B51EC100B05F01AF89DED0C0B02
:1071F00041EC1C0B53EC102B9DED080B51EC100BCC
:1072000005F01AFA53EC1A2B05F03EF99FED5E1BC0
:1072100053EC112B05F004F853EC1C2B04F056FD35
:1072200041EC1A0B51EC1B0B53EC1A2B04F04EFDE6
:10723000CDE902019DED020B53EC1B2B51EC100B21
:1072400005F0FAF953EC1A2B05F01EF99DED020B2F
:1072500041EC1A0B53EC102B51EC100B04F0E0FF37
:10726000CDE908014A489DED080B0521784400F05E
:1072700033FB9DED081B51EC100B53EC112B04F06C
:10728000CFFF9DED021B53EC112B05F0FDF8CDE96E
:1072900006019DED020B53EC1A2B51EC100B04F080
:1072A000BFFF53EC1A2B04F011FD9FED3B0B41EC9B
:1072B0001A0B53EC102B9DED060B51EC100B05F047
:1072C000BBF99DED060B41EC1B0B53EC102B9DED18
:1072D000020B51EC100B04F0A3FF53EC1B2B04F03A
:1072E000B1FD53EC1A2B05F0A7F99DED021B53ECF1
:1072F000112B05F0A1F953EC192B05F0C5F8CDE9D8
:10730000020101EB065001150029C8BF039015DCEE
:107310009DED020B324651EC100B05F024FBFFF7FC
:1073200093F8042808BF00F047FD32469DED020B9C
:1073300051EC100B05F017FBCDE902019DED020B9E
:1073400051EC180B53EC102B04F06AFFFFF73ABB1B
:107350000000904000000000FE822B654715973C1E
:1073600000CC904000346F3F01FCFFFF0000E03F85
:10737000506E0000FFFF0F0000000000432EE63FAC
:10738000396CA80C615C20BEEF39FAFE422EE63F54
:10739000206D000000000000000000000000004020
:1073A00000B52DED048BB0EE409AF0EE609A83B0FC
:1073B00051EC190B05F074F841EC180B18EE100A9B
:1073C00018EE901A8DED008B002818BF012008439D
:1073D00020F00040C0F17F6000F1E040C00F14D009
:1073E00019EE101A19EE900A8DED009B002918BFB6
:1073F0000121084320F00040C0F17F6000F1E0402F
:10740000C00F04BF0120F9F7D3F8B0EE480A03B06B
:10741000F0EE680ABDEC048B00BD00000000000027
:1074200010B51D499FED1A1B2DED020B84B0059878
:1074300020F000408842DCBF01209DED040B21DDDF
:107440001649884209D1049840B94FF00100F9F774
:10745000AFF800F091FC06B010BD05DB9DED040B0C
:1074600000F076FC06B010BD68469DED040B00F000
:1074700017F800F001000121A1EB40009DED021B77
:107480009DED000B00F0A4FA06B010BD0000000056
:107490000000000000000000FB21E93F0000F07F39
:1074A0002DE9F14F04462DED020B2DED088B8AB02E
:1074B0009FEDE70B80ED020B139EE74826F0004599
:1074C00085420ADC9DED120B002084ED000B0AB012
:1074D000BDEC088B03B0BDE8F08FE0489FEDE0AB5A
:1074E0009FEDE1BBA84247DDE14F9FEDE39B9FEDA0
:1074F000E48B9DED120B53EC1A2B51EC100B002E6C
:107500001CDD05F099F841EC100BBD4208D053EC9E
:107510001B2B51EC100B05F08FF8C4E900010BE0B8
:1075200053EC192B51EC100B05F086F853EC182B8B
:1075300005F082F8C4E900010120C8E704F0C6FBA9
:1075400041EC100BBD4208D053EC1B2B51EC100B3F
:1075500004F0BCFBC4E900010BE053EC192B51EC27
:10756000100B04F0B3FB53EC182B04F0AFFBC4E991
:1075700000014FF0FF30AAE7C348A84279DB9DED38
:10758000120B51EC100B00F0B3FF41EC180B9FED08
:10759000C00B53EC102B04F043FE9FEDBF1B53ECCC
:1075A000112B04F093FB04F0A5FD074604F0D1FD78
:1075B00041EC190B53EC1A2B04F032FE53EC182B50
:1075C00004F062FF41EC180B53EC1B2B51EC190B30
:1075D00004F026FEDFF8C8A241EC100B4FEA155864
:1075E0000125FA4453EC102B51EC180B05F024F84C
:1075F000032DC4E900013DD0C1F30A5005EB45114C
:10760000A8EB00001139814234DA0AEB051BB0EE19
:1076100048AA9BED000BF0EE68AA53EC102B51EC3E
:10762000190B04F0FDFD41EC1B0B51EC1A0B53EC54
:107630001B2B05F001F841EC180B51EC1A0B53EC25
:10764000182B04F0F9FF53EC1B2B04F0F5FF9BED16
:10765000020B41EC1A0B53EC102B51EC190B04F0FC
:10766000DFFD53EC1A2B04F0E7FF41EC100B6D1C0F
:10767000B8E70EE0002EA8BF3846BFF628AF94ED5D
:10768000000B51EC100B04F0E3FAC4E9000178425E
:107690001DE7C6F3130040F4801EC6F30A50A0F2A3
:1076A000F530471100F01F05C5F12000DDF848B0A6
:1076B00008900020069007900520EC467949002D9F
:1076C00007EB0002794408BF51F8221009D051F8A5
:1076D000223001EB8201AB404A68089922FA01F19D
:1076E0001943A1FB0E26A1FB0B131A449A4234BF87
:1076F0000123002303EB06080CEB8003D3E901A66A
:107700000E448E4234BF0121002192448A4411B1BB
:10771000924502D903E0924501D2012100E0002107
:10772000C3E901A641444CF82010011EA0F101005C
:10773000C4DC029800F10050850F0298DDE9036770
:107740008000DDF8148004F004FD41EC1A0B304693
:1077500004F016FD9FED541B53EC112B04F060FD5B
:1077600041EC1B0B384604F00BFD9FED511B53EC15
:10777000112B04F055FD41EC180B404604F000FDC0
:107780009FED4D1B53EC112B04F04AFD41EC190BFE
:1077900051EC180B53EC192B04F098FA53EC1B2BFB
:1077A00004F094FA53EC1A2B04F090FACDE9080196
:1077B000002008909DED080B53EC1A2B51EC100B98
:1077C00004F03AFF53EC1B2B04F036FF53EC182B5C
:1077D00004F032FF53EC192B04F056FE9FED381BDA
:1077E00053EC112B04F01CFD9FED370B41EC180BF3
:1077F00053EC102B9DED080B51EC100B04F010FD19
:1078000053EC182B04F062FA9FED310B41EC180B8E
:1078100053EC102B9DED080B51EC100B04F000FD08
:1078200053EC182B04F052FA41EC100B139810F0A3
:10783000004F06D06D4251EC100B04F009FA41ECF8
:10784000100B284684ED000B41E60000000000000C
:107850000000000000000000FB21E93F7CD902404D
:1078600000004054FB21F93F3163621A61B4D03DFE
:10787000FB21F93F000000000000601A61B4D03D18
:107880007370032E8A19A33BFB21394100000000CD
:1078900083C8C96D305FE43F000000000000E03F96
:1078A000DA69000028690000000000000000103EB6
:1078B000000000000000103C000000000000103A32
:1078C000182D4454FB21F93D3326A611460B113CDB
:1078D00000000054FB21F93D70B504462DED028BEC
:1078E0004D1E00EBC500B0EE408AF0EE608A90EDD0
:1078F000000B35F0060017D053EC182B51EC100B91
:1079000004F08EFC41EC100B6D1E04EBC50090EDF5
:10791000001B51EC100B53EC112B04F0D7F941EC88
:10792000100B35F00600E7D1022D36D0042D1CD007
:10793000062D1CBFBDEC028B70BD53EC182B51EC17
:10794000100B04F06DFC94ED0A1B53EC112B04F0AA
:10795000BDF953EC182B04F063FC94ED081B53ECB9
:10796000112B04F0B3F941EC100B53EC182B51EC34
:10797000100B04F055FC94ED061B53EC112B04F096
:10798000A5F953EC182B04F04BFC94ED040B53ECCD
:10799000102B04F09BF941EC100B53EC182B51EC1D
:1079A000100B04F03DFC94ED021B53EC112B04F082
:1079B0008DF953EC182B04F033FC94ED001B53ECC1
:1079C000112B04F083F9BDEC028B41EC100B70BD60
:1079D000F1B506462DED040BBD482DED0C8B8AB09C
:1079E000B0EE418AF0EE618A179D25F000449FEDCC
:1079F000BABB9FEDBBCB844208DA9DED160B51EC70
:107A0000100B04F077FB002800F0E980B64FA74286
:107A100031DC002D0DDA9DED160B51EC100B04F04E
:107A200017F9CDE9160151EC180B04F011F941ECEE
:107A3000180B9FEDAF0B53EC102B9DED160B51EC7B
:107A4000100B04F021FD53EC182B9FEDAB0BCDE98F
:107A5000040151EC100B04F0EFFD41EC100B53EC62
:107A6000102B9DED040B51EC100B04F02FF99FED42
:107A7000A48BCDE916019DED160B53EC102B51ECA8
:107A8000100B04F0CDFBCDE904019DED040B53EC8C
:107A9000102B51EC100B04F0C3FB41EC190B9A486E
:107AA0000621B0EE490AF0EE690A7844FFF714FFA8
:107AB0009648B0EE40DAF0EE60DAB0EE490AF0EE49
:107AC000690A06217844FFF707FF9DED041B51EC7E
:107AD000100B53EC112B04F0A3FB9DED040B41ECB8
:107AE0001A0B53EC102B9DED160B51EC100B04F000
:107AF00097FB41EC190B53EC1A2B51EC1D0B04F0C6
:107B0000E5F853EC192B04F08BFB53EC182B04F025
:107B1000DDF89DED041B53EC112B04F081FB53ECBD
:107B2000182B04F0D3F841EC180B9FED790B51ECB6
:107B3000190B53EC102B04F073FB53EC182B04F0CF
:107B4000C5F841EC190B9DED160B53EC192B51ECBC
:107B5000100B04F0BBF841EC180BA74269DC30466F
:107B600004F0F7FA41EC1A0B51EC180B53EC1A2BFA
:107B700004F0ACF841EC1B0B53EC182B51EC180B38
:107B800004F04EFB53EC1B2B04F05CF953EC192B67
:107B900004F052FD9DED161B53EC112B04F074FC08
:107BA0009FED5D1B53EC112B04F03AFB53EC1A2BA9
:107BB00004F06AFC41EC180B022000EAA570C0F149
:107BC000010004F0C6FA53EC182B04F029FB00BFA7
:107BD00041EC100B0AB0BDEC0C8B05B0F0BD711C74
:107BE0001698214308430CD09DED160B012E1CBFA7
:107BF00053EC102B51EC1C0B10D000BF04F022F9F9
:107C0000E6E79DED160B51EC100B00F071FC41EC1A
:107C1000100B51EC1B0B53EC102BEFE751EC100B3E
:107C2000FEF712FC042808BF00F0C6F89DED160B05
:107C3000D0E7012E04BFB0EE480AF0EE680AC9D0C2
:107C40008DED048B002404949DED040B53EC102B5C
:107C50009DED160B51EC100B04F016FC53EC192B98
:107C600004F012FC41EC190B53EC182B51EC1C0BDB
:107C700004F0E8F841EC180B8DED008B00949DEDBD
:107C8000040B53EC102B9DED000B51EC100B04F08A
:107C9000C7FA53EC1B2B04F019F89DED000B41ECD7
:107CA0001A0B53EC192B51EC100B04F0B9FA53ECEE
:107CB0001A2B04F00BF853EC182B04F0B1FA9DEDDD
:107CC000001B53EC112B04F001F881E700000000C9
:107CD0000000303E00000000000000000000F03F07
:107CE000000000000000F0BF2894E53F0000000005
:107CF000182D4454FB21E93F075C143326A6813C30
:107D00000000000000000000DA650000F0650000DF
:107D1000635555555555D53F000000000000004003
:107D20009FED070B10B553EC102B9FED070B51EC9B
:107D3000100B04F087F841EC100B10BD00000000A0
:107D40000000000000000000000000000000F03F04
:107D500010B553EC102B51EC100B03F0B7FF41ECB6
:107D6000100B10BD10B553EC112B51EC100B03F0A0
:107D7000ADFF41EC100B10BD9FED050B10B553ECA2
:107D8000102B51EC100B04F05DF841EC100B10BD02
:107D900000000000000000009FED050B10B553EC43
:107DA000102B51EC100B04F03BFA41EC100B10BD02
:107DB00000000000000000709FED050B10B553ECB3
:107DC000102B51EC100B04F02BFA41EC100B10BDF2
:107DD000000000000000001000BF704701462D4861
:107DE000006828B92C480088401C2B4A108002E00B
:107DF0000020294A10802748006828B927480078C1
:107E000010B90120254A107025480078B0B92348E0
:107E10000078012807D123480078401C214A1070BF
:107E200001201F4A10701F480078022806D1002048
:107E30001C4A10701C4A10800220704715480068C8
:107E4000012804D10020154A1070154A10701548F9
:107E5000007801281CD114480088401C124A108068
:107E60001046008888420ADD0B480088884206DAFE
:107E700000200C4A10700C4A10800120DDE70648F3
:107E80000088884204DD0020064A1070064A1080EF
:107E90000020D2E700024242320000202C000020E5
:107EA0002D0000202E0000203000002008B500F03A
:107EB00047FB00900DE03221684602F077FD00F0AC
:107EC00009F8FDF707FFFEF72DF9FEF73BF9F9F783
:107ED0001DFBF0E710B52DED0A8B7B20FE490876DF
:107EE0007D21FD4880F82E10FC480078062873D2CA
:107EF000DFE800F00373EFEDECEBF94890ED000ADA
:107F0000F848D0ED000A30EE200AF748D0ED000A1C
:107F100030EE200AF548D0ED000A30EE200AF1EEEE
:107F2000000A80EE201A9FEDF20A21EE000ABDEE53
:107F3000C00A10EE100A01B2E7484183E84890ED0C
:107F4000000AE848D0ED000A30EE600AE648D0EDBD
:107F5000000A30EE200AE548D0ED000A30EE600A53
:107F6000F1EE000A80EE201A9FEDE10A21EE000AF0
:107F7000BDEEC00A10EE100A01B2D7488183D8487E
:107F800090ED000AB1EE400AD648D0ED000A30EE7E
:107F9000600AD548D0ED000A30EE200AD348D0ED73
:107FA000000A70EE200AB1EE001A80EE810AD14874
:107FB000D0ED000AD04890ED001A30EE811AC0EEE4
:107FC000010A9FEDCB0A20EE800ABDEEC00A10EE3A
:107FD000100A01B2C048C18362E19FEDC80BFFF7F0
:107FE000DFF9B0EE40CAF0EE60CA9FEDC60B53EC6D
:107FF000102B51EC1C0B03F025FF41EC1A0BBA4877
:1080000090ED000AB748D0ED000A30EE600AF0EEBD
:10801000000A80EE201A11EE104A204604F0F6FB0A
:1080200041EC1B0B53EC1A2B03F00CFF41EC190B2A
:108030009FEDB60B53EC102B04F0F2F841EC180B4B
:1080400004F058F801B2A4484183A64890ED000A14
:10805000A348D0ED000AB0EE001A10EE810AA24843
:10806000D0ED000A30EE600AB0EE081AC0EE010A48
:108070009FED9F0A20EE800ABDEEC00A10EE100AA6
:1080800001B295488183964890ED000A9548D0ED5D
:10809000000A30EE200A9448D0ED000A70EE200A63
:1080A000B0EE081A80EE810A9A48D0ED000A80EE00
:1080B000201A9FED8F0A21EE000ABDEEC00A10EED5
:1080C000100A01B28448C183EAE0B7E065E032E01B
:1080D000FFE7834890ED000A8248D0ED000A30EEB9
:1080E000200AF0EE000A80EE201A9FED810A21EEB0
:1080F000000ABDEEC00A10EE100A01B276484183B4
:1081000000218183774890ED000A7548D0ED000A80
:1081100030EE600A7848D0ED000A80EE201A9FED1C
:10812000740A21EE000ABDEEC00A10EE100A01B278
:108130006948C183B4E06A4890ED000A6948D0ED0F
:10814000000A30EE200AB0EE001AC0EE010A9FEDE0
:10815000680A20EE800ABDEEC00A10EE100A01B2D5
:108160005D484183002181835E4890ED000A5C48B0
:10817000D0ED000A70EE600A5F4890ED001A80EEC4
:10818000810ADFED5B0A20EE200ABDEEC00A10EE88
:10819000100A01B25048C18382E0514890ED000AB4
:1081A0005048D0ED000A30EE200A4F48D0ED000ACA
:1081B00030EE200A4D48D0ED000A70EE200AB1EEF4
:1081C000001A80EE810ADFED4A0A20EE200ABDEE99
:1081D000C00A10EE100A01B23F484183002181839A
:1081E000404890ED000AB1EE400A3D48D0ED000A4B
:1081F00030EE600A3C48D0ED000A30EE200A3B48E1
:10820000D0ED000A70EE200AB0EE001A80EE810A6E
:108210003848D0ED000A384890ED001A30EE811A47
:10822000C0EE010A9FED320A20EE800ABDEEC00AC0
:1082300010EE100A01B22848C18331E0284890EDC1
:10824000000A2848D0ED000A30EE200AF0EE000ABD
:1082500080EE201A9FED260A21EE000ABDEEC00A2C
:1082600010EE100A01B21C484183002181831D4891
:1082700090ED000A1A48D0ED000A30EE600A1E4860
:10828000D0ED000A80EE201A9FED190A21EE000AB7
:10829000BDEEC00A10EE100A01B20F48C18300BF44
:1082A00000BF1D4841880C4841841B48008840425B
:1082B00001B209488184184881880748C184174859
:1082C00041880548018515480088404201B20248AE
:1082D00041851348007825E08C06002064010020C9
:1082E000745A0020885A00209C5A0020B05A00205E
:1082F00000007A44900100208C0100200000000062
:1083000000000840000000000000004000000000E5
:1083100000408F40940100203602002030020020EF
:108320005C01002020B93B4881883B48818502E000
:10833000002139488185394890ED000A5FED140A23
:1083400020EE200ABDEEC00A10EE100A01B232483B
:108350000184007E30490870314800784870084632
:10836000408B000A88700846807EC8700846808B63
:10837000000A08710846007F48710846C08B000A51
:1083800088710846807FC8710846408C000A0872D0
:10839000084690F8220048720846808C000A8872CD
:1083A000084690F82400C8720846C08C000A08737A
:1083B000084690F8260048730846008D000A887326
:1083C000084690F82800C8730846408D000A0874D3
:1083D000084690F82A0048740846808D000A887480
:1083E000084690F82C00C8740846008C000A0875EE
:1083F000084690F82000487501211620F9F7BCF8CE
:1084000005498875084690F82E00C875BDEC0A8BA2
:1084100010BD0000300200208C0600201800002053
:108420005C01002070B504460420FCF7BBFA0C4840
:10843000047025464FF47A704543012009490880AD
:108440004FF0E020006940F002004FF0E0210861A9
:1084500008464561006940F00100086170BD0000F8
:10846000C8000020CA00002070B5044603F048F997
:10847000012810D00B480088844206D309480088A0
:10848000B4FBF0F5284602F057FA06480088B4FB22
:10849000F0F100FB11444FF47A7104FB01F000F09D
:1084A00003F870BDCA00002070B5034600224FF0EB
:1084B000E02675690D4E367803FB06F44FF0E02692
:1084C000B16910E04FF0E026B06988420BD08842D5
:1084D00002D20E1A324402E02E1A0E4432440146F1
:1084E000A24200D300E0EDE700BF70BDC80000204D
:1084F00082B0CDE9000121F0004001909DED000B1C
:1085000002B051EC100B7047F0EE400AF5EEC00AD5
:10851000F1EE10FA02DBB0EE600A7047B1EE600ACD
:10852000FBE7000000BF054A128802F04002002A63
:10853000F9D0C2B2014B1B1D1A80704700440040A5
:1085400010B503F0DDF8012802D003F0E9F810BD02
:1085500001480068FBE70000CC00002009E0054866
:108560000068C0430449C1F8B0020448006802F042
:10857000E3F9F4E7B0024042000040423800002036
:108580001CB501F0FDFD0748012100230A02CDE9D9
:10859000001005A1074803F083F802F0D7FB002084
:1085A0001CBD00000000002073746172745F746170
:1085B000736B000081A0000810B50246012000E0A6
:1085C00050430B1EA1F10104E1B2F9D110BD00002E
:1085D00038B54FF4AD70FE4908600A210920FAF75A
:1085E00007F9FB49096890FBF1F4052C00DD05242F
:1085F000F84890ED000ADFEDF80A20EE200ABDEE03
:10860000C00AF64880ED000AF5480068401CF449AD
:108610000860F448006800287ED1062C28D2DFE8E4
:1086200004F003090F151B21EFA200210846FBF7F8
:10863000E3F81DE0EEA200210846FBF7DDF817E0A5
:10864000EDA200210846FBF7D7F811E0ECA20021CB
:108650000846FBF7D1F80BE0EBA200210846FBF738
:10866000CBF805E0EAA200210846FBF7C5F800BFF9
:1086700000BFE948007818B1E748007801282AD1FE
:10868000E6A200213720FBF7B7F8E548B0F904006F
:10869000002810DAE3A200215020FBF7ADF80C20EF
:1086A0000090DF48B0F904004242052300215A201F
:1086B000FBF758F84BE0DCA200215020FBF79CF8B8
:1086C0000C200090D648B0F90420052300215A2040
:1086D000FBF748F83BE0D048007802280BD0CE48A2
:1086E0000078032807D0CC480078042803D0CA4873
:1086F000007805282BD1CDA200213720FBF77CF88C
:10870000CC48B0F90400002812DAC6A200215A2091
:10871000FBF772F80C2000E0FEE30090C548B0F9CA
:1087200004004242032300216420FBF71BF80EE003
:10873000BDA200215A20FBF75FF80C200090BD4835
:10874000B0F90420032300216420FBF70BF8B248A2
:10875000007838B1B0480078012803D0AE480078DE
:10876000042878D1B4A20A210020FBF745F8B348C9
:1087700090ED020AB5EEC00AF1EE10FA19D2A9A2E4
:108780000A210F20FBF738F80C200090AB4890ED41
:10879000020AB1EE400ADFEDAA0A20EE200ABCEE82
:1087A000C00A10EE102A05230A211420FAF7DAFF76
:1087B00016E09DA20A210F20FBF71EF80C20009066
:1087C0009E4890ED020ADFED9E0A20EE200ABCEEE4
:1087D000C00A10EE102A05230A211420FAF7C2FF5E
:1087E000964890ED000AB5EEC00AF1EE10FA19D2E3
:1087F0008CA20A213C20FAF7FFFF0C2000908F4842
:1088000090ED000AB1EE400ADFED8D0A20EE200A5D
:10881000BCEEC00A10EE102A05230A214B20FAF7FD
:10882000A1FF4EE080A20A213C20FAF7E5FF0C20D0
:108830000090824890ED000ADFED810A20EE200AC8
:10884000BCEEC00A10EE102A05230A214B20FAF7CD
:1088500089FF36E0FFE770480078022807D06E48AD
:108860000078032803D06C480078052829D175A228
:108870000A210020FAF7C0FF6948B0F90400002877
:1088800010DA68A20A213C20FAF7B6FF0C2000900B
:108890006348B0F90400424205230A214B20FAF74D
:1088A00061FF0EE060A20A213C20FAF7A5FF0C2030
:1088B00000905B48B0F9042005230A214B20FAF709
:1088C00051FF5548007838B153480078012803D04B
:1088D00051480078042879D15CA214210020FAF7CD
:1088E0008BFF5B4890ED020AB5EEC00AF1EE10FA7C
:1088F00019D24CA214210F20FAF77EFF0C20009011
:10890000534890ED020AB1EE400ADFED4D0A20EE29
:10891000200ABCEEC00A10EE102A052314210846D6
:10892000FAF720FF16E040A214210F20FAF764FFA7
:108930000C200090464890ED020ADFED410A20EE3F
:10894000200ABCEEC00A10EE102A052314210846A6
:10895000FAF708FF3E4890ED000AB5EEC00AF1EEC6
:1089600010FA19D22FA214213C20FAF745FF0C204F
:108970000090374890ED000AB1EE400ADFED300A72
:1089800020EE200ABCEEC00A10EE102A05231421A6
:108990004B20FAF7E7FE16E023A214213C20FAF759
:1089A0002BFF0C2000902A4890ED000ADFED240AEE
:1089B00020EE200ABCEEC00A10EE102A0523142176
:1089C0004B20FAF7CFFE23A21E2145E0BEE00000B7
:1089D00060010020180000200000C842140200209E
:1089E00028020020B80100204D656320000000002F
:1089F0004F6D6E6900000000416B6D2000000000AB
:108A000044696666000000003457442000000000FE
:108A100054616E6B0000000064010020475A0000A2
:108A2000300200202D0000002B000000424941537D
:108A3000000000005002002041000000745A002095
:108A400000007A444759524F5F5A3A0042000000F2
:108A5000885A0020430000000020FAF7CDFEFD48B0
:108A600090ED020AB5EEC00AF1EE10FA1AD2AFF29A
:108A70004C021E210F20FAF7BFFE0C200090F54893
:108A800090ED020AB1EE400A5FED130A20EE200AD3
:108A9000BCEEC00A10EE102A05231E211420FAF79E
:108AA00061FE17E0AFF280021E210F20FAF7A4FE4C
:108AB0000C200090E74890ED020A5FED1F0A20EEBF
:108AC000200ABCEEC00A10EE102A05231E21142035
:108AD000FAF748FEDF4890ED000AB5EEC00AF1EE65
:108AE00010FA1AD2AFF2C4021E213C20FAF784FE1B
:108AF0000C200090D74890ED000AB1EE400A5FEDDF
:108B0000300A20EE200ABCEEC00A10EE102A05231F
:108B10001E214B20FAF726FE1AE1AFF2F4021E21C5
:108B20003C20FAF769FE0C200090CA4890ED000A3C
:108B30005FED3D0A20EE200ABCEEC00A10EE102ABE
:108B400005231E214B20FAF70DFE01E1C2480078F3
:108B5000022807D0C0480078032803D0BE48007818
:108B60000528D9D1BDA214210020FAF745FEBC4842
:108B700090ED020AB5EEC00AF1EE10FA1AD2AFF289
:108B80005C1214210F20FAF737FE0C200090B44835
:108B900090ED020AB1EE400A5FED570A20EE200A7E
:108BA000BCEEC00A10EE102A052314210846FAF77D
:108BB000D9FD17E0AFF2901214210F20FAF71CFE36
:108BC0000C200090A64890ED020A5FED630A20EEAB
:108BD000200ABCEEC00A10EE102A05231421084614
:108BE000FAF7C0FD9E4890ED000AB5EEC00AF1EE1E
:108BF00010FA1AD2AFF2D41214213C20FAF7FCFD7D
:108C00000C200090964890ED000AB1EE400A5FED0E
:108C1000740A20EE200ABCEEC00A10EE102A0523CA
:108C200014214B20FAF79EFD17E0AFF20422142125
:108C30003C20FAF7E1FD0C200090894890ED000AF5
:108C40005FED810A20EE200ABCEEC00A10EE102A69
:108C5000052314214B20FAF785FD82A21E21002056
:108C6000FAF7CAFD804890ED020AB5EEC00AF1EEAF
:108C700010FA1AD2AFF254221E210F20FAF7BCFDCF
:108C80000C200090784890ED020AB1EE400A5FEDAA
:108C9000940A20EE200ABCEEC00A10EE102A05232A
:108CA0001E211420FAF75EFD17E0AFF284221E2188
:108CB0000F20FAF7A1FD0C2000906B4890ED020AFE
:108CC0005FEDA10A20EE200ABCEEC00A10EE102AC9
:108CD00005231E211420FAF745FD634890ED000A94
:108CE000B5EEC00AF1EE10FA1AD2AFF2C8221E2178
:108CF0003C20FAF781FD0C2000905B4890ED000AC3
:108D0000B1EE400A5FEDB20A20EE200ABCEEC00AC6
:108D100010EE102A05231E214B20FAF723FD17E041
:108D2000AFF2FC221E213C20FAF766FD0C200090D9
:108D30004D4890ED000A5FEDBE0A20EE200ABCEE21
:108D4000C00A10EE102A05231E214B20FAF70AFD57
:108D50004148007818B140480078042879D143A2EE
:108D600028210020FAF748FD414890ED020AB5EEAF
:108D7000C00AF1EE10FA1AD2AFF2583228210F20B1
:108D8000FAF73AFD0C200090394890ED020AB1EE56
:108D9000400A5FEDD50A20EE200ABCEEC00A10EEB4
:108DA000102A052328211420FAF7DCFC17E0AFF283
:108DB000883228210F20FAF71FFD0C2000902C4844
:108DC00090ED020A5FEDE20A20EE200ABCEEC00A36
:108DD00010EE102A052328211420FAF7C3FC24489A
:108DE00090ED000AB5EEC00AF1EE10FA1AD2AFF219
:108DF000CC3228213C20FAF7FFFC0C2000901C48C4
:108E000090ED000AB1EE400A5FEDF30A20EE200A71
:108E1000BCEEC00A10EE102A052328214B20FAF7D9
:108E2000A1FC05E1AFF2004228213C20FAF7E4FC66
:108E30000C2000900E4890ED000ADFED0E0A20EEA7
:108E4000200ABCEEC00A10EE102A052328214B2070
:108E500012E014E09C5A0020640100204C3A00000B
:108E6000745A0020523A0000885A00204400000042
:108E7000B05A002000007A44FAF774FCD8E0B148F8
:108E8000007801282CD1B0A228210020FAF7B4FCE8
:108E9000AF48B0F91A00002811DAAFF27842282161
:108EA0003C20FAF7A9FC0C200090A948B0F91A0060
:108EB0004242052328214B20FAF754FCB8E0AFF2D8
:108EC000984228213C20FAF797FC0C200090A048FB
:108ED000B0F91A20052328214B20FAF743FCA7E01C
:108EE0009848007802282BD19AA228210020FAF76E
:108EF00083FC9A480068002812DAAFF2D842282191
:108F00003C20FAF779FC0C20042300909348006879
:108F100042422821502000E011E1FAF723FC87E0CB
:108F2000AFF2FC4228213C20FAF766FC0C20042317
:108F300000908A48282102685020FAF713FC77E055
:108F400080480078032803D07E48007805286FD138
:108F500083A228210020FAF74FFC824890ED010AF5
:108F6000B5EEC00AF1EE10FA16D2AFF2485228213F
:108F70001420FAF741FC0C2000907A4890ED010A89
:108F8000B1EE400ABCEEC00A10EE102A04232821DC
:108F90001E20FAF7E7FB13E0AFF2745228211420E9
:108FA000FAF72AFC0C2000906E4890ED010ABCEE06
:108FB000C00A10EE102A042328211E20FAF7D2FB43
:108FC00069A228213C20FAF717FC684890ED010AB5
:108FD000B5EEC00AF1EE10FA16D2AFF2B85228215F
:108FE0005020FAF709FC0C200090604890ED010A2F
:108FF000B1EE400ABCEEC00A10EE102A042328216C
:109000005A20FAF7AFFB13E0AFF2E45228215020C8
:10901000FAF7F2FB0C200090544890ED010ABCEEE8
:10902000C00A10EE102A042328215A20FAF79AFBCE
:109030004F480078012805D14EA232210020FAF7CE
:10904000DBFB33E04D480078012805D14CA23221EA
:109050000020FAF7D1FB29E04B480078012805D120
:109060004AA232210020FAF7C7FB1FE049480078E6
:10907000012805D148A232210020FAF7BDFB15E0F6
:109080004748007810B94748007808B1012000E04F
:109090000020012805D144A232210020FAF7ACFBC0
:1090A00004E043A232210020FAF7A6FB4248006800
:1090B000012808D14148007828B941A232212D2049
:1090C000FAF79AFB04E03FA232212D20FAF794FB35
:1090D0003D480068642190FBF1F50C2002232A46EC
:1090E000322100904B20FAF73DFB38A23221582064
:1090F000FAF782FB34480068642190FBF1F201FB2F
:1091000012050C2002232A46322100906220FAF731
:1091100029FB2FA232216E20FAF76EFB2A48006845
:10912000642190FBF1F201FB12000A2807DA0C20FF
:1091300002230022322100905C20FAF713FBFAF799
:1091400097FA38BD640100204D4F56455F5A000024
:109150008C060020534552564F3A0000680100200B
:109160004D410000745A00204D420000885A0020F2
:109170009801002050533220200000009901002067
:1091800041505020200000009A010020522D432021
:10919000200000009B01002043414E2020000000E1
:1091A0009C0100209D0100205553415254000000B5
:1091B000524F5320200000000C8241425C010020ED
:1091C0004F204E004F464600140200202E000000A3
:1091D000560000002DE9F04105460E461C48076880
:1091E0001C480068001D01F0E9F950B919480068F1
:1091F00090F82C10012088401749096881431648CF
:109200000160681C38B936B112480168091D13485D
:1092100001F012FA1AE07C190E4800684460BC4262
:1092200007D20C480168091D0D48006801F0EAF9F1
:109230000CE008480168091D0A48006801F0E2F9DD
:1092400009480068844201D207480460BDE8F08103
:10925000FC000020E8000020000100202C0A002073
:10926000F0000020EC0000201801002010B504469A
:1092700001F0EEF924480068401C234908602348A7
:10928000006840B9214804600846006801280DD1F3
:1092900000F0EEF90AE01E48006838B91B48006883
:1092A000C06AE16A884201D8184804601948006819
:1092B000401C1849086008460068606494F82C1047
:1092C0000120884014490968084313490860E16A8D
:1092D00001EB8101114A02EB8100211D01F0ACF983
:1092E00001F0FAF90A48006868B108480068C06AE5
:1092F000E16A884207D24FF0805009490860BFF305
:109300004F8FBFF36F8F10BDF8000020E8000020E2
:109310000401002014010020000100205C0700204F
:1093200004ED00E010B501F093F910480068D0B9E1
:109330000F4801F057F90F4801F054F90C480E4955
:1093400008600C480D49086000221021052001F03A
:1093500077FE064908600846006820B108A1034866
:10936000006801F0ADFA01F0B7F910BD2C01002042
:10937000400A0020540A0020240100202801002077
:10938000546D72510000000070B523E001F034FD0F
:109390001348006808B9012000E00020054602F0EB
:1093A0003BFBBDB901F054F90D48C068C468201DED
:1093B00001F004F90B480068401E0A4908600A4899
:1093C0000068401E0849086001F086F9204600F058
:1093D00060F800BF044800680028D7D170BD0000C5
:1093E000180A0020F8000020F400002070B50446A0
:1093F0000D46206C70B1216CE0680844E060616843
:10940000E068884201D32068E0602846226CE16869
:10941000F7F756F870BD2DE9F04104460F461546A2
:109420004FF00008A66B206C40B9206860BB6068F4
:1094300002F02CFA80460020606025E07DB93946B4
:10944000226CA068F7F73CF8216CA0680844A06083
:10945000D4E90110884217D32068A06014E039468F
:10946000226CE068F7F72CF8216CE068401AE060A5
:109470002168E068884203D2216C6068401AE0608D
:10948000022D01D106B1761E701CA0634046BDE8D6
:10949000F08110B50446206B01F056F9204601F02A
:1094A00053F910BD0146084A126812680AB9012230
:1094B00000E000220A600A6822B9034A1268D268F2
:1094C000106800E0002070472401002030B54FF400
:1094D000A043174800F007042CB1C01D20F007007E
:1094E000134C041B1B1B0246124C22600024114D1E
:1094F0006C60D018083820F007000F4C2060002462
:109500000D4D2D686C600C4D2D682C601146441A71
:109510004C60094C24680C60084D4C682C60084D68
:109520004C682C604FF00044064D2C6030BD0000AC
:10953000680A0020440100204C0100205401002052
:10954000500100205801002000BFFFF71DFF064812
:1095500000680128F9D94FF0805004490860BFF332
:109560004F8FBFF36F8FF0E75C07002004ED00E042
:109570002DE9F04106460D4617469846069C0DB962
:10958000246000E02760E66325640121204601F0A5
:1095900075FE84F850800020A064BDE8F0810000D2
:1095A0002DE9F05F82460F4690469B460A9E0C9C32
:1095B0004FEA8801A522206BF6F7C7FFA8F101004A
:1095C000216B01EB800929F0070909F0070008B9B0
:1095D000012000E0002028B940F22B321BA120A07E
:1095E000F6F7C8FE002507E0795D04F13400415527
:1095F000785D00B902E06D1C102DF5D300BF00218D
:1096000043200155202E00D31F26E662E664002089
:109610002065201D00F0F3FF04F1180000F0EFFFBB
:109620002461C6F12000A06164620020606584F8B6
:1096300058005A465146484600F00EFC20600B98F0
:1096400008B10B980460BDE8F09F00002E2E5C4628
:1096500072656552544F535C7461736B732E630073
:109660004572726F723A25732C25640D0A00000052
:1096700010B5002407E004EB84010F4A02EB8100DF
:1096800000F0B0FF641C202CF5D30C4800F0AAFFBA
:109690000B4800F0A7FF0B4800F0A4FF0A4800F0B9
:1096A000A1FF0A4800F09EFF0448094908600448E9
:1096B0000849086010BD00005C070020DC0900209C
:1096C000F0090020040A0020180A00202C0A0020BB
:1096D000EC000020F000002010B50146164800E024
:1096E000006803688B42FBD30246436813448B42F5
:1096F00004D143684C682344436001460A464B68E2
:1097000013440468A34211D10C4C03682468A3429B
:1097100008D04B680468646823444B6003681B6886
:109720000B6005E0054B1B680B6001E003680B60F4
:10973000884200D0016010BD440100204C0100208F
:109740002DE9F04104460D4616461F464FF000082D
:1097500065602461B5420CD8F01BA169884202D330
:109760004FF0010811E0211D0948006800F04AFF90
:109770000BE0BE4204D2BD4202D34FF0010804E028
:10978000211D0448006800F03DFF4046BDE8F0811F
:10979000280100202401002070B5054600F058FF84
:1097A000A86B08B9012400E0002400F095FF2046D2
:1097B00070BD70B5054600F04BFFA86BE96B8842A1
:1097C00001D1012400E0002400F086FF204670BD96
:1097D0002DE9F3410D460098846C00272CB940F622
:1097E000CE121AA11EA0F6F7C5FDA06BE16B884250
:1097F00001D2012000E0002028B940F6CF1213A1C9
:1098000017A0F6F7B7FDA06BE16B88421BD294F965
:1098100045602A4669462046FFF7FDFD0746701C55
:1098200060B9606A08B9012000E0002050B904F175
:10983000240002F097F828B1012703E0701C40B221
:1098400084F8450000BF3846BDE8FC812E2E5C46FA
:1098500072656552544F535C71756575652E630072
:109860004572726F723A25732C25640D0A00000050
:10987000F8B505460F4613480068C068C468201D47
:1098800000F09CFEE069012818D1A06941192B461F
:109890003A462046FFF754FF80B1002003462A468F
:1098A00001460090204602F081F906462EB94FF499
:1098B000027205A10AA0F6F75DFD00BF2046616AAD
:1098C0008847F8BD240100202E2E5C467265655243
:1098D000544F535C74696D6572732E630000000011
:1098E0004572726F723A25732C25640D0A000000D0
:1098F000F0B587B070E0039800280CDA04AE2EB9FA
:1099000040F2E7223AA140A0F6F734FDD6E9002064
:10991000B168904700BF039800285DDB059C606933
:1099200008B9012000E0002010B9201D00F046FE1B
:1099300002A800F0C7F8054603980A284AD2DFE8D3
:1099400000F00905072C2E4506082D2F00BF00BF8B
:1099500000BF00BF0498A269811803462A4620462A
:10996000FFF7EEFEC0B12046616A8847E069012832
:1099700012D1002000900498A169421800231946D2
:10998000204602F013F907462FB940F2213218A100
:109990001DA0F6F7EFFC00BF1DE000BF1BE000BFFD
:1099A0000498A061A06908B1012000E0002028B956
:1099B0004FF44E720EA114A0F6F7DCFCA069411919
:1099C0002B462A462046FFF7BBFE04E0204600F067
:1099D000BBFE00E000BF00BF00231A4603A90E48EB
:1099E000006801F067FB002885D107B0F0BD0000DA
:1099F0002E2E5C4672656552544F535C74696D65DA
:109A000072732E63000000004572726F723A257304
:109A10002C25640D0A0000002C010020F8B5054635
:109A20000C4601F0E9F9684600F04CF8064600984B
:109A300020BB44B9B54206D801F0EEFF31462846B6
:109A4000FFF716FF1CE03CB10E480068006808B93B
:109A5000012000E000200446A91B22460A480068B5
:109A600000F044FF01F0D8FF50B94FF08050074993
:109A70000860BFF34F8FBFF36F8F01E001F0CCFFA1
:109A8000F8BD0000280100202C01002004ED00E0BA
:109A90000A490968096809B9012100E0002121B1DA
:109AA0004FF0FF31064A116006E004490968C968B1
:109AB000C868034A4168116070470000EC0000204C
:109AC0001801002070B5044601F02AFE054607483B
:109AD0000068854204D200F00BF80120206001E00C
:109AE0000020206001480560284670BD3401002038
:109AF0002DE9F8432DE021480068C06805681F483B
:109B00000068C068C468201D00F058FD2046616AE6
:109B10008847E06901281CD1A0694619AE4207D9DF
:109B200066602461211D1548006800F06BFD10E09F
:109B3000002003462A4601460090204602F036F8EF
:109B400007462FB940F292320DA113A0F6F712FC8E
:109B500000BF0A480068006808B9012000E0002042
:109B60000028C8D00548D0F800800F480068034995
:109B700008600D48C0F80080BDE8F883240100208B
:109B80002E2E5C4672656552544F535C74696D6548
:109B900072732E63000000004572726F723A257373
:109BA0002C25640D0A000000280100200C480068E4
:109BB000401C08B9012000E0002028B940F20F1233
:109BC00008A113A0F6F7D6FB00BF502080F3118840
:109BD000BFF34F8FBFF36F8F00BF00BFFEE70000E2
:109BE000380100202E2E5C4672656552544F535C3E
:109BF000706F727461626C655C525644535C415282
:109C00004D5F434D34465C706F72742E63000000EC
:109C10004572726F723A25732C25640D0A0000009C
:109C200008B500BF6846FFF73DFC04462046009992
:109C3000FFF7F4FEFFF75CFEF4E770B5044600F0B2
:109C400007FD94F945501AE0A06C38B10021204678
:109C5000FFF7BEFD88B100F09DFF0EE0606A08B915
:109C6000012000E0002038B904F1240001F07AFE60
:109C700018B100F08FFF00E003E0681E45B2002D30
:109C8000E2DC00BFFF2084F8450000F025FD00F075
:109C9000DFFC94F9445010E0206908B9012000E08D
:109CA000002048B904F1100001F05CFE08B100F09A
:109CB00071FF681E45B200E001E0002DECDC00BF42
:109CC000FF2084F8440000F007FD70BD08B5FEF7E2
:109CD00037FC009005E00A21684600F067FEF9F7BE
:109CE000E5FEF8E72DE9F04104464FF0000801F0E9
:109CF00083F83E48006808B9FFF7E8FB3C48006875
:109D0000204000285FD1A4B1083404F0070080B1DE
:109D100004F00700C0F10800044404F0070008B98B
:109D2000012000E0002020B9BF2232A13BA0F6F7BD
:109D300021FB002C47D03D480068844243D83C4E6C
:109D40003046056801E02E462D686868A04202D2C0
:109D500028680028F7D125480068854233D030684C
:109D600000F10808286830606868001B102813D9C3
:109D70002F1907F0070008B9012000E0002020B9E2
:109D8000EC221CA125A0F6F7F5FA6868001B7860A4
:109D90006C603846FFF7A0FC244968680968081A17
:109DA000224908600846006822490968884203D2AF
:109DB0001E4800681F4908600D4968680968084323
:109DC00068600020286001F027FE08F0070008B94D
:109DD000012000E0002028B94FF4967205A10FA0E1
:109DE000F6F7C8FA4046BDE8F08100004C010020BB
:109DF000580100202E2E5C4672656552544F535C0C
:109E0000706F727461626C655C4D656D4D616E67FB
:109E10005C686561705F342E630000004572726F8C
:109E2000723A25732C25640D0A00000050010020B1
:109E300044010020540100200648006830B1054963
:109E4000096801F15000096D491C01600148006872
:109E500070470000E8000020001F4FF0807303608F
:109E6000001F21F001030360001F054B036014383D
:109E70000260001F6FF0020303602038704700008B
:109E8000AD9B000808B5FEF75BFB0090ADE0002439
:109E90006421684600F08AFD54480068322803DADD
:109EA0000120534908600AE050480068332806DB67
:109EB0004E480068642802DA00204D4908604D4889
:109EC0000068012803D04C480068012802D1002016
:109ED0004A49086049480068052804DA474800688C
:109EE000401C4649086045480068052803DA0120FF
:109EF0003F49086006E041480068052802D100207B
:109F00003B490860002409E0F8F78AFC3C48D0EDA2
:109F1000000A30EE200A80ED000A641C0A2CF3DBF4
:109F2000374890ED000AF2EE040A80EE201A354818
:109F300080ED001A9FED340A314880ED000A2D486B
:109F40000068012804D12B480068401C294908609A
:109F500029480068012804D127480068401C264988
:109F60000860284890ED000ADFED280AB4EEE00A08
:109F7000F1EE10FA04DB9FED250A80ED000A2FE0D8
:109F8000204890ED000AF2EE040AB4EEE00AF1EE89
:109F900010FA12DB90ED000AF2EE050AB4EEE00AC8
:109FA000F1EE10FA09D213480068022805DA1148C8
:109FB0000068401C0F49086012E0124890ED000A4A
:109FC000F2EE040AB4EEE00AF1EE10FA08D2094803
:109FD0000068022804DA08480068401C0649086046
:109FE000F6F7D8FCFEF7F4FA00BF50E7D4010020E2
:109FF000A002404220020020240200201C02002077
:10A000002000002018000020000000009A9949411B
:10A0100000B52DED048B83B041EC190B02F040FA32
:10A0200041EC180B18EE100A18EE901A8DED008B0B
:10A03000002818BF0120084320F00040C0F17F60D5
:10A0400000F1E040C00F14D019EE101A19EE900A7A
:10A050008DED009B002918BF0121084320F000402E
:10A06000C0F17F6000F1E040C00F04BF0120F6F7AF
:10A070009FFA51EC180B03B0BDEC048B00BD00003F
:10A080001CB5044600F0E4FA002004210346CA018E
:10A09000CDE900101FA1234801F002FB002003219D
:10A0A00003464FF48072CDE900101FA1224801F051
:10A0B000F7FA0020032103464FF40072CDE90010A7
:10A0C0001EA1214801F0ECFA002003210346802262
:10A0D000CDE900101DA1204801F0E2FA0020042182
:10A0E00003468A01CDE900101CA11F4801F0D8FAEF
:10A0F000002004210346CA01CDE900101BA11E481F
:10A1000001F0CEFA1D48006800F0BEFC00F0E4FA51
:10A110001CBD000042616C616E63655F7461736BAE
:10A1200000000000E10B00084D5055363035305F1F
:10A130007461736B000000009531000873686F77DD
:10A140005F7461736B000000859E00086C65645F3E
:10A150007461736B000000005D8500085053545714
:10A160004F5F7461736B0000CD9C00084441544103
:10A170005F7461736B000000AD7E0008000000207A
:10A1800008B54FF44070F9F783F9A820FEF74AF9B3
:10A19000F8F7F6FEF6F7B0FEF7F712FEF9F7CEF98C
:10A1A000F8F7BAFE4FF4E13000F06AF84FF41650B9
:10A1B00000F0BEF84FF4E13000F012F94FF4E13056
:10A1C00000F066F9F6F788FCF6F7C8FC00200323D8
:10A1D0000622072100900120F6F7AAFEFAF760F99F
:10A1E000F7F706FEF7F778FEF7F7D4FEF7F730FF3C
:10A1F000532142F20F70FAF75BFDA72142F20F7074
:10A20000FBF74AF8002144F29F10FAF7B7FD00214E
:10A2100044F29F10FBF7F2F8002144F29F10FAF786
:10A22000A3FC002144F29F10FAF7EEFCF8F770FB54
:10A23000F8F758FFF9F70EFCF9F714FD08BDF0EE3A
:10A24000401AF4EEE01AF1EE10FA02D2B0EE600A13
:10A250007047F4EEC11AF1EE10FA02DDB0EE410AD9
:10A26000F6E7B0EE610AF3E703468B4201DA0846EF
:10A270007047934201DD1046FAE71846F8E7000000
:10A2800010B588B0044601210846F9F77DFE01218A
:10A290001020F9F799FE072209212348F7F77EFFDE
:10A2A00007220A212048F7F779FF4FF4C060069093
:10A2B00002208DF81C0000208DF81E0002208DF871
:10A2C0001D0001208DF81F0006A91748F7F71EFF93
:10A2D00025208DF8040001208DF8050000208DF860
:10A2E000060001208DF8070001A8F9F795F80294FF
:10A2F0000020ADF80C00ADF80E00ADF81000ADF880
:10A3000014000C20ADF8120002A90848FBF786FFE4
:10A31000012240F225510548FBF75AFF012103486D
:10A32000FBF720FF08B010BD000002400010014004
:10A3300010B588B0044601210820F9F725FE012157
:10A340004804F9F731FE072205212348F7F726FFD5
:10A35000072206212048F7F721FF602006900220FF
:10A360008DF81C0000208DF81E0002208DF81D00C5
:10A3700001208DF81F0006A91748F7F7C7FE262011
:10A380008DF8040001208DF8050000208DF80600EE
:10A3900001208DF8070001A8F9F73EF8029400208B
:10A3A000ADF80C00ADF80E00ADF81000ADF81400DB
:10A3B0000C20ADF8120002A90848FBF72FFF01227C
:10A3C00040F225510548FBF703FF01210348FBF745
:10A3D000C9FE08B010BD0000000C0240004400405F
:10A3E00010B588B0044601210820F9F7CDFD012100
:10A3F0008804F9F7D9FD072208212348F7F7CEFE94
:10A40000072209212048F7F7C9FE4FF44070069053
:10A4100002208DF81C0000208DF81E0002208DF80F
:10A420001D0001208DF81F0006A91748F7F76EFEE2
:10A4300027208DF8040002208DF8050000208DF8FB
:10A44000060001208DF8070001A8F8F7E5FF029447
:10A450000020ADF80C00ADF80E00ADF81000ADF81E
:10A4600014000C20ADF8120002A90848FBF7D6FE34
:10A47000012240F225510548FBF7AAFE01210348BD
:10A48000FBF770FE08B010BD000C02400048004011
:10A4900010B588B0044601210420F9F775FD0121AB
:10A4A0000820F9F771FD01210805F9F77DFD082263
:10A4B0000C212C48F7F772FE082202212A48F7F7F0
:10A4C0006DFE4FF48050069002208DF81C00002095
:10A4D0008DF81E0002208DF81D0001208DF81F0050
:10A4E00006A92048F7F712FE0420069002208DF8F6
:10A4F0001C0000208DF81E0002208DF81D00012098
:10A500008DF81F0006A91848F7F700FE35208DF8D2
:10A51000040002208DF8050000208DF806000120BF
:10A520008DF8070001A8F8F777FF02940020ADF836
:10A530000C00ADF80E00ADF81000ADF814000C20C2
:10A54000ADF8120002A90948FBF768FE012240F2AB
:10A5500025510648FBF73CFE01210448FBF702FEAB
:10A5600008B010BD00080240000C0240005000403E
:10A570000449888000BF0349098801F0400100298F
:10A58000F9D07047001001400549088000BF044918
:10A59000091F098801F040010029F8D07047000028
:10A5A000044800400449888000BF0349098801F03D
:10A5B00040010029F9D070470050004001460A6967
:10A5C000D1E901309860D1E90103586050688842B0
:10A5D00001D188685060002008611068401E10603A
:10A5E0001068704700F1080141604FF0FF31816051
:10A5F00000F10801C1600161002101607047002184
:10A600000161704710B502460B685C1C0CB91069FB
:10A6100007E002F1080000E04068446824689C42BA
:10A62000FAD944684C604C68A160886041600A6156
:10A630001468641C146010BD42684A6093688B60A3
:10A64000936859609160086103685B1C0360704700
:10A6500010B500BF502080F31188BFF34F8FBFF3B8
:10A660006F8F00BF0B480068401C0A49086008460D
:10A67000006801280DD108480068C0B208B901205F
:10A6800000E0002028B940F2B91204A10EA0F5F7AD
:10A6900071FE10BD3801002004ED00E02E2E5C4656
:10A6A00072656552544F535C706F727461626C6571
:10A6B0005C525644535C41524D5F434D34465C708E
:10A6C0006F72742E630000004572726F723A2573C8
:10A6D0002C25640D0A00000010B50B48006828B94D
:10A6E0004FF4E07209A114A0F5F744FE0648006893
:10A6F000401E054908600846006820B9002080F324
:10A70000118800BF00BF10BD380100202E2E5C460E
:10A7100072656552544F535C706F727461626C6500
:10A720005C525644535C41524D5F434D34465C701D
:10A730006F72742E630000004572726F723A257357
:10A740002C25640D0A00000070B506463546002E23
:10A7500035D0083D2C461A4960680968084008B1A0
:10A76000012000E0002028B94FF4A07215A11FA01D
:10A77000F5F700FE206808B9012000E0002028B9A4
:10A7800040F241120FA119A0F5F7F4FD0C496068E1
:10A790000968084098B1206888B909496068096863
:10A7A0008843606000F028FB144960680968084429
:10A7B000124908602046FEF78FFF01F02DF970BDA9
:10A7C000580100202E2E5C4672656552544F535C32
:10A7D000706F727461626C655C4D656D4D616E6722
:10A7E0005C686561705F342E630000004572726FB3
:10A7F000723A25732C25640D0A00000050010020D8
:10A80000064800684FF47A71B0FBF1F0401E4FF03B
:10A81000E021486107200861704700000400002023
:10A8200070B5F5F781FD0546102D11D305F1E02037
:10A8300090F8F04310480078844201DB012000E0EA
:10A84000002028B94FF440720CA117A0F5F792FD33
:10A850001948006800F4E06018490968884201D886
:10A86000012000E0002028B94FF4447203A10EA09B
:10A87000F5F780FD70BD00003C0100202E2E5C46E7
:10A8800072656552544F535C706F727461626C658F
:10A890005C525644535C41524D5F434D34465C70AC
:10A8A0006F72742E630000004572726F723A2573E6
:10A8B0002C25640D0A0000000CED00E04001002092
:10A8C000024600200BE0084B53F8303033B9064BFA
:10A8D00043F8301003EBC0035A6002E0401C082824
:10A8E000F1D300BF704700001C0700202DE9F041A4
:10A8F00005460E4617462C46FFF7AAFE94F944007B
:10A90000401C10B9002084F8440094F94500401C14
:10A9100010B9002084F84500FFF7DEFEA06B28B9CF
:10A920003A46314604F1240000F064F92046FFF76E
:10A9300084F9BDE8F081000070B504460025ACB193
:10A940000F48006808B9012000E0002028B940F253
:10A95000CF420CA110A0F5F70DFD00F04DFA00213B
:10A960002046FEF737FC01F057F805463DB94FF099
:10A9700080500D490860BFF34F8FBFF36F8F70BDDC
:10A98000200100202E2E5C4672656552544F535CA8
:10A990007461736B732E63004572726F723A257324
:10A9A0002C25640D0A00000004ED00E02DE9F047BD
:10A9B00004460F464FF000092CB940F2794226A117
:10A9C0002AA0F5F7D7FC0FB1012000E0002028B93C
:10A9D00040F27A4220A125A0F5F7CCFC2748006878
:10A9E00008B9012000E0002028B940F27B421AA1FA
:10A9F0001EA0F5F7BFFC00F0FFF9214806682068AB
:10AA0000C5192068B04207D92068A8420BD9B542C1
:10AA100009D94FF0010906E02068A84201D8B542E3
:10AA200001D94FF001092560B9F1000F03D0A81B2F
:10AA30000021FEF7CFFB00F0EFFF8046B8F1000FDA
:10AA400007D14FF080500F490860BFF34F8FBFF31D
:10AA50006F8FBDE8F08700002E2E5C467265655250
:10AA6000544F535C7461736B732E63004572726F45
:10AA7000723A25732C25640D0A0000002001002085
:10AA8000FC00002004ED00E070B50546FFF7E0FD96
:10AA900015B92D48006800E028460446201DFFF740
:10AAA0008DFD78B9E06A00EB8000284951F820005C
:10AAB00040B994F82C100120884025490968814349
:10AAC00023480160A06A18B104F11800FFF776FD71
:10AAD00020480068401C1F4908601B4800688442E9
:10AAE00009D1211D1C48FFF7A7FD1C480068401C28
:10AAF0001A49086009E01A480068401E18490860B1
:10AB00002046FEF7C6FCFEF7C3FFFFF7E5FD15483C
:10AB10000068C0B10C480068844214D11248006833
:10AB200008B9012000E0002028B940F265420FA1D9
:10AB300013A0F5F71FFC4FF0805015490860BFF3D4
:10AB40004F8FBFF36F8F70BDE80000205C070020BF
:10AB50000001002014010020180A0020F400002049
:10AB6000F800002004010020200100202E2E5C4669
:10AB700072656552544F535C7461736B732E63003E
:10AB80004572726F723A25732C25640D0A0000001D
:10AB900004ED00E001200149086070470C0100202D
:10ABA00070B504460D462CB940F6063207A10CA03C
:10ABB000F5F7E0FB0E48016818312046FFF722FD4B
:10ABC00001212846FEF706FB70BD00002E2E5C46D4
:10ABD00072656552544F535C7461736B732E6300DE
:10ABE0004572726F723A25732C25640D0A000000BD
:10ABF000E800002070B505460E4614462DB940F613
:10AC0000313209A10DA0F5F7B5FB104801681831E4
:10AC10002846FFF711FD0CB14FF0FF3621463046B4
:10AC2000FEF7D8FA70BD00002E2E5C4672656552A4
:10AC3000544F535C7461736B732E63004572726F73
:10AC4000723A25732C25640D0A000000E8000020EC
:10AC500070B505462C46002D4BD02649E06A0968A0
:10AC6000C96A884245D2A06900F0004028B921484D
:10AC70000068C06AC0F12000A061E16A01EB8101B7
:10AC80001D4A02EB81016069884201D1012000E088
:10AC9000002050B3201DFFF791FC78B9E06A00EB6B
:10ACA0008000154951F8200040B994F82C1001207B
:10ACB0008840124909688143104801600D480068C6
:10ACC000C06AE06294F82C10012088400B490968A2
:10ACD00008430A490860E16A01EB8101064A02EB78
:10ACE0008100211DFFF7A8FC03E002480068C06A4C
:10ACF000E06270BDE80000205C0700200001002039
:10AD000010B504462CB940F6C13205A109A0F5F7EB
:10AD100031FB0C48006820600B480068606010BD83
:10AD20002E2E5C4672656552544F535C7461736B92
:10AD3000732E63004572726F723A25732C25640D71
:10AD40000A00000010010020FC0000201CB51A4879
:10AD500000210B468222CDE9001018A1194800F00D
:10AD60009FFC0446012C02D100F0E6FE0446012CB3
:10AD700015D100BF502080F31188BFF34F8FBFF370
:10AD80006F8F00BF4FF0FF300F49086001200F495F
:10AD9000086000200E49086000F08AF80BE0601C93
:10ADA00008B1012000E0002028B940F2847209A116
:10ADB0000DA0F5F7DFFA1CBD1C01002049444C45ED
:10ADC000000000004995000818010020040100203F
:10ADD000FC0000202E2E5C4672656552544F535C79
:10ADE0007461736B732E63004572726F723A2573D0
:10ADF0002C25640D0A00000002480068401C01492F
:10AE0000086070472001002010B51B48006818B189
:10AE100001201A4908602DE00020184908601848F0
:10AE20000068B0FA80F0C0F11F0404EB84001549FB
:10AE300051F8200008B1012000E0002028B940F6B8
:10AE4000F62211A115A0F5F795FA04EB84010D4A3D
:10AE500002EB810041684968416000F108014268E5
:10AE60008A4202D14168496841604168C9680F4A15
:10AE7000116000BF10BD0000200100200C01002067
:10AE8000000100205C0700202E2E5C467265655292
:10AE9000544F535C7461736B732E63004572726F11
:10AEA000723A25732C25640D0A000000E80000208A
:10AEB0001CB5404800684049884201D0012000E0AC
:10AEC000002028B940F259123CA147A0F5F752FAE8
:10AED000384800683849491E884201D0012000E006
:10AEE000002028B94FF4AD7234A13FA0F5F742FA23
:10AEF000414C204600780190FF202146087008460A
:10AF0000007800909DF8000000F0F0009DF800101F
:10AF1000884201D1012000E0002028B940F27312DC
:10AF200026A131A0F5F726FA9DF8000000F05000A8
:10AF30003249087007203249086009E0304800684B
:10AF4000401E2F4908609DF800004006000E00904A
:10AF50009DF8000000F080008028EFD028480068AD
:10AF60000002274908600846008800F4E060086095
:10AF70002149019808700F482030006840F47000A3
:10AF80000C49203108600846006840F070400860B5
:10AF9000FFF736FC00201B490860F5F78DF91A48C9
:10AFA000006840F0404018490860F5F775F9002046
:10AFB0001CBD000000ED00E071C20F412E2E5C466A
:10AFC00072656552544F535C706F727461626C6548
:10AFD0005C525644535C41524D5F434D34465C7065
:10AFE0006F72742E630000004572726F723A25739F
:10AFF0002C25640D0A00000000E400E03C01002064
:10B00000400100203801002034EF00E010B500BFFF
:10B01000502080F31188BFF34F8FBFF36F8F00BFB5
:10B0200000F084FB18B14FF080500449086000BF65
:10B03000002080F3118800BF10BD000004ED00E087
:10B040002DE9F84305460E4690460DB1012000E07B
:10B05000002028B94FF4C4720DA112A0F5F78AF9A7
:10B060000EB9002701E005FB06F707F15400FEF7D3
:10B0700039FE044644B104F1540943464A46314678
:10B0800028460094FEF774FA2046BDE8F8830000D5
:10B090002E2E5C4672656552544F535C7175657512
:10B0A000652E63004572726F723A25732C25640D0C
:10B0B0000A0000002DE9FF4782B005460E461F46F4
:10B0C0004FF0000A2C462CB940F2DC4261A166A088
:10B0D000F5F750F90EB9206C08B9012000E0002006
:10B0E00028B940F2DD425BA15FA0F5F743F900F01B
:10B0F00007FB08B9049808B9012000E0002028B92E
:10B100004FF49C6253A158A0F5F734F900BFFFF744
:10B110009FFAD4F83890B9F1000F3DD0D4F80C80E4
:10B1200031462046FEF762F9DFB9A9F10100A063BC
:10B13000206810B9FEF780FE6060206908B9012020
:10B1400000E0002010BB04F1100000F00BFCE8B19F
:10B150004FF0805048490860BFF34F8FBFF36F8FA7
:10B1600014E0C4F80C80606A08B9012000E00020F7
:10B1700060B904F1240000F0F5FB38B14FF08050C5
:10B180003D490860BFF34F8FBFF36F8FFFF7A4FAFD
:10B19000012006B0BDE8F087049818B9FFF79CFAC3
:10B1A0000020F6E7BAF1000F04D16846FFF7A8FDCA
:10B1B0004FF0010AFFF790FAFFF71EFEFFF748FA7B
:10B1C00094F94400401C10B9002084F8440094F91C
:10B1D0004500401C10B9002084F84500FFF77CFAB8
:10B1E00004A9684600F00CFA40BB2046FEF7D4FAEA
:10B1F000F0B1206830B9FFF72BFA6068FFF728FD3F
:10B20000FFF76AFA04F124000499FFF7C9FC20460D
:10B21000FEF713FD00F000FC00287FF478AF4FF03C
:10B22000805015490860BFF34F8FBFF36F8F6EE7F3
:10B230002046FEF702FD00F0EFFB68E72046FEF730
:10B24000FCFC00F0E9FB2046FEF7A6FA0028EED051
:10B2500000209EE72E2E5C4672656552544F535C6B
:10B2600071756575652E63004572726F723A25734C
:10B270002C25640D0A00000004ED00E070B50546C1
:10B280000E462C462CB940F21B121EA122A0F5F747
:10B2900071F8FFF7DDF9D4E90F12206801FB020015
:10B2A00060600020A0632068A060E06B401E226CFC
:10B2B000216800FB0210E060FF2084F8440084F85D
:10B2C00045009EB9206908B9012000E00020A8B916
:10B2D00004F1100000F046FB80B14FF0805012499D
:10B2E0000860BFF34F8FBFF36F8F07E004F11000CA
:10B2F000FFF778F904F12400FFF774F9FFF7ECF990
:10B30000012070BD2E2E5C4672656552544F535C11
:10B3100071756575652E63004572726F723A25739B
:10B320002C25640D0A00000004ED00E02DE9FF4328
:10B3300083B0064688461D464FF0000934462CB9B6
:10B3400040F2D92260A165A0F5F714F8B8F1000F1A
:10B3500001D1206C08B9012000E0002028B940F29A
:10B36000DA2259A15DA0F5F705F8022D02D1E06BB4
:10B37000012801D1012000E0002028B940F2DB22A1
:10B3800051A156A0F4F7F6FF00F0BAF908B90598F4
:10B3900008B9012000E0002028B940F2DE224AA1CD
:10B3A0004EA0F4F7E7FF00BFFFF752F9A06BE16B87
:10B3B000884201D3022D38D12A4641462046FEF765
:10B3C0002AF80746A06C68B129462046FEF700FA25
:10B3D00028B34FF0805045490860BFF34F8FBFF34B
:10B3E0006F8F1CE0606A08B9012000E0002068B996
:10B3F00004F1240000F0B6FA88B14FF080503B49C8
:10B400000860BFF34F8FBFF36F8F08E03FB14FF07D
:10B41000805036490860BFF34F8FBFF36F8FFFF73F
:10B420005BF9012007B0BDE8F083059818B9FFF774
:10B4300053F90020F6E7B9F1000F04D101A8FFF796
:10B440005FFC4FF00109FFF747F9FFF7D5FCFFF765
:10B45000FFF894F94400401C10B9002084F844001F
:10B4600094F94500401C10B9002084F84500FFF70E
:10B4700033F905A901A800F0C3F8F0B92046FEF79A
:10B4800098F9A0B104F110000599FFF789FB204657
:10B49000FEF7D3FB00F0C0FA002885D14FF08050B2
:10B4A00012490860BFF34F8FBFF36F8F7CE72046D0
:10B4B000FEF7C3FB00F0B0FA76E72046FEF7BDFBCF
:10B4C00000F0AAFA0020ADE72E2E5C4672656552A8
:10B4D000544F535C71756575652E63004572726FCC
:10B4E000723A25732C25640D0A00000004ED00E07B
:10B4F0002DE9F05F80468A4615461E4644462CB923
:10B5000040F29F3235A13AA0F4F734FFBAF1000FB0
:10B5100001D1206C08B9012000E0002028B94FF4C7
:10B5200068722EA132A0F4F725FF022E02D1E06B43
:10B53000012801D1012000E0002028B940F2A13209
:10B5400026A12BA0F4F716FFFFF76AF900BF5021E0
:10B55000EFF3118081F31188BFF34F8FBFF36F8F2B
:10B5600000BF0746A06BE16B884201D3022E2BD1AE
:10B5700094F945B0324651462046FDF74CFF0BF199
:10B580000100C8B9A06C40B131462046FEF720F951
:10B59000B8B1B5B10120286013E0606A08B9012094
:10B5A00000E0002068B904F1240000F0DBF940B1AC
:10B5B0003DB10120286004E00BF1010040B284F8A5
:10B5C00045004FF0010901E04FF0000900BF87F38B
:10B5D000118800BF4846BDE8F09F00002E2E5C4653
:10B5E00072656552544F535C71756575652E6300C5
:10B5F0004572726F723A25732C25640D0A000000A3
:10B600002DE9F04104460D462CB940F6CB3219A184
:10B610001DA0F4F7AFFE2DB940F6CC3215A11AA04B
:10B62000F4F7A8FEFFF714F81B4807682868401CC9
:10B6300008B9002619E0194920680968884204D031
:10B640006068B84201D801260FE06068381A29689E
:10B65000884209D228686168791A401A2860204611
:10B66000FFF74EFB002600E00126FFF735F83046D5
:10B67000BDE8F0812E2E5C4672656552544F535CD6
:10B680007461736B732E63004572726F723A257327
:10B690002C25640D0A000000FC0000201001002091
:10B6A0002DE9FF4F85B0804689461746DDE912AB8C
:10B6B000B800FEF717FB064656B15C20FEF712FBFA
:10B6C00004460CB1266304E03046FFF73DF800E085
:10B6D00000247CB10020CDE900ABCDE902403A4620
:10B6E00049464046089BFDF75BFF2046FDF7BEFD3F
:10B6F000012501E04FF0FF35284609B0BDE8F08F85
:10B700000549096809B9012005E00449096809B932
:10B71000022000E0002070470401002020010020EA
:10B720000149086870470000FC0000202DE9F04145
:10B730004FF0000841480068002872D14048006876
:10B74000451C3F480560EDB93E480068006808B9EF
:10B75000012000E0002028B940F6D9123AA13FA00C
:10B76000F4F708FE37480768404800683549086024
:10B770003E4807603E480068401C3D490860FEF7AF
:10B7800087F900BF3B48006885423CD300BF2D4885
:10B790000068006808B9012000E0002020B14FF0E7
:10B7A000FF30344908602DE026480068C068C4684E
:10B7B0006668B54202D22F48066023E0201DFEF7DE
:10B7C000FDFEA06A18B104F11800FEF7F7FE94F828
:10B7D0002C10012088402849096808432649086040
:10B7E000E16A01EB8101254A02EB8100211DFEF790
:10B7F00023FF2349E06A0968C96A8842C7D34FF02A
:10B800000108C4E700BF1E480068C06A00EB800062
:10B810001A4951F82000012801D94FF0010805E02C
:10B82000FFE718480068401C164908601648006881
:10B8300008B14FF001084046BDE8F081200100202A
:10B84000FC000020EC0000202E2E5C467265655244
:10B85000544F535C7461736B732E63004572726F47
:10B86000723A25732C25640D0A000000F0000020B8
:10B870001001002018010020000100205C070020BA
:10B88000E8000020080100200C01002070B50546EA
:10B890002C460026002D4BD026480068844201D15A
:10B8A000012000E0002028B940F6C76222A127A0AD
:10B8B000F4F760FD206D28B940F6C9621EA123A0EF
:10B8C000F4F758FD206D401E2065E16CE06A884267
:10B8D0002ED0206D60BB201DFEF770FE78B9E06AA7
:10B8E00000EB80001D4951F8200040B994F82C105D
:10B8F000012088401A490968814319480160E06CB9
:10B90000E062E06AC0F12000A06194F82C100120F0
:10B91000884013490968084311490860E16A01EB4E
:10B9200081010E4A02EB8100211DFEF785FE0126F2
:10B93000304670BDE80000202E2E5C4672656552D0
:10B94000544F535C7461736B732E63004572726F56
:10B95000723A25732C25640D0A0000005C07002054
:10B960000001002070B50646F068C4682CB940F6A6
:10B9700061321AA11EA0F4F7FDFC04F11800FEF7D5
:10B980001DFE1F480068A8B9201DFEF717FE94F899
:10B990002C10012088401B49096808431949086098
:10B9A000E16A01EB8101184A02EB8100211DFEF7DB
:10B9B00043FE04E004F118011448FEF73DFE14496B
:10B9C000E06A0968C96A884204D901250120114941
:10B9D000086000E00025284670BD00002E2E5C4661
:10B9E00072656552544F535C7461736B732E6300C0
:10B9F0004572726F723A25732C25640D0A0000009F
:10BA000020010020000100205C070020040A002023
:10BA1000E80000200C01002070B500240026344806
:10BA2000006828B94FF4FD6232A137A0F4F7A2FCF8
:10BA3000FEF70EFE2E480068401E2D49086008469D
:10BA4000006800284FD13448006800284BD024E01B
:10BA50003248C068C46804F11800FEF7AFFD201D2D
:10BA6000FEF7ACFD94F82C10012088402C490968A1
:10BA700008432B490860E16A01EB8101294A02EB86
:10BA80008100211DFEF7D8FD2749E06A0968C96ACF
:10BA9000884202D30120254908602048006808B97F
:10BAA000012000E000200028D2D00CB1FDF7F0FF0B
:10BAB0001F48056865B100BFFFF738FE10B10120CF
:10BAC0001A4908606D1E002DF6D100201849086043
:10BAD0001648006838B10126300716490860BFF3E0
:10BAE0004F8FBFF36F8FFEF7F7FD304670BD00003C
:10BAF000200100202E2E5C4672656552544F535C27
:10BB00007461736B732E63004572726F723A2573A2
:10BB10002C25640D0A000000F8000020040A002013
:10BB2000000100205C070020E80000200C0100203C
:10BB30000801002004ED00E01CB50024FDF7F2FB35
:10BB40000B48006858B10B481F2100234FF4827244
:10BB5000CDE9001008A10A48FFF7A2FD04462CB960
:10BB600040F2331207A10DA0F4F704FC20461CBDDF
:10BB70002C01002030010020546D722053766300A8
:10BB8000219C00082E2E5C4672656552544F535C12
:10BB900074696D6572732E63000000004572726FE8
:10BBA000723A25732C25640D0A0000002DE9FF4729
:10BBB00004460D4616461F46DDF830804FF000095A
:10BBC0002CB94FF4D37217A11CA0F4F7D3FB1F4874
:10BBD000006810B3009501960294062D15DAFFF760
:10BBE0008FFD022808D100234246694617480068A5
:10BBF000FFF79CFB814610E000231A466946134874
:10BC00000068FFF793FB814607E000233A46694648
:10BC10000E480068FFF76CFC8146484604B0BDE85A
:10BC2000F08700002E2E5C4672656552544F535CBF
:10BC300074696D6572732E63000000004572726F47
:10BC4000723A25732C25640D0A0000002C01002097
:10BC500081F00041704780F00040704721F00041C2
:10BC6000704720F00040704721F00042A2F160527E
:10BC7000B2F5801F01F0004328BFD2F17F6C0BD9D1
:10BC80005FEA001C43EAC20242EB507018BF7047E3
:10BC900028BF20F001007047B2F5801FBCBF1846D6
:10BCA00070474FEA410C1CF5001F02D2084600F015
:10BCB00023BE70B500F05EFB00000089FFF7F6BF01
:10BCC0004FF00040A0F580007047000010B591EAE9
:10BCD000030F48BF83F0004300F1B684841A71EB70
:10BCE000030C05D2121943EB0C03001B61EB0C0192
:10BCF000DFF824E14FEA1154A4EB135C1EEA430F72
:10BD000018BF9EEA445F73D023EA0E03DCF1200ED5
:10BD100021EA045143F4801332D322FA0CFE10EBD3
:10BD20000E0023FA0CFE41EB0E01CCF1200E03FABB
:10BD30000EFE10EB0E0051F10001B1F5801FCCF1A9
:10BD4000200E32D201EB045112FA0EF2BDE810407F
:10BD500058BF7047401C38BF5FEA420218BF7047A7
:10BD6000002814BF20F0010041F100014FEA410317
:10BD700013F5001F38BF7047A1F1C04100F048BB68
:10BD8000012A43EB0302ACF1200CDCF11F0E32BFA1
:10BD90004FF0000E23FA0CF310EB030041EB0451BB
:10BDA000B4EB115FD0D0A1EB045101F5801149082B
:10BDB0005FEA300001EB04510ED350F1000038BFB0
:10BDC00012FA0EFE08D1BDE81040C9E7401C38BF8A
:10BDD0005FEA4202CAD1C3E7BDE810404FEA41031F
:10BDE00013F5001F38BF7047A1F1C04100F010BB30
:10BDF0009EEA445F08D011EA5E0FBDE8104004BF20
:10BE000001F0004100207047BDE8104070B500F01F
:10BE1000B1FA00BF64FBBE3E0000E0FF02494FF0F4
:10BE2000000000F06EBD00BF0000F87F491058BF51
:10BE3000C1F140415B1058BFC3F140438B42EFF367
:10BE4000008070472DE9C04130B4DFF8A0C23CEA61
:10BE5000111418BF3CEA131400F0EC8081EA0305CA
:10BE60001CEA111444EAD57418BF1CEA131500F03B
:10BE7000C780A4EB05044FF0004545EAC12145EA1F
:10BE8000C32341EA505143EA525304F17F7499426B
:10BE900004F500344FEAC0204FEAC22208BF9042A6
:10BEA00000F09C804FEA13650FF24016765D4FEA72
:10BEB000134506FB05F7C7F1807706FB07F74FEA46
:10BEC000D737A7FB03687642C8F58038A7FB06CEB4
:10BED00038BFA8F1010807FB08E64FF0000EA6FBEB
:10BEE000028CE6FB03CEDCF1000CCEF1004E38BF35
:10BEF000AEF1010EA6FB0C584FF000074FF0000505
:10BF0000E6FB0E87A1FB08C6A0FB07CE16EB0E06CC
:10BF100045F10005E1FB076515F1E04E7EBFA4F594
:10BF200080345FEA46066D4116F1800745F1000551
:10BF30004FEA17274FEA066647EA0567A6F1DE468D
:10BF4000B6F1805F4FEA15251FD9384624F0010C61
:10BF500005EBC471BCF1FE6F01EB0C1102D8F0BC13
:10BF6000BDE8008124425CBF01F5801E9EEAC47FCB
:10BF700002D4F0BCBDE80081244238D4F0BCA1F169
:10BF8000C041BDE8004100F043BA4FEAD22242EA84
:10BF900043524FEAD323A7FB02864FEAD02040EA60
:10BFA000415007FB03661EEA0E0F4FEAD12105FB45
:10BFB000026658BFA6EB0056B6EB00564FEA520E8B
:10BFC0004EEAC37E18EB0E0E56EB530EBDD518EBA2
:10BFD00002085E417F1C55F10005B6E74FF480155D
:10BFE0004FF000074FF000064FF00008ADE7F0BC3F
:10BFF0004FF0000001F1C04101F00041BDE80081B7
:10C0000011EA0C1F0CEA131500D00CE013EA0C1F08
:10C0100000F025804FF00000F0BC81EA030101F040
:10C020000041BDE80081F0BCBDE8004181EA0301A8
:10C0300000F0EEB9F0BCBDE8004170B500F09AF92F
:10C04000097EFC3E00F007B881EA03014FF00000D2
:10C0500001F00041704781EA030100F0D9B9F0BC5A
:10C06000BDE800414FF0000021497047FFFDFBF99A
:10C07000F7F5F4F2F0EEEDEBE9E8E6E4E3E1E0DE1B
:10C08000DDDBDAD8D7D5D4D3D1D0CFCDCCCBCAC88D
:10C09000C7C6C5C4C2C1C0BFBEBDBCBBBAB9B8B7B4
:10C0A000B6B5B4B3B2B1B0AFAEADACABAAA9A8A8A7
:10C0B000A7A6A5A4A3A3A2A1A09F9F9E9D9C9C9B75
:10C0C0009A99999897979695959493939291919020
:10C0D0008F8F8E8E8D8C8C8B8B8A898988888787B1
:10C0E0008685858484838382828181800000FF0726
:10C0F0000000F87F4FEA41034FEA5353A3F58063F2
:10C10000D3F11E03C8BFD3F1210C0CDD4FF0004268
:10C1100042EAC12242EA505232FA03FC8CEAE17C44
:10C12000ACEBE1707047102BC4BF0020704703F5E3
:10C13000787CBCF1FF3F04D06FF0004282EA21001E
:10C14000704770B500F016F94992248000207047BE
:10C15000F2E710F0004248BF4042B0FA80F310FA14
:10C1600003F10AD0C3F11D0303F580634FEA415088
:10C1700002EB035202EBD12170474FF000007047F1
:10C18000B0FA80F310FA03F10AD0C3F11D0303F5EE
:10C1900080634FEA41504FEA035202EBD1217047CE
:10C1A0004FF000007047000051EA030C17D41CF553
:10C1B000801F58BFBCF5801F00F10680994218BF50
:10C1C000704708BF9042704707D711F5801F58BFCE
:10C1D00013F5801F19D499427047894270471CF5A6
:10C1E000801F08D5BCF5801FF7D58B4218BF70475C
:10C1F00008BF824270474FF4001C1CEB410F38BF50
:10C200001CEB430F01D28B42704770B500F0B2F8BF
:10C21000922449004FF000514FF08053FFF706BEC3
:10C22000DFF848C170B51CEA111E1EBF1CEA1315C9
:10C230009EEA0C0F95EA0C0F00F06F8081EA030470
:10C2400023EA4C134EEAD47E21EA4C1141F48011CA
:10C2500043F48013AE44A1FB024CA0FB0365AEF196
:10C260007F7E361955EB0C05A1FB034C4CF1000306
:10C27000A0FB021C16EB0C06654153F100030942BA
:10C2800018BF46F0010613F4007F0BD14FEA0331CB
:10C290004FEA0530340341EA155140EA16506FF079
:10C2A00003020AE04FEAC3214FEAC520F40241EA43
:10C2B000555140EA56506FF0020202EB2E4201EB5C
:10C2C000025585EACE710AD05FEA440C18BF24F00B
:10C2D000004450F1000041F1000120EAD47040F226
:10C2E000FE7C624500D270BDA84214BF4FF080446E
:10C2F0004FF04044002E08BF0024BEF1806FA8BF5D
:10C30000A1F1C041BDE8704080F282804FF0000092
:10C3100001F1C04101F0004170479EEA0C0F0CEAA8
:10C32000131518BF95EA0C0F06D04FF0000081EAF4
:10C33000030E0EF0004170BD00F01CF88900013EB4
:10C3400000F007B800F009B84FEA430C5FEA5C5C04
:10C3500008D081EA030100F05BB84FEA410C5FEAC4
:10C360005C5CF6D14FF00000014970470000FF0708
:10C370000000F87F0EF1020E2EF0030E5EF8046B43
:10C38000364205D4012A43EB030515F5001F12D8E8
:10C39000012841EB010C1CF5001F0CD80ED14FEA0F
:10C3A000D17C15F5001F0CEB4C0C0CF1020C08BFF6
:10C3B0004CEBD37C04E04FF0080C01E04FEAD37C57
:10C3C0000CEB4C0526FA05F606F00706B6F1040C50
:10C3D00006D20EEB860CBDE870404CF0010C6047B5
:10C3E000DFE80CF0090B02024FF000414FF00000B3
:10C3F000A1F5002170BD19461046012851EB01043A
:10C4000018BFD4F5001484BF002001F0004170BDB6
:10C410000808A0F500114FEA3101704753EA010CFA
:10C4200017D41CF5801F58BFBCF5801F00F1068093
:10C430008B4218BF704708BF8242704707D713F579
:10C44000801F58BF11F5801F19D48B4270479B4243
:10C4500070471CF5801F08D5BCF5801FF7D59942A1
:10C4600018BF704708BF904270474FF4001C1CEB88
:10C47000430F38BF1CEB410F01D2994270470FB4F4
:10C480000CBC03BCFFF7C1BE91EA030F10B581F0ED
:10C4900000413FF523AC83F0004300F0D5B8000025
:10C4A0002DE9F04101F5801CBCF5001FC0F2A98008
:10C4B0004FEA115C21EA0C510CF1FD0C41F48011A2
:10C4C0005FEA5C0C0CF5C07C01D34000494130A40C
:10C4D000890241EA905187028E0E0A0CA45D04FB8A
:10C4E00004F602FB06F6C6F14046A4FB0662F60D12
:10C4F00046EA422606FB06F4A4FB01235242C3F19E
:10C50000404338BF5B1EA6FB02420024E6FB032427
:10C51000D20B42EA4446A6FB0623A1FB02E2A3FBA0
:10C5200007E4E3FB61426442C2F1404E38BFAEF122
:10C53000010EA6FB04234FF00002E6FB0E32A2FB25
:10C5400003463400E2FB6264A1FB06E6A4FB07E8B5
:10C55000E4FB61687642C8F1405838BFA8F1010891
:10C56000A2FB06E4A3FB08E5E2FB6854A1FB05E699
:10C57000A7FB04E8E1FB648618F1200556F10006EC
:10C58000A809A8F11B08B10908F03F08B8F10A0F83
:10C5900040EA86601CD901EB0C51BDE8F08100BF78
:10C5A000FCF5EEE8E2DDD8D3CFCBC7C3C0BDB9B64A
:10C5B000B4B1AEACA9A7A5A3A19F9D9B9A9896954F
:10C5C0009392908F8D8C8B898887868584838281D6
:10C5D000A0FB006800FB01F208EB4208B8EB8728DB
:10C5E00007D5341858EB0104D5D5401C51F1000192
:10C5F000D1E7341A78EB0104CDD4401E71F100016B
:10C60000C9E75FEA4C0C5FEA9C5C0DD105D34FF0A3
:10C61000000001F00041BDE8F081BDE8F04170B5D7
:10C62000FFF7A8FE6DDBFFBEBDE8F0414FF0000054
:10C63000004970470000F87F10B591EA030F48BF2A
:10C6400083F000433FF54AAB841A71EB030C07D229
:10C6500012198CF0004C43EB0C03001B61EB0C0136
:10C66000DFF8A4E14FEA1154A4EB135C1EEA430F78
:10C6700018BF9EEA445F00F0B08023EA6E03524286
:10C6800021EA0451C3EB6E0338BF5B1EDCF1200EC0
:10C6900025D322FA0CFE10EB0E0043FA0CFE41EB00
:10C6A0000E01CCF1200E03FA0EFE10EB0E0051F13C
:10C6B0000001CCF1200E29D412FA0EF201EB045144
:10C6C000BDE8104058BF7047401C1CBFB2F1004F7E
:10C6D000704700280CBF491C20F00100704712EB86
:10C6E000020E43EB030218BF4FF0010E4EEA420266
:10C6F000ACF1200CDCF11E0E54D943FA0CFE10EB09
:10C700000E0051F1FF31CCF11E0ED5D50EF1010E08
:10C7100012FA0EFE404141EB010101EB445C5FEA7D
:10C720005C5C10D910EBDE7001EB045138BFBEF138
:10C73000004FBDE8104018BF704700280CBF491CCF
:10C7400020F00100704730D24FEAD42C11F50011CF
:10C7500024F400641BD0B1FA81F20B3AA41AA41E8F
:10C76000D2F12003914030FA03F31943904001EBDA
:10C77000CC71002C01EB0451BDE81040A8BF7047FC
:10C7800001F1C0414FF0000001F000417047B0FAE4
:10C7900080F310FA03F100D110BDE41A173C4805EC
:10C7A000C90AE4E701EB045110BD491001EB045143
:10C7B000BDE810404FEA300002E04FF00001704742
:10C7C0004A0008BF0042F8D0B2F5001F28BF7047EA
:10C7D00001F000414FF0000070479EEA445F07D02F
:10C7E00011EA5E0FBDE8104004BF00210020704731
:10C7F000BDE8104070B5FFF7BDFD00BF40DFF63E5D
:10C8000083F00041104670470000E0FF43004FEA0C
:10C81000D30C4FEA3C0C43401FBF40070CF1605162
:10C8200013F0FE4F70471CF0006F03D100200CF096
:10C83000004170470CF0004343EA507010B540EAE5
:10C84000CC0000F00EF800BF000000924FEA00019B
:10C85000FFF7DEBD4FF000414FF00000A1F50021D1
:10C8600070470EF1020E2EF0030E5EF8044B2442C8
:10C8700004D44FEA4102B2F17F4F11D84FEA40038E
:10C88000B3F17F4F0CD80ED14FEAD07CB2F17F4F7D
:10C890000CEB4C0C0CF1020C08BF4CEBD17C04E00F
:10C8A0004FF0080C01E04FEAD17C0CEB4C0324FA6A
:10C8B00003F404F00704B4F1040C06D20EEB840C6C
:10C8C000BDE810404CF0010C6047DFE80CF00708B1
:10C8D00002024FF00040A0F5800010BD0846420063
:10C8E00018BFD2F1807288BF00F0004010BD4FF039
:10C8F0004070E1EE100A7047FF2141EAD050C005B8
:10C9000070470CF00F03092B08BF082000F0598076
:10C910000A2B0BD0082B18BF704708BF1CF0400F24
:10C920000AD04FF000004FF0000170471CF0400F9C
:10C9300018BF4FF0004070471CF0100F08D020F0D7
:10C94000704300F07F4242EAD3014FEA43707047E0
:10C9500000F0604021F07F4242EA000201F07F4097
:10C9600040EA727070474FF0FF0C4CF4E06C1CEA28
:10C9700011531CBF9CEA030C9445C2BFDA4201EB81
:10C9800002517047002B0DD0BCF1000F0FD0002AD0
:10C9900001F00041A4BF41F0E04141F07F614FF060
:10C9A0000000704701F000414FF00000704750EA6E
:10C9B00001334FF09B0C18BF4CF0806C7FF42EAA13
:10C9C00070471CF4801F11D01CF4E02F03D06FEAD5
:10C9D000CC31490070474FF04050EFF3008222F015
:10C9E000704242EA000282F3008870474FF0000074
:10C9F0007047000000000000000000000000000080
:10CA000000003F4000000000000000003000400037
:10CA100030004000000009000BC03D000BC03D008D
:10CA2000090018C024407FE0224031800000180037
:10CA300024C01B000D803240018003801C40274031
:10CA40001C80074000401000600000000000000053
:10CA500000000000000000001F8020404020000077
:10CA6000402020401F8000000000090006001F80B9
:10CA7000060009000000040004003F8004000400D8
:10CA80000000001000600000000000000000040032
:10CA90000400040004000400000000000040000046
:10CAA000000000000000002001C006003800400027
:10CAB00000001F802040204020401F800000000018
:10CAC00010403FC000400000000018C0214022403C
:10CAD00024401840000010802040244024401B8047
:10CAE000000002000D0011003FC0014000003C802A
:10CAF000244024402440238000001F802440244000
:10CB00003440038000003000200027C0380020009F
:10CB100000001B802440244024401B8000001C0097
:10CB200022C0224022401F80000000000000084078
:10CB30000000000000000000000004600000000091
:10CB40000000000004000A0011002080404009009D
:10CB50000900090009000900000000004040208091
:10CB600011000A00040018002000234024001800CF
:10CB700000001F802040274029401F400000004047
:10CB800007C039000F0001C0004020403FC02440D2
:10CB900024401B8000001F80204020402040308027
:10CBA000000020403FC0204020401F800000204067
:10CBB0003FC024402E4030C0000020403FC02440F1
:10CBC0002E00300000000F001080204022403380F3
:10CBD000020020403FC0040004003FC0204020402D
:10CBE00020403FC020402040000000602020202046
:10CBF0003FC02000200020403FC024400B0030C038
:10CC0000204020403FC020400040004000C03FC0C6
:10CC10003C0003C03C003FC0000020403FC00C402F
:10CC200023003FC020001F802040204020401F8064
:10CC3000000020403FC024402400180000001F8056
:10CC40002140214020E01FA0000020403FC02440A0
:10CC5000260019C0004018C02440244022403180E2
:10CC60000000300020403FC0204030000000200085
:10CC70003F80004000403F80200020003E0001C077
:10CC8000070038002000380007C03C0007C038000B
:10CC90000000204039C0060039C0204000002000BC
:10CCA000384007C0384020000000304021C02640F6
:10CCB000384020C00000000000007FE040204020FD
:10CCC0000000000070000C00038000400000000025
:10CCD000402040207FE000000000000020004000D5
:10CCE00020000000000000100010001000100010D4
:10CCF00000100000000040000000000000000000E4
:10CD000002800540054003C0004020003FC00440B1
:10CD100004400380000000000380044004400640FB
:10CD2000000000000380044024403FC00040000099
:10CD300003800540054003400000000004401FC080
:10CD4000244024402000000002E005500550065019
:10CD5000042020403FC00440040003C00040000005
:10CD6000044027C000400000000000100010041024
:10CD700027E00000000020403FC00140070004C041
:10CD80000440204020403FC000400040000007C059
:10CD9000040007C0040003C00000044007C00440B2
:10CDA000040003C0004000000380044004400380EE
:10CDB0000000041007F0045004400380000000004D
:10CDC00003800440045007F00010044007C00240F4
:10CDD000040004000000000006400540054004C0B7
:10CDE0000000000004001F80044000400000040018
:10CDF00007800040044007C000400400070004C052
:10CE0000018006000400060001C0070001C0060002
:10CE10000000044006C0010006C0044000000410E9
:10CE2000071004E00180060004000000044005C073
:10CE30000640044000000000000004007BE04020A9
:10CE40000000000000000000FFF0000000000000F3
:10CE500040207BE004000000000040008000400013
:10CE60002000200040000000000000000000000042
:10CE70000000000000000000000000001FCC000CBB
:10CE80000000000000000000080030006000080002
:10CE9000300060000000022003FC1E20022003FC82
:10CEA0001E200220000000000E1811043FFF108415
:10CEB0000C78000000000F0010840F3800C00778C5
:10CEC00018840078000000780F8410C411240E9894
:10CED00000E4008400080800680070000000000002
:10CEE00000000000000000000000000007E018182B
:10CEF000200440020000000040022004181807E04F
:10CF00000000000000000240024001800FF001809C
:10CF10000240024000000080008000800FF8008086
:10CF20000080008000000001000D000E00000000E5
:10CF300000000000000000000080008000800080F1
:10CF40000080008000800000000C000C0000000049
:10CF500000000000000000000006001800600180D2
:10CF6000060018002000000007F008081004100454
:10CF7000080807F000000000080408041FFC000473
:10CF800000040000000000000E0C101410241044D7
:10CF900011840E0C000000000C1810041104110480
:10CFA00012880C700000000000E003200424082414
:10CFB0001FFC0024000000001F98108411041104BD
:10CFC000108810700000000007F008881104110498
:10CFD00018880070000000001C00100010FC1300F6
:10CFE0001C001000000000000E3811441084108452
:10CFF00011440E38000000000700088C1044104453
:10D00000088807F00000000000000000030C030C7B
:10D010000000000000000000000000010106000008
:10D020000000000000000000008001400220041009
:10D030000808100400000220022002200220022022
:10D040000220022000000000100408080410022042
:10D0500001400080000000000E001200100C106C57
:10D0600010800F00000003E00C1813E4142417C410
:10D07000082807D000000004003C03C41C400740FF
:10D0800000E4001C000410041FFC1104110411042E
:10D090000E880070000003E00C1810041004100447
:10D0A00010081C10000010041FFC100410041004D1
:10D0B000080807F0000010041FFC1104110417C435
:10D0C00010040818000010041FFC1104110017C000
:10D0D00010000800000003E00C18100410041044B5
:10D0E0001C780040000010041FFC108400800080A9
:10D0F00010841FFC10040000100410041FFC100416
:10D1000010040000000000030001100110011FFEC8
:10D1100010001000000010041FFC110403801464B0
:10D12000181C1004000010041FFC1004000400046C
:10D130000004000C000010041FFC1F0000FC1F0076
:10D140001FFC1004000010041FFC0C04030000E08E
:10D1500010181FFC100007F0080810041004100439
:10D16000080807F0000010041FFC108410801080D5
:10D1700010800F00000007F0081810241024101C65
:10D18000080A07F2000010041FFC1104110011C06E
:10D1900011300E0C000400000E1C110410841084C9
:10D1A00010441C3800001800100010041FFC10046C
:10D1B00010001800000010001FF810040004000404
:10D1C00010041FF8100010001E0011E0001C007079
:10D1D00013801C0010001FC0103C00E01F0000E086
:10D1E000103C1FC000001004180C163401C001C010
:10D1F0001634180C100410001C00130400FC130457
:10D200001C00100000000804101C1064108413049B
:10D210001C04101800000000000000007FFE400207
:10D22000400240020000000030000C00038000605B
:10D23000001C0003000000004002400240027FFE8C
:10D24000000000000000000000002000400040003E
:10D250004000200000000001000100010001000169
:10D26000000100010001000040004000200000001B
:10D270000000000000000000009801240144014467
:10D28000014400FC000410001FFC0088010401049C
:10D290000088007000000000007000880104010494
:10D2A00001040088000000000070008801040104EF
:10D2B00011081FFC0004000000F80144014401446F
:10D2C000014400C800000000010401040FFC110427
:10D2D000110411001800000000D6012901290129BC
:10D2E00001C90106000010041FFC008401000100B8
:10D2F000010400FC000400000104190419FC0004EE
:10D3000000040000000000000003000101011901F9
:10D3100019FE0000000010041FFC0024004001B4AE
:10D32000010C010400000000100410041FFC0004A4
:10D33000000400000000010401FC0104010001FCE4
:10D340000104010000FC010401FC00840100010053
:10D35000010400FC0004000000F8010401040104C1
:10D36000010400F80000010101FF0085010401042F
:10D3700000880070000000000070008801040104B3
:10D38000010501FF00010104010401FC0084010406
:10D39000010001800000000000CC012401240124D0
:10D3A00001240198000000000100010007F80104B9
:10D3B000010400000000010001F800040004000462
:10D3C000010801FC0004010001800170000C001044
:10D3D00001600180010001F0010C003001C000304B
:10D3E000010C01F0010000000104018C00740170C7
:10D3F000018C01040000010101810171000E00187F
:10D4000001600180010000000184010C013401442D
:10D410000184010C00000000000000000000010079
:10D420003EFC400240020000000000000000FFFF40
:10D430000000000000000000400240023EFC01002D
:10D44000000000000000000060008000800040003C
:10D45000400020002000404281FE00000121D21443
:10D460000814E2010000080808FF090419111197C7
:10D47000711111151900000000000000FF000000EC
:10D480000080600000004040404040407F404042FB
:10D490004140404040000106F840404040FE4040CE
:10D4A0004241FE00000000007F444444447F444465
:10D4B00044447F000000000106F880808080808066
:10D4C0008080C00000000000001F1010907010103D
:10D4D00010101F000000404281FE00000121D21404
:10D4E0000814E2010000080808FF09041911119747
:10D4F0007111111519008080FE848A6418E422A23B
:10D50000A2FAA2A22200020CF72424012739082A39
:10D510002AFF2A3E08004080FE0808FC0106F89019
:10D5200090FC9291FE002021273A2223040817E460
:10D5300024272C340700000000FC09120418E00026
:10D54000E01804020100020242330000000000FF64
:10D550000000000000000001020CF00000000000CC
:10D56000FF0000000000014141417F414141414134
:10D570007F41414101000244A810688400007F42BD
:10D580004242427F000008080FF8080F0002071A05
:10D59000E2020A060300000000FF222222222222C9
:10D5A00022FF000000000000001F113151911111F5
:10D5B000111F0000000020C000FF0082221A8272AA
:10D5C000061AE202020008080BFF090A040A32C226
:10D5D000320A040202000102040830C00000FC020A
:10D5E0000202020E00000002424242437E424342D7
:10D5F0004242020200004241FE8222A4A8B0A07F63
:10D60000B0A8A4A222000808FF080907F494979084
:10D610009794F4070000800000FF00000000FF1056
:10D620001010101000000001061FE0020CF01F1186
:10D63000111111101000106080FF80608101020242
:10D64000E40830C000002424257FC44400031C00EB
:10D65000FF0010080600020418E0007F4242424228
:10D6600042427F0000000000003F24242424444460
:10D6700044C444040400000204F80402FA12220222
:10D680008242A21A0200020242330000FF929293E9
:10D690009292FE010000003E0202020202FE02021D
:10D6A0000202023F000000003E02020202FF0202EC
:10D6B00002023F000000020202FE020202FE02021B
:10D6C000020202020200004040434040407F4141CC
:10D6D000414141400000408000FF0282828282FE80
:10D6E000828282820200101011131C30D010101799
:10D6F000101010101000000000FF2222222222220F
:10D7000022FF000000000000001F11315191111193
:10D71000111F0000000020C000FF0082221A827248
:10D72000061AE202020008080BFF090A040A32C2C4
:10D73000320A0402020000001A1C0000000000006F
:10D7400000000000000000000000000000000000D9
:10D75000000000000000106080FF80608101020274
:10D76000E40830C000002424257FC44400031C00CA
:10D77000FF0010080600020418E0007F4242424207
:10D7800042427F0000000000003F2424242444443F
:10D7900044C444040400008181828CF0808080FEB7
:10D7A0008181818F0000083020242424A464242453
:10D7B0002424202830000106F8000804F80102841F
:10D7C000681864821F0000001F111111111010FF52
:10D7D000109050131000101810FF202000FF42423C
:10D7E000FE4242FF0000131DF1171111000F08083F
:10D7F000FF08080F00000106F890909090FE9090AE
:10D800009291FE00000004081724E4242427242C0D
:10D81000340407000000000204F80412224282FAD5
:10D820008242221202000202423300202F2929FFE5
:10D8300029292F200000020CF1012132AAA4A4A45E
:10D84000AA320101010000003F2424243FA46424E3
:10D850003F2424242000000000FF22222222222232
:10D8600022FF000000000000001F11315191111132
:10D87000111F0000000020C000FF0082221A8272E7
:10D88000061AE202020008080BFF090A040A32C263
:10D89000320A04020200008181828CF0808080FEC6
:10D8A0008181818F0000083020242424A464242452
:10D8B0002424202830000106F8000804F80102841E
:10D8C000681864821F0000001F111111111010FF51
:10D8D0001090501310008080FE848800FF92929276
:10D8E0009292FF000000020CF724261212FE121280
:10D8F00012FE121202000000FE042921222428F048
:10D90000282422212100024233000001794949499B
:10D91000494979010000800000FF0000000000C0BC
:10D92000300804021F000001061FE0040404FE0585
:10D930000888680808004080FE0808FC00101010E5
:10D9400010121102FC002021273A222300404F41EF
:10D9500041417F0101000000F810101010FE11116C
:10D960001111F9010F0000001F11111111FF111108
:10D9700011111F0000000106F80202020202FE025D
:10D9800002221A02020000007F40414141415F41F2
:10D99000414141414000000204F8040202820212A7
:10D9A0000AF20202020002024233001012111010A9
:10D9B00010FF10101000800000FF0000FF020400A4
:10D9C00082710C021F000001061FE0003F2121218F
:10D9D0007F41C14101000000FF000181A29488F451
:10D9E00082828181010001061FE02027242424FF78
:10D9F00024242427200000FF48484A49FE00007ED6
:10DA0000111121410700103352921252331800FEB7
:10DA10001111214107000001020CF000000000007C
:10DA2000FF0000000000014141417F41414141416F
:10DA30007F4141410100818182828488B0C0B088E9
:10DA4000848282818100000008886808080F080825
:10DA500028C808000000818182828488B0C0B08814
:10DA6000848282818100000008886808080F080805
:10DA700028C80800000000FF001020408804F800BB
:10DA8000000201FE0000001F8044044444455F443E
:10DA90004444407F00001018122122FC00FE0A12AC
:10DAA0006282621A0200405F41417F01007F40486C
:10DAB000464146584000083CC808281D020C7080AA
:10DAC000020102FC0000022223222222020808FF97
:10DAD0000808080F000044E644484848020204C809
:10DAE000302844821F00040C35C60418010909FFC0
:10DAF000099252120200020CF1010202C4281028FD
:10DB000044820201010000003F24242724244444CD
:10DB100044C546000000202241FE804141526AC4B3
:10DB2000444A72414000080808FF080A222AA663F6
:10DB300022262A2202001018122122FC00FE0A12BC
:10DB40006282621A0200405F41417F01007F4048CB
:10DB5000464146584000083CC808281D020C708009
:10DB6000020102FC0000022223222222020808FFF6
:10DB70000808080F0000202241FE800001F1020C7D
:10DB8000F00804F30000080808FF080900037A4AB7
:10DB90004A4A7A030000101810E020281020408024
:10DBA000FF0000C03000040404FF040420202021F2
:10DBB00027382120200044E644484A1CE0FF90FE1C
:10DBC00090FC91FF0000040C35C60C003F24A464B7
:10DBD0002424243C00004080FE0808FC00101010A3
:10DBE00010121102FC002021273A222300404F414D
:10DBF00041417F01010010102F2949498F00804FBA
:10DC00004929291F100001017949494979070179FA
:10DC10004D4B49790100202241FE800001F1020CA8
:10DC2000F00804F30000080808FF080900037A4A16
:10DC30004A4A7A030000101810E020281020408083
:10DC4000FF0000C03000040404FF04042020202151
:10DC50002738212020000000F810101010FE1111AC
:10DC60001111F9010F0000001F11111111FF111105
:10DC700011111F00000020207E820CF004C8928148
:10DC8000FE8090C8040008064031007F404F4A5A89
:10DC90006A4A4A4F400008102040800000FF000000
:10DCA000008040300000004040404041424F704200
:10DCB000414040400000106080FF00C10620263136
:10DCC0002D2123E806002424257FC544102949C9B5
:10DCD0004959690F000001020478040202FE222261
:10DCE000222222020200083022222222A2632222C1
:10DCF00022222228300020207E80027E42427E4264
:10DD00007E42427E02000806403100007F494949B8
:10DD100049497F000000020CF1012132AAA4A4A409
:10DD2000AA320101010000003F2424243FA46424FE
:10DD30003F2424242000000204F80402028202127C
:10DD40000AF2020202000202423300101211101005
:10DD500010FF10101000007F40405E52525252528D
:10DD60005E40417F0000202020202F29A969292919
:10DD70002F20202020000000F810101010FE11119C
:10DD80001111F9010F0000001F11111111FF1111E4
:10DD900011111F00000020C000FF00C106F80000A4
:10DDA00000FC02021E0008080BFF0908007F40402B
:10DDB000407F0000000044E644484848020204C88E
:10DDC000302844821F00040C35C60418010909FFDD
:10DDD000099252120200202241FE804141526AC43F
:10DDE000444A72414000080808FF080A222AA66334
:10DDF00022262A2202008080FE848800FF929292CE
:10DE00009292FF000000020CF724261212FE12125A
:10DE100012FE121202001020C000000201FE0000DB
:10DE200000000080700000000007000000FF0000FC
:10DE300000040201000010109090909090FF9090CC
:10DE4000909090101000001011121418F01710107C
:10DE5000101010100000020202FE020202FE020276
:10DE6000020202020200004040434040407F414124
:10DE700041414140000000007C40404040FF4040A4
:10DE800048447800000004181057351515F515158D
:10DE900035571014180000004FBB610567ACDD3F1B
:10DEA000182D4454FB21E93F9BF681D20B73EF3FC1
:10DEB000182D4454FB21F93FE2652F227F2B7A3C39
:10DEC000075C143326A6813CBDCBF07A8807703CF2
:10DED000075C143326A6913CC4EB98999999C9BF65
:10DEE000711623FEC671BCBF6D9A74AFF2B0B3BF9A
:10DEF0009AFDDE522DDEADBF2F6C6A2C44B4A2BF5A
:10DF00000D5555555555D53FFF8300922449C23FC5
:10DF10006E204CC5CD45B73F513DD0A0660DB13FF9
:10DF2000EB0D76244B7BA93F11DA22E33AAD903F0B
:10DF3000000000000000F03F000000000000F83F7B
:10DF400000000000000000000000004003B8E23FB5
:10DF5000000000000000000006D0CF43EBFD4C3E67
:10DF6000033333333333E33FFFAB6FDBB66DDB3F5C
:10DF70004D268F515555D53F01411DA96074D13FA4
:10DF800065DBC9934A86CD3FEF4E454A287ECA3F9E
:10DF90003E5555555555C53F93BDBE166CC166BF20
:10DFA0002CDE25AF6A56113FF16BD2C541BDBBBE19
:10DFB000D0A4BE726937663E000000000000000079
:10DFC00000004054FB21F93F3163621A61B4D03D37
:10DFD0000000601A61B4D03D7370032E8A19A33B10
:10DFE0000000002E8A19A33BC14920259A837B3962
:10DFF00000000000000000006E83F9A22915444EC5
:10E00000D15727FCC0DD34F5999562DB4190433C44
:10E01000AB6351FE61C5BBDE3A6E24B7E0D24D4220
:10E02000EA2E49061C92D1091CEB1DFE3EA729B120
:10E03000F53582E88444BB2E26709CE9417E5FB4AE
:10E0400039D69139F43953838B5F849C3B28F9BDD1
:10E05000FF97F81F0F9805DE8B112FEF1F6D0A5ADF
:10E06000CF7E366DB709CB27663F464F2DEA5F9EC0
:10E07000C7BA27757BF1E5EBF739073DEA92528A7B
:10E08000B15FFB6B085D8D1F7AFE10111111C13F4E
:10E0900037D60684F464963F280356C9226D6D3F37
:10E0A0000165F2F2D844433FA69237A0887E143F20
:10E0B000735360DBCB75F3BEFE41B31BBAA1AB3F1C
:10E0C00093846EE9E326823F1583E0FEC8DB573F69
:10E0D00068108D1AF726303FE9A7F0320FB8123FCB
:10E0E000D47ABF74702AFB3E08E1000800000020CB
:10E0F00080020000C40100086CE1000880020020DA
:10E10000D05E00002002000851847A030AC0090191
:10E11000020304060708090213017AF415140142E8
:10E12000011202120312041205120612071208123B
:10E1300009120A120B120C120D120E120F022D10E0
:10E140000B1CDC0504012A29CA0912CE01461AAAB1
:10E1500001091F82719204E3FA431A9610038C4856
:0CE1600044B264024D190314803F00001B
:040000050800018965
:00000001FF
